:10000000C0250020CD4500001D950000A145000041
:10001000A1450000A1450000A1450000000000002E
:10002000000000000000000000000000A5420000E9
:10003000A1450000000000004D420000A145000065
:100040006143000061430000614300006143000020
:100050006143000061430000614300006143000010
:100060006143000061430000614300006143000000
:1000700061430000614300006143000061430000F0
:1000800061430000614300006143000061430000E0
:1000900061430000614300006143000061430000D0
:1000A00061430000614300006143000061430000C0
:1000B00061430000614300006143000061430000B0
:1000C00061430000614300006143000061430000A0
:1000D0006143000061430000614300006143000090
:1000E0006143000061430000614300006143000080
:1000F0006143000061430000614300006143000070
:1001000053B94AB9002908BF00281CBF4FF0FF317E
:100110004FF0FF3000F06CB9ADF1080C6DE904CE82
:1001200000F006F8DDF804E0DDE9022304B07047D2
:100130002DE9F047089E0D4604468E46002B40F000
:1001400082808A42174646D9B2FA82F24AB1C2F197
:10015000200105FA02F320FA01F1974041EA030E6B
:1001600094404FEA1748230CBEFBF8FCB9B208FBD9
:100170001CEE43EA0E430CFB01F098420AD9FB182F
:100180000CF1FF3580F01681984240F21381ACF1FA
:10019000020C3B441B1AA4B2B3FBF8F008FB10336B
:1001A00044EA034400FB01F1A14209D93C1900F1E2
:1001B000FF3380F00181A14240F2FE8002383C44CE
:1001C000641A40EA0C4000211EB1D4400023C6E965
:1001D0000043BDE8F08702B9FFDEB2FA82F2002ADE
:1001E0004FD1CB1B4FEA174E1FFA87F80121B3FB03
:1001F000FEFC250C0EFB1C3345EA034508FB0CF303
:10020000AB4207D97D190CF1FF3002D2AB4200F2AC
:10021000E7808446ED1AA3B2B5FBFEF00EFB105545
:1002200043EA054408FB00F8A04507D93C1900F152
:10023000FF3302D2A04500F2D7801846A4EB080491
:1002400040EA0C40C0E78B4208D9002E00F0AF8096
:100250000021C6E900050846BDE8F087B3FA83F13E
:1002600000294BD1AB4202D3824200F2B780841AFC
:1002700065EB030301209E46002EAAD0C6E9004E7E
:10028000A7E7C2F1200C01FA02F3974020FA0CF024
:100290004FEA174E21FA0CFC1843BCFBFEF1050C8B
:1002A0000EFB11CC1FFA87F845EA0C4501FB08F359
:1002B000AB4204FA02F409D97D1901F1FF3C80F048
:1002C0008B80AB4240F2888002393D44EB1A85B204
:1002D000B3FBFEF00EFB103345EA034500FB08F3C9
:1002E000AB4207D97D1900F1FF3C71D2AB426FD907
:1002F00002383D44EB1A40EA014178E7C1F1200C95
:100300008B4022FA0CF71F4320FA0CF405FA01F394
:100310004FEA174E25FA0CF51C43230CB5FBFEF9EA
:100320001FFA87F80EFB195543EA054509FB08FA41
:10033000AA4502FA01F200FA01F308D97D1909F180
:10034000FF3047D2AA4545D9A9F102093D44A5EBA2
:100350000A05A4B2B5FBFEF00EFB105544EA0544B5
:1003600000FB08F8A04507D93C1900F1FF352DD254
:10037000A0452BD902383C4440EA0940A4EB0804CC
:10038000A0FB02894C45C6464D4619D316D05EB136
:10039000B3EB0E0264EB050404FA0CFCCA404CEA11
:1003A0000202CC40C6E900240021BDE8F0873146B6
:1003B00030460EE7AC46EDE6184601E74345E6D287
:1003C000B8EB020E69EB07050138E0E72846D3E7F2
:1003D00060468FE78146BAE7614677E708464BE714
:1003E000ACF1020C3D4415E702383C4426E700BF5F
:1003F000704700BF1FB5124807F0C7FD002004F08A
:1004000051FC18B90F4807F0C0FD0CE00023019320
:10041000039369460123029307F033FE011E05DAB8
:10042000094807F0B2FD05B05DF804FB029B9B078D
:10043000FCD1039909B10548F3E70548E3E700BF9C
:1004400054B2000071B2000092B20000ACB20000E1
:10045000CCB2000008B5054B0F225A700821044B9E
:10046000044A08F0C8FA002008BD00BF00000020C0
:10047000DFB2000001B3000008B5054B06225A7038
:100480000821044B044A08F0B6FA002008BD00BF5A
:100490000000002010B3000001B3000008B5054BB8
:1004A00005225A700821044B044A08F0A4FA0020DF
:1004B00008BD00BF000000202DB3000001B3000004
:1004C00008B5054B04225A700821044B044A08F071
:1004D00092FA002008BD00BF000000204AB30000CF
:1004E00001B3000008B5054B03225A700821044BE4
:1004F000044A08F080FA002008BD00BF0000002078
:1005000063B3000001B3000008B5054B01225A7027
:100510000821044B044A08F06EFA002008BD00BF11
:10052000000000207CB3000001B3000010B5054BB3
:10053000054A00245C700821044B08F05CFA204650
:1005400010BD00BF0000002001B3000095B3000003
:10055000034BD8229A700821024B034A08F04BBA89
:1005600000000020AEB30000CDB30000034BE22238
:100570009A700821024B034A08F03DBA000000209F
:10058000DBB30000CDB30000034BEC229A700821CE
:10059000024B034A08F02FBA00000020FAB3000013
:1005A000CDB30000034BF0229A700821024B034A9E
:1005B00008F021BA0000002019B40000CDB30000FB
:1005C000034BF4229A700821024B034A08F013BA35
:1005D0000000002038B40000CDB30000034BF82227
:1005E0009A700821024B034A08F005BA0000002067
:1005F00057B40000CDB30000034BFC229A700821D1
:10060000024B034A08F0F7B90000002075B400005F
:10061000CDB30000034B00229A700821024B034A1D
:1006200008F0E9B90000002093B40000CDB3000049
:10063000034B02229A700821024B034A08F0DBB9EF
:1006400000000020AEB40000CDB30000034B032235
:100650009A700821024B034A08F0CDB9000000202F
:10066000CCB40000CDB30000034B04229A700821E3
:10067000024B034A08F0BFB900000020EAB40000B2
:10068000CDB30000034B05229A700821024B034AA8
:1006900008F0B1B90000002008B50000CDB300009B
:1006A000034B06229A700821024B034A08F0A3B9B3
:1006B0000000002026B50000CDB30000034B072248
:1006C0009A700821024B034A08F095B900000020F7
:1006D00044B50000CDB30000034B044A08219970D3
:1006E000034B08F088B900BF00000020CDB3000024
:1006F00062B5000008B5054B02221A700821044BB0
:10070000044A08F078F9002008BD00BF000000206E
:1007100080B500009AB5000008B5054B01221A709B
:100720000821044B044A08F066F9002008BD00BF08
:1007300000000020B4B500009AB5000010B5054BCC
:10074000054A00241C700821044B08F054F9204687
:1007500010BD00BF000000209AB50000CEB500001B
:1007600030B5424D424A85B00821044608F043F9AD
:100770006B780F2B27D8DFE803F0081A261C1E2001
:10078000222626262626262626243A4B3A4A0821C1
:10079000204608F030F9AB78082B16D8082B1DD866
:1007A000DFE803F0521C504E4C4A48462400334BBD
:1007B000ECE7334BEAE7334BE8E7334BE6E7334B01
:1007C000E4E7334BE2E7334AE1E7F42B40D007D8C4
:1007D000EC2B41D0F02B3DD0D82B3FD02E4A07E058
:1007E000F82B33D0FC2BF9D12C4B00E02C4B2D4AAD
:1007F0000821204608F0FFF82B78012B30D0022B7F
:1008000030D0002B30D1284B284A2046082108F050
:10081000F2F8EB680293AB6801932B7900932046C2
:10082000EB78234A082108F0E6F8002005B030BD37
:10083000204BDCE7204BDAE7204BD8E7204BD6E70C
:10084000204BD4E7204BD2E7204BD0E7204BCEE71C
:10085000204BCCE7204BCAE7204BC8E7204BC6E72C
:10086000204BD1E7204BCFE7204ACEE70000002005
:10087000E6B5000095B3000001B300007CB30000B2
:1008800063B300004AB300002DB3000010B30000B2
:10089000DFB20000F3B500001AB6000075B4000026
:1008A00062B50000CDB30000CEB500009AB50000DF
:1008B00052B6000044B5000026B5000008B500009F
:1008C000EAB40000CCB40000AEB4000093B4000061
:1008D00057B4000038B4000019B40000FAB30000A7
:1008E000AEB30000B4B5000080B5000030B6000023
:1008F00038B50F4C054600211022204608F0D2FFE3
:10090000042323700B4B5A786270DA7822712046E8
:100910001A799B686271A36000F08AFC064B012281
:100920001A702846054A082108F065F8002038BDED
:10093000180700200000002054110020ADB6000070
:1009400038B50F4C054610220021204608F0AAFFBA
:10095000032323700B4B5A789968627020461A79EA
:100960005B88A160A380A27100F062FC064B0122AB
:100970001A702846054A082108F03DF8002038BDC5
:10098000180700200000002054110020B7B6000016
:10099000014807F0FABA00BFC1B600001FB504460F
:1009A0000C22002101A808F07DFF01A800F010FD35
:1009B0002046094A082108F01EF8DDE90112204608
:1009C00008F026F82046039B044A082108F013F893
:1009D000002004B010BD00BFE0B60000F3B6000078
:1009E000014800F03FBD00BF18070020012910B5E5
:1009F0000C4603D108F024F8204610BD022907D97F
:100A00001368064A012107F0F6FF6FF01500F4E7BE
:100A100002D15368024AF5E70020EEE70AB700006A
:100A200025B7000037B50E4B5B780F2B044614D169
:100A30000B390F2911D90B251A23CDE90053094A87
:100A4000094B082107F0D7FF084A2B46082120460A
:100A500003B0BDE8304007F0CEBF03B030BD00BFEB
:100A6000000000203AB70000DFB2000070B70000BD
:100A7000F8B5114C237805461BB100F09FFC00230C
:100A800023700E4E0E4CF1782846FFF7CBFF102254
:100A90000021204608F006FF737863707388A380F6
:100AA00000272046277000F0C3FB2846054A08218E
:100AB00007F0A1FF3846F8BD5411002000000020C7
:100AC0001807002083B700002DE9F0411F4C237860
:100AD0000546884617461BB100F070FC00232370C2
:100AE0001B4E2846F178FFF79DFFB8F1020F09D998
:100AF00028463B68174A012107F07DFF6FF015007B
:100B0000BDE8F081144C10220021204608F0CAFEF6
:100B10000123237073786370B3782371F378A37122
:100B2000B8F1020F3378637105D1786808F0FDFCE5
:100B30000A4BA060E360084800F07AFB2846084AA8
:100B4000082107F058FF0020DAE700BF5411002009
:100B5000000000200AB700001807002091090000DB
:100B600099B70000012970B506460C4603D107F07D
:100B700067FF204670BD022907D91368184A012172
:100B800007F039FF6FF01500F4E7506808F0CDFC6E
:100B9000642805D9134A0121304607F02CFFF1E7FC
:100BA000114D124CE978E8603046FFF73BFF102208
:100BB0000021204608F076FE052323706B786370D1
:100BC000AB7823712B786371EB78A3712046EB68C7
:100BD000A36000F02DFB064B01221A700020C9E72C
:100BE0000AB70000B9B70000000000201807002075
:100BF0005411002038B5104D2B7804461BB100F07D
:100C0000DDFB00232B700D4D20460D4CE978FFF7DE
:100C100009FF10220021204608F044FE0223237021
:100C20006B786370EB78637120462B78237100F04A
:100C3000FFFA002038BD00BF541100200000002042
:100C400018070020012910B50C4603D107F0F8FE63
:100C5000204610BD022907D91368064A012107F072
:100C6000CAFE6FF01500F4E702D15368024AF5E7B7
:100C70000020EEE70AB70000DFB70000012938B511
:100C800005460C4603D107F0DBFE204638BD02299D
:100C900007D913680D4A012107F0ADFE6FF015006A
:100CA000F4E7506808F041FC5028034605D9084A8B
:100CB0000121284607F09FFEF0E7064A082110713F
:100CC0002846054A07F097FE0020DFE7F5B7000049
:100CD0000FB800000000002031B80000012938B52D
:100CE00005460C4603D107F0ABFE204638BD02296D
:100CF00007D913680D4A012107F07DFE6FF015003A
:100D0000F4E7506808F011FC6328034605D9084A47
:100D10000121284607F06FFEF0E7064A082190609F
:100D20002846054A07F067FE0020DFE7F5B7000018
:100D300049B800000000002071B80000012938B552
:100D400005460C4603D107F07BFE204638BD02293C
:100D500007D91368154A012107F04DFE6FF0150001
:100D6000F4E7506808F0E1FB012805D9104A012199
:100D7000284607F040FEF1E74FF08044C0B200F093
:100D80003FFBD4F880350B4A03F0010308212846C5
:100D900007F031FED4F87835074A284603F00103FE
:100DA000082107F028FE0020D0E700BFF5B70000BB
:100DB00088B80000A5B8000007B90000012938B5BF
:100DC00005460C4603D107F03BFE204638BD0229FC
:100DD00007D913680D4A012107F00DFE6FF01500C9
:100DE000F4E7506808F0A1FB5028034605D9084AEB
:100DF0000121284607F0FFFDF0E7064A0821D070E0
:100E00002846054A07F0F7FD0020DFE7F5B70000A8
:100E10000FB800000000002031B90000012910B512
:100E20000C4603D107F00CFE204610BD022907D95D
:100E30001368064A012107F0DEFD6FF01500F4E7A4
:100E400002D15368024AF5E70020EEE7F5B700004B
:100E500025B700000B4B00224FF0FF31C3F80022F2
:100E6000C3F80813C3F81021D3F81021064A012152
:100E700003F5887311601A68002AFCD000221A60FA
:100E80001B687047001000401010004073B5194BEC
:100E9000194E187030460C4605F0E6FA174B002143
:100EA000D3F80022C3F800124FF0FF32C3F8082332
:100EB000D3F810254FF47A53D2B2A4FB0345C2F104
:100EC000200305FA03F3A2F1200024FA02F225FA26
:100ED00000F01A43012302430093304609F028F83A
:100EE000304609F00BF8304602B0BDE8704005F01E
:100EF000ADBA00BF5511002020AC000000800040BA
:100F00000F4B1A6810B532B100221A600D4A1B68E7
:100F10001368013313600C4B1A687AB100221A600F
:100F20000A4A1B681368013313608268934205D133
:100F3000FFF790FFBDE81040C368184710BD00BF21
:100F400030110040280700200C1100402C07002021
:100F50001FB5544B4FF40072C3F850260022C3F85B
:100F60003425C3F83825C3F82C25012291420446C4
:100F7000C3F8302524D002291CD0002977D1AB2218
:100F8000C3F824254FF0AB32C3F81C2500210D22F5
:100F9000684608F087FC444B0293062C4FF001038F
:100FA0008DF80C3011D8042C63D800D000238DF8B4
:100FB00005301CE0CC22C3F824254FF0CC32E3E707
:100FC0006A22C3F82425394ADEE70F2CEED102232A
:100FD0008DF805307F238DF808300023ADF80A30F6
:100FE0008DF80C302F4B40F20122C3F850269DF8AB
:100FF00002309DF801209DF806409DF804009DF800
:1010000005101B0443EA02239DF80320002A14BFA5
:101010004FF480120022002C14BF4FF08064002493
:10102000234343EA805343EA01639DF8071043EAF0
:10103000417313431B4A43F00803C2F814359DF86B
:101040000A109DF8083043EA01439DF80B1000296F
:1010500014BF4FF0807100210B439DF80C10002944
:1010600014BF4FF0007100210B43C2F8183504B0D3
:1010700010BD7F238DF8083040F20233ADF8043004
:1010800003238DF80730ADF80A30064B40F20122F9
:10109000C3F8502640F20312C3F834250022C3F8E7
:1010A0003825A4E700100040FF0004011B81FE5812
:1010B000F8B505460C46FFF74BFF0F2D14491548B0
:1010C000154F0CBF7E23FF230B700A46FF23F0252C
:1010D000CC26ACB90460D0F800C0D0F800C0BCF198
:1010E000000FFAD0D7F808C582F801C0013B13F011
:1010F000FF0302F10102ECD1084BC3F80415F8BD5F
:10110000022C01D15670F1E7012C08BF5570EDE7B4
:101110005612002000D1004000D0004000100040D6
:101120000F28084B06D1A1F10B020F2A05D801EBBD
:1011300081013239C3F8081570470522C3F8082524
:10114000704700BF0010004070B5134C05460E46B6
:101150001046FFF77FFEC4F81055D4F8003243F074
:101160002103C4F800320D4BC4F80435014628466B
:10117000FFF7EEFE31462846FFF7D2FF084B00226C
:101180001A604FF48053C4F8043303F180430433EE
:1011900001221A6070BD00BF0010004056110020EF
:1011A00028070020B0F5A07FF8B50C4633D10978A8
:1011B000032920D11B4B607827791E781A4DFFF741
:1011C00049FEC5F81005D5F8003243F00103C5F813
:1011D00000323146C5F80C75FFF7A2FF01232B60E2
:1011E0006079A4790F490A780132D3B2A34288BF4B
:1011F00003460B70F8BD042908D10A4B60782279A8
:101200001978FFF7A1FF20796479EBE7BDE8F84092
:10121000064806F0BABEB0F5A27F02BF024B01221B
:101220001A60E7E7551100200010004088C0000058
:10123000F7B502780346052A19D8DFE802F0031A49
:101240004F575E6140781E795D79564CFFF702FE7C
:10125000C4F81005D4F8003243F00103C4F800329A
:101260002946C4F80C65FFF75BFF0123236003B038
:10127000F0BD45780779867940794A4CFFF7EAFD59
:1012800001462846FFF714FF062D20D8042D20D94B
:10129000D4F8003243F4001343F00103C4F80032E1
:1012A0003146C4F810552846C4F80C75FFF738FFCE
:1012B0003D4B00221A603D4B1A601A680822C4F8A0
:1012C0000423012222601A68002AFCD0CFE70F2DE8
:1012D000DED0D4F8003243F02103DFE70279417910
:1012E000407803B0BDE8F040FFF72EBF8168407939
:1012F00003B0BDE8F040FFF7C9BD81680079F7E7AA
:1013000045782B4A9B68545D0779867940794FF47C
:1013100083726243C3F164045443B4FBF3F4144492
:10132000FFF798FD01462846FFF7C2FE1D4BC3F8A4
:101330001055D3F8002242F00302C3F800223146D0
:10134000C3F80C752846FFF7EBFE1A4805F08CF839
:10135000194BD3F800220022C3F800224FF0FF32CD
:10136000C3F80823D3F81025D2B2210FC2F120030D
:10137000240101FA03F3A2F1200024FA02F221FA77
:1013800000F01A430121024300910223094808F0AA
:10139000CFFD084808F0B2FD064803B0BDE8F040B4
:1013A00005F054B8001000402C0700200C1100403C
:1013B000C9C0000020AC00000080004008B5034810
:1013C00005F052F8BDE80840FFF744BD20AC00002E
:1013D000084B094AD3F8103503F00F030F2B0CBF4D
:1013E0007F234FF48073C0E90023044B1B688360A4
:1013F000704700BF00100040561100202807002051
:10140000D0B94FF08043D3F88035DB070DD4114BB2
:101410001B68082B0ED1104B1B68052B0AD80F4AEE
:10142000D35C01200BB10E4B18604FF08043C3F822
:10143000800570470120F8E7012809D84FF0804265
:10144000D2F8783503F0010383F00103C2F8783550
:10145000704700BF3001001034010010C3C000000D
:101460003806004030B5184B85B001221A600023C1
:10147000ADF809308DF80B3004238DF80830039057
:10148000022302A9114A8DF80A300446104804F0DC
:101490008FFF104B9842014602D00F4806F075FDB1
:1014A000002500220621082002F05EFE0B4A00956E
:1014B00023460621012002F06FFE012002F036FED5
:1014C000284605B030BD00BF00D00040A511000087
:1014D00020AC00000000AD0BA2C00000010F000016
:1014E0000B6801330B60014B1B681847100000208C
:1014F000014B1860704700BF1000002007B50B4675
:10150000002102460191034801A900F0FFF803B051
:101510005DF804FBE114000030B585B0CDE90101B0
:101520000446002501A90548039500F0EFF8DDE920
:1015300002309842B8BF255405B030BD657F000029
:101540002DE9F84FB0F8189019F0080804469346B2
:101550000DD001290CBF49F0100949F02009A0F86D
:1015600018908BF31188BFF36F8FBDE8F88F09F0E7
:101570000709022907D1204606F021FD0028F0D0F6
:101580000128238B50D16769218B002F15DA25683C
:1015900021F00701C4E9008841F001012183002600
:1015A000218B01F0070ACA4502D0A368002B5CD149
:1015B0000DB9002E74D0002358E001F007035A1F24
:1015C000012A20D821F00701062B256889B2C4E939
:1015D00000880CD1002D2B4638BF00232BB1628B25
:1015E0001B6801326283002BF8D141F00201218394
:1015F000204606F0E4FC06460028D1D0238B43F0B9
:1016000020032383CBE7042B0CD121F0070189B2FF
:101610002183204606F0D3FC05460028BFD041F0C8
:10162000200121830025BAE7032809D1226923F08C
:101630000703166843F00603238300252F46AFE710
:10164000042806D1226923F00703566843F00403F7
:10165000F2E7052806D1226923F00703966843F0D4
:101660000503E9E700252E46E8E7012341F00801DC
:1016700021838BF31188BFF36F8F03BB002D33D110
:1016800016B121492046B0474FF02003EFF3118BEC
:1016900083F31288BFF36F8F238B23F00803238318
:1016A000238BDA0628D523F0100323830121B4F815
:1016B000189009F0070900297FF45BAF51E7A16892
:1016C0000029DBD00B68D1F804B0002B38BF002311
:1016D000994652463B462046D847B9F1000FCDD037
:1016E000D9F800304946EEE729463B4652462046A7
:1016F0002D6806F080FCC1E713F020011EBF23F027
:10170000200323830221D2E7238000002DE9F04F3C
:1017100091B08B46029092461C4600259AF8000034
:1017200008B928465EE325280AF1010707D0029B85
:10173000594698470028C0F25583013510E2182217
:1017400000210AA808F0AEF89AF80130252B78D0CD
:1017500000229446164696461046394617F8013B35
:101760002B2B00F09D8000F29480202B00F09B80BA
:10177000232B00F09A8028B19DF8300040F004003F
:101780008DF83000BEF1000F05D09DF8300040F01C
:1017900008008DF830002EB19DF8300040F01000A8
:1017A0008DF83000BCF1000F05D09DF8300040F0FE
:1017B00020008DF830002AB19DF8302042F0400220
:1017C0008DF830209DF8302002F04400442803D1E9
:1017D0006FF386128DF830209DF830202A2B42F0CE
:1017E00080028DF830207BD19DF8312042F001023B
:1017F0004B1C8DF831201A782E2A9DF831200CBF11
:101800000121002161F341028DF8312074D15A7811
:101810002A2A6AD0013300210A26184610F8012B23
:10182000A2F13007092F40F28E809DF830200E91F2
:10183000C2F3400040EAD17161F341028DF83020DB
:101840005AE00AF102078DF833309DF83130D9079C
:1018500040F1498154F8049BB9F1000F07DA9DF873
:10186000302042F004028DF83020C9F100095A07F7
:1018700040F1428154F8048BB8F1000F80F24181AD
:101880009DF831306FF341038DF831304FF0FF3860
:1018900037E12D2B0CD0302B7FF46DAF01225CE7AC
:1018A0004FF0010E59E7012657E74FF0010C54E7BE
:1018B000012052E70CFB0202303A33461E4616F86E
:1018C000010BA0F13007092FF4D9994293D09DF86C
:1018D00030100D92D20F62F341018DF830108AE77B
:1018E0000B4600224FF00A0CE8E79DF8312042F049
:1018F00004028DF8312002331F4617F8012B6C2AA1
:1019000041D025D8682A2BD06A2A46D04C2A4CD000
:101910001F4617F8012B9DF831308DF83320782AB7
:1019200000F2D980572A4DD8412A03D0453A022ADD
:1019300000F2D1809DF83230042262F302038DF868
:10194000323001239EE006FB01213039034664E773
:10195000742A26D07A2ADBD19DF8313006220DE098
:101960005A78682A9DF8312006D1012161F3C60218
:101970008DF831209F1CCCE71346022262F3C60388
:101980008DF83130C5E75A786C2A9DF8312001D1A5
:101990000421EBE713460322F0E79DF831300522DE
:1019A000ECE79DF831300722E8E7BDF8303023F44A
:1019B000F04323F0020343F4804343F00203ADF805
:1019C0003030A6E7A2F15801202900F2848001A05E
:1019D00050F821F0991A0000D71A0000D71A000019
:1019E000D71A0000D71A0000D71A0000D71A000033
:1019F000D71A0000D71A000035190000D71A0000C6
:101A0000991A0000591A0000351900003519000014
:101A100035190000D71A0000591A0000D71A000023
:101A2000D71A0000D71A0000D71A0000A11A000028
:101A3000991A0000BD1A0000D71A0000D71A00003A
:101A4000BD1A0000D71A0000991A0000D71A00002A
:101A5000D71A0000991A00009DF83210012003F0F7
:101A6000780360F30201402B8DF8321002BF9DF81D
:101A7000301041F001018DF83010632A31D1003B64
:101A800018BF01239DF83020C2F340010B4363F3DC
:101A900041028DF83020D8E69DF832100220DEE7B2
:101AA0009DF8322003F07803A3F14000032161F395
:101AB000020243428DF832204341E3E79DF8322091
:101AC000032113F0780F61F302028DF8322014BF66
:101AD00001230023D6E79DF8303043F001038DF851
:101AE00030300023CEE79DF93020002AB4BFDDF866
:101AF00034904FF0FF39BAE69B077FF5C7AEDDF8AB
:101B000038809DF831200023CDE90D339DF8323027
:101B100003F00703012BC2F3C30236D1D31E042BFB
:101B200020D8DFE803F00307071F1F0054F8040B59
:101B3000C11704E0073424F00704F4E80201CDE9FA
:101B40000A019DF8303013F0030654D002983B464A
:101B50005246594606F095FB0028C0F243810544E1
:101B6000BA46DBE554F8040B012A4FEAE071CDE9EF
:101B70000A0105D19DF828300A9300230B93E0E772
:101B8000022ADED1BDF92800D2E7022B23D1D31ED1
:101B9000042B13D8DFE803F0030A0A1212002068AE
:101BA0000A900021231D0B911C46CAE7073424F03C
:101BB0000703F3E80201CDE90A01F5E754F8043B15
:101BC0000A93012A4FF000030B93D3D0022AB8D115
:101BD000BDF82830D0E7042B07D1073424F00704E0
:101BE000F4E80201CDE90A01ABE7032B04BF54F886
:101BF000043B0A93A5E79DF833007828B0D8622803
:101C000022D825283FF493AD5828A9D10DF12603F9
:101C10000093DDE90A0104AB0CAA06F0E7FA82465C
:101C2000B8F1000F0DF126000CDB9DF83020A0EB81
:101C30000A036FF3861298458DF8302002D9A8EB7D
:101C400003030D9380463DE06338152888D801A131
:101C500051F820F0D51C0000391D0000611B000068
:101C6000611B0000611B0000611B0000391D0000AA
:101C7000611B0000611B0000611B0000611B000074
:101C8000971D0000651D0000691D0000611B00001C
:101C9000611B0000AD1C0000611B0000651D000001
:101CA000611B0000611B0000651D0000B8F1000F02
:101CB000DDF828A00ADB4146504607F09DFD0AEBFF
:101CC00000080026BAF1000F0CD149E7504607F092
:101CD0008CFDF4E70A9B8DF8103000260DF11108F9
:101CE0000DF1100AA8EB0A0306B101339DF832206A
:101CF000D0066BD5023352060D9948BF0E9A0B449D
:101D000048BF9B18B9F1000F79DD9DF83020A9EB91
:101D10000309C2F380030393530770D4500664D5BC
:101D200046B1029B59463046984700285ADB039B30
:101D300001351E46302359E01E0711D413F010065A
:101D400018BF2026DDE90A23002A73F10001BFF63F
:101D50005DAF524263EB4303CDE90A232D2655E7DD
:101D60002B26EFE7002651E70A9848B30DF126032A
:101D700000930CAA04AB002106F038FABDF832300B
:101D800003F0EF0343F4F04343F010038246ADF851
:101D90003230002644E70A9B072A3FF6E1AEDFE82F
:101DA00002F00D04060D08080D0D1D70D8E61D800B
:101DB000D6E62846E917C3E90001D1E61D60CFE663
:101DC000DFF8C4800646A8F1050A8BE7110748BF73
:101DD000013390E7184603935946029B9847002821
:101DE000039B04DA11B0BDE8F08F20234D444A462E
:101DF000002AA5EB090109F1FF39EBDC0D4636B1EC
:101E0000029B5946304698470028EBDB01359DF888
:101E10003230D90601D41A0706D5029B5946302024
:101E200098470028DEDB01359DF83230DB0607D508
:101E30009DF83300029B594698470028D2DB0135B4
:101E40000D9E2E44731B002B16DC0298434652460F
:101E5000594606F016FA0028C4DB0544A944A9EB4C
:101E60000503002B7FF77CAE029B59462020984744
:101E70000028B7DB0135F2E7029B5946302098472E
:101E80000028AFDB0135DDE7DEC0000008B54FF00C
:101E90002002EFF3118382F31288BFF36F8F02F0F9
:101EA00029FD034806F071F802F028F9FCE700BFAD
:101EB000DFC0000013B5044604F034FEC0F307236E
:101EC0000193C0F307430093044A030E0821204600
:101ED00006F091FD002002B010BD00BF08C1000057
:101EE0002DE93048044608F010FA4FF47A75A0FB4B
:101EF00005BC05FB01CC4FEADB3242EA4C432046ED
:101F0000034A082106F077FD0020BDE8308800BFB5
:101F100021C1000010B5044603F0E6FC084A034660
:101F20000821204606F067FD064A2046082106F0F3
:101F300062FD0548214604F081FC002010BD00BF71
:101F400030C100004FC10000AD1F000030B5014698
:101F500087B00446114804F071FC114A002312F8BE
:101F6000011BAA2903D10133B3F5006FF7D1C3F5E3
:101F7000006164224A43D20A059200254FF40062B0
:101F8000CDE90312CDE901232046064B064A009510
:101F9000082106F030FD284607B030BD8D20000036
:101FA000602700204027002059C10000F0B587B00D
:101FB000D0F8A07004460D4608F05FF8064605F01C
:101FC000E5F9234B234A002E08BF1E46224BCDE9DC
:101FD0000046844218BF1346082128461F4A06F0CF
:101FE0000AFDD4E90A23CDE9022394F90E301C4AF4
:101FF00000930821237B284606F0FDFC204604F0D0
:1020000065FC626E00920346164A0821284606F0D7
:10201000F2FC05A9204608F034F8034630B1124A14
:102020000821284606F0E7FC07B0F0BD059A6423B6
:10203000B91ACDE900214B430C4AB3FBF7F3082151
:10204000CDE9027328463B4606F0D5FCECE700BF1D
:10205000A1C10000A8C800009FC10000A4C10000E9
:10206000B0C10000DCC10000F3C1000020C20000CC
:1020700010B5044607F0CCFE034A0346082120466B
:1020800006F0B9FC002010BD57C20000F0B5D0F832
:10209000A06089B004460D4607A907F0F2FF034689
:1020A00030B1104A0821284606F0A5FC09B0F0BD61
:1020B000204607F0E2FF0C4F079A002808BF384679
:1020C000B11A6423CDE90221CDE900064B43074A4A
:1020D000B3FBF6F30821CDE904632846234606F056
:1020E0008AFCE3E7F3C10000A1C100006DC200005B
:1020F0000346006810B50C46114608B1027822B9B3
:10210000024A204602F0ACFB204610BD77C3000017
:1021100010B50C68D1E90112FFF7EAFF034A034644
:102120000821204606F067FC002010BD7CC300009B
:102130002DE9F0478AB0054601A804F04DFA019B4D
:102140001B4ADFF87880DFF87890DFF878A018264F
:1021500006FB00360821284606F04DFC019CB442DF
:1021600003D300200AB0BDE8F08705AF394614223A
:102170002046FFF7BDFF424603460821284606F0E9
:102180003AFC204607F0F1FE0A4A002814BF4B46ED
:1021900053460821284606F02EFC14232046064903
:1021A000049302AACDE90257183407F0E8FED6E7F7
:1021B0009BC30000AAC3000011210000A5C30000BA
:1021C0008CC3000092C300002DE9F043114BDFF8EF
:1021D000489053F82140013187B053F821800646DA
:1021E0000027A04503D8384607B0BDE8F083204655
:1021F00007F0BBFE054658B1142201A92046FFF79F
:1022000077FF4A4603460821304606F0F4FB2F4686
:102210001834E6E728AD0000B1C3000010B508216E
:1022200004461E4A06F0E7FB00212046FFF7CCFFDC
:1022300020B91B4A0821204606F0DDFB0821204674
:10224000184A06F0D8FB01212046FFF7BDFF20B950
:10225000134A0821204606F0CEFB08212046124AE8
:1022600006F0C9FB02212046FFF7AEFF20B90C4A59
:102270000821204606F0BFFB082120460B4A06F045
:10228000BAFB03212046FFF79FFF20B9044A08212B
:10229000204606F0B0FB002010BD00BFB7C3000011
:1022A000C6C30000CEC30000DDC30000EBC30000C6
:1022B0008B1E022B2DE9F04107468846144633D881
:1022C00060681022002107F0CCF9B8F1020F064631
:1022D0001ED0A0680A22002107F0C3F9C5B2214A26
:1022E0002B460821384606F086FBB8F1040F1ED0B5
:1022F000102D0FD0202D10D0082D10D13378DBB247
:10230000194A0821384606F076FB0020BDE8F08126
:102310002025E4E733889BB2F2E73368F0E7134AFD
:102320000821384606F067FB6FF01500EEE7E0681D
:102330001022002107F095F90D4A034604460821B2
:10234000384606F058FB102D06D0202D07D0082D5A
:10235000E5D1E4B23470D8E7A4B23480D5E7346074
:10236000D3E700BF4FC400007AC4000064C400007B
:102370008BC4000070B50F4C054623780E4639B16A
:1023800033B10D4A012106F036FB6FF00F0070BD2E
:1023900083F00103237033B1084A0821284606F070
:1023A0002AFB012323702846314606F05EFB0020FD
:1023B000EDE700BF581300209FC40000DAC40000FE
:1023C0002DE9F74F06462E48DFF8CC90DFF8CCA079
:1023D000DFF8CCB0002303600D462A482A49036089
:1023E0000B7014460091012D274654F8043F21D963
:1023F000184602224946019307F013FA019B88B957
:1024000022689278003A18BF012203EB0208514675
:102410000222404607F005FA30B9009A01231370F2
:10242000013DE0E70022F0E74946404607F0EDF9BC
:10243000B0B9043700221146786807F09CF8134BB6
:10244000002211461860786807F095F8104B114982
:1024500018603046FFF78EFF002003B0BDE8F08F14
:1024600098F800202D2AE5D198F80120002AE1D023
:1024700043465A460821304606F0BDFAD0E700BF71
:10248000340700203C0700205913002030070020AB
:1024900038070020A524000004C5000007C500007F
:1024A0000AC5000070B53E4B05461878182802D1C1
:1024B0000878112831D0013A08465418844225D1B1
:1024C0008A5C1A700A78374CA2F13003092B04D9C0
:1024D00022F02003413B052B04D823683249CA541B
:1024E000013323602368022B34D110222E480021AF
:1024F00007F0B7F82D4A136803F8010B13602C4A54
:102500001368013313600023236023E010F8016B8C
:10251000182ED3D10678112ED0D1254C254A236808
:102520000821284606F067FA00212846FFF722FF17
:10253000214B187870B9214A23681168042B0ADCF2
:1025400008B11160236013F003010BD11268136806
:102550001BBA136070BD086800BA41F8040B043B55
:102560000120EBE75B4203F0030358BF5942022905
:1025700007D112681168C1F3072343EA01239BB214
:10258000E7E70329E6D1106802681104C2F30743A4
:1025900001F47F010B4302F47F4213430360D9E748
:1025A0005A13002034070020561300203007002063
:1025B0003C0700201FC500005913002038070020E9
:1025C00013B5094807F0D1FC58B1084A064912680A
:1025D000074800240094012300F076FD204602B055
:1025E00010BD6FF01200FAE71CA70000C4AD000098
:1025F00034A7000070B546680C463168B0688B603F
:102600000025C1E900420822C0E9005529461044CE
:1026100007F048F9F0680822C0E90055294610443F
:1026200007F040F93368DD60A3682BB19B6C1BB1E8
:102630000549324620469847A3689B6A0BB120465D
:102640009847002070BD00BF6B87000010B58168FF
:102650000446083101F06EF9A168034A20460831AA
:10266000BDE8104001F008B9D5C5000037B50446F3
:102670008068D0F864325A070D4605D5002106F06F
:1026800051F9E06806F043FEE368DB686BB9002DA2
:1026900037D0A068423006F032F9A36898B303F14E
:1026A000420103F5A17007F075F8A268E0680DF12A
:1026B00006034232294606F02DFE58B9A06800F5FF
:1026C000A171423007F066F8A068423006F017F9B1
:1026D000ADF80600204606F067FCA368D3F8603228
:1026E0009B0603D50949606906F00FF9204600F002
:1026F00017FFA368BDF80620DA879A87204600F006
:10270000D1FE03B030BD83F84201CEE750A80000EF
:102710008368022210B51A719B6B0446CBB982689C
:1027200082F84230D3638368D3F86432DB040BD57C
:102730000321084B084A06F0E7FCA0686FF48051BB
:1027400000F5197006F08FF82046BDE8104001F042
:1027500001B810BDE3C50000A7C300002DE9F04F8C
:1027600000239FB0CDE905338368044642330393C9
:1027700006F020FC204606F0A5FB18B99F496069C9
:1027800006F0C3F8A06814220021083007F08AF888
:10279000204606F044FBA168E0688A8F423100269B
:1027A00006F0EFFD204606F072FE4FF0FF38B1460E
:1027B000B24611AF02963546B346DDE90532012A2D
:1027C00000F0D7800B2B40F2AF80069B022B40F02D
:1027D000AF808B4B8B4A012114E0039A02233946C8
:1027E00006A806F0ADF906997A680392034629B95E
:1027F0006FF0070528461FB0BDE8F08F012905D10D
:1028000020B1814A204606F07FFCF1E7059B4BB3DF
:10281000386801F0B3F898B166B1A5680D9608352F
:102820000CAE0FCE0FC533682B602046FFF70EFFAE
:102830000125DFE7754A0121204606F065FCD7E750
:10284000059B7BB13A682946204601F0F7F902283A
:1028500000F08F80032805D0059B013305930123E9
:102860000293AAE7BAF1000F05D1396807AA5846C2
:1028700006F051FA0546043708F1FF38002D41D023
:10288000029B4BB1EB683BB1204606F093FB204620
:1028900000F008FE5E4ACEE7EB68CBB1A368DDF836
:1028A0001490AE4603F1080CBEE80F00ACE80F0030
:1028B000DEF80030CCF80030AB684BB96B7CFE2BF7
:1028C00001BF95F8108009F1010308F1FF38059365
:1028D000D5F804C0BCF1000F08D0AE46BEE80F002A
:1028E0000CAE0FC6DEF8003033606646AB46B8F17A
:1028F000000F03D1069B022B7FF45FAF059B0133D2
:1029000005935AE7059B63B9A368DB690BB1DB68E4
:102910003BB9404B0093404A119B0121204606F0F1
:10292000F3FB4FF0010AE2E7B8F1000F7FF455AF77
:10293000029B4BB1204606F0CFFDA2680C23423229
:1029400011A905A806F0FCF8059DA0681EAB03EBD5
:102950008503002243F8342C436973B9002E3FF4F9
:1029600047AFC368B3423FF460AF0D9600F108056E
:1029700056E7059B0B2BDBD927E7037EA5EB090563
:10298000B3B1427E4FF6FF71FF2A08BF0A469D424F
:1029900002D313449D420BD98368204A012120466B
:1029A00006F0B2FB2046FFF751FE6FF0150521E758
:1029B0004FF4006100F5197005F046FFA06800F5BE
:1029C0003E7005F09AFFA36811AA294602EB89021E
:1029D0005B69204698470546A0684FF0FF324FF0EC
:1029E000FF3300F53E7005F0C7FFA0686FF400618B
:1029F00000F5197005F037FFFCE600BF55C2000076
:102A00009CC60000B3C3000027C600003BC6000000
:102A100059C6000088C600001DC90000C0C60000DD
:102A20002DE9F04F04468068ABB0012100F5197024
:102A300005F00AFFA3681B79022B17D100230B9323
:102A4000A36860689E6B03681D690BABC6B110225A
:102A50001DA9A8470B9A4AB11DA92046B047A368F3
:102A60009B6B002BECD12046FFF752FEA0686FF065
:102A7000010100F5197005F0F6FE2BB0BDE8F08FEE
:102A800001220DF12B01A8470B9B002BEED09DF9E5
:102A90002B209DF82B30A068002AD1DB4279032A35
:102AA00000F2FF82DFE812F004007F029602FD02CE
:102AB0000D2B1AD00A2B18D0B0F864226FF3CA027B
:102AC000A0F86422092B4DD033D8002BB8D0082BA6
:102AD00000F0CB81A3F120025E2A00F2D281012115
:102AE00005F020FF9DF82B10E9E0D0F86422C2F336
:102AF000C7022AB1D0F86422C2F3C7029342E1D1DF
:102B0000B0F86422818F63F3CA02A0F8642261B92D
:102B100005F008FFE06806F0FAFBAD49606905F0D2
:102B2000F4FE2046FFF7F4FD8AE72046FFF716FE85
:102B3000F7E71B2B13D07F2BCCD1D0F860329D0749
:102B40007FF57EAF012105F0EDFEA368D3F860327A
:102B5000190700F19281204606F017FB70E7012368
:102B600043716DE7D0F860329B077FF569AF0121B3
:102B700005F0D8FEA068838FFF2B3FF461AFC28FB2
:102B800000F1420100F5A17006F081FEA268D38F2A
:102B90001344002583F842511DA90C2302F5A172AC
:102BA0000DA805F0CDFF0D990C293FF649AF2AABD2
:102BB00003EB810343F8345CA368DA8F134493F882
:102BC0004130202B00F06F82093B042B40F26B82D6
:102BD00001294FD800250C950C9B2AAA02EB8303F0
:102BE000002653F834AC504605F089FEB0468146C5
:102BF0000496374618AA3946284600F0F5FB834666
:102C0000002844D1012E63D10C9B2AAA02EB830336
:102C100053F8340C05F073FEA268064608324146AC
:102C2000284600F0E1FB0546006805F068FE864294
:102C300006D02968821B92B23144204606F0A3FADE
:102C4000A068C38F034493F84230202B3BD0093B4C
:102C5000042B38D9D0F86032DF072FD5002105F0DA
:102C600071FE2021204600F03DFDA068012105F005
:102C700069FEE5E6013900200EAB009301900CAB34
:102C80001DAA06F068F805460028A5D1D8E6DBF8AD
:102C900000004A46514606F0C4FD68B9DBF8000062
:102CA00006F0A3FD049B834238BF03469BB2002E6F
:102CB00008BFB8460493013601379BE72021204620
:102CC00000F010FDBCE60121204606F00FF9B7E642
:102CD0007FF6B6AE0C9B2AAA02EB830353F834AC02
:102CE000504605F00CFEA3680690A3F830B0DFF85C
:102CF000E4B00596CDF80C80A26803990832284606
:102D000000F072FB039B013307460393BAF1000FF7
:102D100053D13B68002B5FD1A2681386059B013B12
:102D20000593E9D12A49606905F0EFFD204600F0DE
:102D300011FD0C9B2AAA02EB830308F1010953F849
:102D4000340C05F0DCFD414613AA0746284600F086
:102D50004BFB8046A068D8F80010FF2200F5A17058
:102D600006F022FDD8F800A04FF6FF7818AA4946D1
:102D7000284609F1010B00F037FB002868D0A36852
:102D8000006803F5A173002213F801CB815C614553
:102D900005D121B101324FF6FF718A42F4D10FB152
:102DA000BA4208DB904506F1FF36A8BF9046012ED7
:102DB0001FFA88F84CD0D946D8E700680028A8D078
:102DC000069A514606F02DFD0028A2D094E700BFD8
:102DD00055C20000A7C800005846079305F08FFDB4
:102DE000049BA168C21892B258464F8D099205F013
:102DF00086FD079B0890184605F081FD099A089901
:102E0000079BA2EB0009A068B0F830C07F1A97FBBF
:102E1000F2F292B2BCFBF2F102FB11C20CF1010E14
:102E200092B21FFA89F9A0F830E05AB90093A04A8B
:102E30005B460621204606F067F94946204600F029
:102E40001BFB6BE79B4A0621204606F05DF9F4E781
:102E5000B8F1000F3FF4F4ADA8EB070292B20AEB11
:102E60000701204606F08FF9EAE5D0F860329E07A8
:102E70007FF5E6AD012105F055FD204606F0A0F9ED
:102E8000DEE5D0F8602292077FF5DAAD013B162B24
:102E90003FF6D6AD01A252F823F000BF7530000016
:102EA000F92E0000012F0000572B000069300000B0
:102EB000212F0000412A0000412A0000412A000081
:102EC000412A0000292F0000312F0000412A000074
:102ED0005B2F0000412A0000652F0000412A0000FE
:102EE000412A0000412A0000412A0000692F000009
:102EF000412A0000972F0000204606F062F89FE567
:102F0000204606F057F8204605F0DCFF18B96A495C
:102F1000606905F0FAFCA068012105F003FD00E6F8
:102F2000204606F056F88BE5204606F05BF887E56C
:102F3000D0F860329F0603D56049606905F0E5FC72
:102F4000A368D3F860329E0603D55D49606905F039
:102F5000DCFC204600F0FEFB72E500212046FFF776
:102F600085FB6DE50121F9E7204606F01DF8A36811
:102F7000002283F84220DA63A068012105F0D2FC28
:102F8000A368D3F860329D067FF55AAD4D4960695C
:102F900005F0BBFC54E5204600F008FBA0680121C9
:102FA00005F0C0FC4CE55B2B01D10223D8E5D0F83D
:102FB0006022900706D5622B08D14FF0FF312046E2
:102FC00005F0B8FFA36800225A7139E5662BF9D1E4
:102FD0000121F4E700224271A268D2F86012890749
:102FE0007FF52EAD313B1B2B3FF62AAD01A151F8E9
:102FF00023F000BF713000007D30000091300000F0
:1030000065300000412A0000412A0000412A0000EA
:10301000412A0000412A0000412A0000412A000004
:10302000412A0000412A0000412A0000412A0000F4
:10303000412A0000652F00005B2F0000212F0000B7
:10304000F92E0000412A000069300000412A0000EA
:1030500075300000412A0000412A0000412A00008A
:103060008130000003235371204605F0A3FFE7E4FD
:1030700003235371204605F097FFE1E403235371C6
:10308000A068D0F8601201F0010181F00101EEE5C5
:1030900003235371A368D3F860329B077FF5D0AC4C
:1030A00059E500235CE500293FF494ADE3E500BF5A
:1030B000DBC60000A7C3000055C2000055A80000F1
:1030C0005AA8000050A800002DE9F043044680688B
:1030D0008846D0F80C1389B015461F46002961D1E7
:1030E0004FF4447206F0DEFBA3682268E0681A60C1
:1030F00006F0B3F9A06800F53E7006F0D7FF4FF474
:103100002A794FF41A76A068304407F056FAA0687E
:103110000022831901214844103607F031FAB6F530
:103120002A7F09F11409EED1A369A06800260221C3
:103130001E6000F5197005F087FBA3681B4A9A62B0
:10314000186805F0DCFBA368194A83F82C00606856
:1031500066F38205C3F86052036841461D68234642
:10316000A8470546D0B9A36801221A71D4E909011C
:1031700000220023CDE906230E230393109B049520
:10318000CDE9017300940B4B4FF4006203F040FC57
:10319000A368216AC3F80C0303F088FB284609B032
:1031A000BDE8F0836FF07705F8E700BF1800500026
:1031B000658900000532000010B504468068037977
:1031C000012B19D14FF0FF324FF0FF3300F53E7065
:1031D00005F0D2FB0821204600F0AAF908496069F1
:1031E00005F093FB2046FFF793FAA06800F53E70C8
:1031F00005F083FB002010BD6FF08500FBE700BFEA
:1032000054C20000F8B504464068036800219B687A
:10321000984700283FD12046FFF7CEFF00283AD13B
:103220001D4F1E4EA06800F52A704FF0FF324FF080
:10323000FF33032104F0A0FA0546A0684FF0FF32E7
:103240004FF0FF3300F53E7075B105F095FB204659
:103250002B46134A012105F057FFA068BDE8F8404E
:1032600000F53E7005F049BB05F086FB6068036819
:103270005B6903B198473A462046022105F027FBD7
:1032800020463246002105F022FBA06800F53E7082
:1032900005F033FBC6E7F8BD85880000212A000051
:1032A000E1C6000010B50D4A0446082105F0A3FB55
:1032B00020460B4A082105F09EFB2046094A0821BA
:1032C00005F099FB2046084A082105F094FB2046AA
:1032D000064A002100F0D0FA002010BDF8C6000018
:1032E00036C7000095C70000E9C7000083C800008A
:1032F0002DE9F04716461F462A4ADFF8B480DFF86A
:10330000B490DFF8B4A00B460821044605F073FB27
:103310000025AF4231D9735D4A460821204605F0A9
:103320006AFB0135102D20D11F4ADFF88C80DFF8B1
:103330008C900821204605F05EFB0025AF422AD97B
:10334000735DA3F120025F2A28BF2E234A4608217D
:10335000204605F050FB0135102D14D12046134AAC
:10336000BDE8F047082105F046BB6A07D1D15246B7
:103370000821204605F03FFBCBE7424608212046C6
:1033800005F039FBCDE76B07D8D14246082120462E
:1033900005F031FBD2E742460821204605F02BFB21
:1033A000D9E700BF99C80000AAC80000ACC8000057
:1033B000A6C80000A0C80000A8C80000CCC8000033
:1033C00010B5044613460A4601460648FEF79EF924
:1033D00023691B7923B12046BDE8104005F048BBA6
:1033E00010BD00BF898A000010B50B46144650B9C5
:1033F0000E490F4A521AB3EBD20F0FD201EBC301A1
:103400004C68204610BD816841B14A68097839B1DD
:103410001846214690472368002BF2D10024F0E79C
:1034200014204343D418D358F6E700BF60A7000028
:1034300028A800008368D3F860329B0603D50249B0
:10344000406905F01EBD704760A800000A1E0DDC33
:103450000ED042238168D1F86012890608D5002A6F
:1034600004494069B8BF524205F00BBD4123F1E762
:10347000704700BFC8C800000A1E0DDC0ED04423F0
:103480008168D1F86012890608D5002A044940698C
:10349000B8BF524205F0F5BC4323F1E7704700BFC7
:1034A000C8C8000010B5044605F00CFD28B16069DD
:1034B0000549BDE8104005F0E4BC04F1080005F042
:1034C000EDFC0028F3D110BD55C200002DE9F041FC
:1034D0000646054656F8084F04F12000A28FE18FFA
:1034E00005F018FB3046B4F82480E78C05F0D6FCD4
:1034F00018B10A49686905F0C4FCB84507D1218CA8
:10350000638C2846C91ABDE8F041FFF7B5BFE18CCE
:10351000A38C2846C91AFFF799FFF0E755C20000AF
:10352000826802494069423205F0ABBCA7C3000083
:1035300008290A4617D8836893F82E10914212D0B2
:1035400083F82E208368082AD3F8603205D09906C4
:1035500009D50549406905F094BC9B0603D503498C
:10356000406905F08EBC7047CFC8000065A8000018
:1035700038B50D4609780446FFF7DAFF6A78072A5E
:1035800011D8A36893F82F1091420CD083F82F2004
:10359000A368D3F860329B0605D560690249BDE88F
:1035A000384005F06EBC38BDD8C80000F8B5836857
:1035B0009A8F0546002A4ED0D88F00284BD0413034
:1035C000184403F142060346C41AB342A4B2194692
:1035D0000DD311F80179202F3BD01946013B087813
:1035E000202804D001349E42A4B21946F5D9631CA8
:1035F0004E1C121B1944304606F032F9A9688A8F16
:10360000121B92B28A870A440023614282F8423038
:1036100009B2284605F06AFCAB68D3F860329A0616
:1036200003D50D49686905F02CFC33460B4A082187
:10363000284605F069FD2846FFF7FCFEAB68D3F885
:1036400060329B0607D568690549BDE8F84005F07A
:1036500018BC0B46B8E7F8BD6AA80000A7C3000075
:103660006EA800002DE9F04104460D4617460AB148
:10367000FFF7E0FEA368D3F86022D88F520700F16D
:103680004200034421D5184606F0AFF8DFF8508019
:103690000646013E14D2204650F8083F9A8FDA873A
:1036A00005F0FCFB28B107B11DB10B49606905F0BD
:1036B000E8FB6942204609B2BDE8F04105F016BCBE
:1036C0006069414605F0DDFBE3E7044A0821204636
:1036D00005F01AFDDFE700BF55C20000A7C30000D8
:1036E0009FC1000013B583688DF80710D3F86022DE
:1036F0000446D00723D5D98F9A8F8A421FD0481C01
:10370000D8870B449DF8072083F84220A368D3F89C
:103710006012890711D5D3F8603260690B4913F044
:10372000040F18BF2A2205F0ACFB204605F0CAFBA7
:1037300018B10749606905F0A4FB02B010BD012271
:103740000DF10701204605F0ECFCF6E7CCC80000BF
:1037500055C2000083680A4A1B6810B5044602215E
:1037600005F0D2FCA368D3F860329B0707D520464A
:10377000FFF7D6FE2046BDE81040FFF7A7BE10BDFC
:10378000A7C300002DE9F047044690460E460029E5
:103790006ED00025735D202B25D0093B042B22D948
:1037A000DFF8D090304606F020F8A368598D80B23B
:1037B000401BA1EB0803984206EB050A15D95046B9
:1037C000002710F8012B202A06D0A2F1090CBCF129
:1037D000040F02D80A2A31D03B4608EB0702914277
:1037E0002BD90137EDE70135D4E753460027B8421E
:1037F00017D013F8012B0A2A05EB07091BD16069C2
:1038000005F036F93A465146204605F00EFC1949B6
:10381000606905F0E6FC4146204609F10105FFF725
:103820002BFE6069711905F0DCFC60691149BDE887
:10383000F04705F0D6BC0137D9E71F46606905F0AF
:1038400017F93A465146204605F0EFFB3D44735DBB
:10385000202B0BD0093B042B08D96069494605F0A1
:10386000C0FC41462046FFF707FE9BE70135EEE727
:10387000BDE8F08755C200002DE9F04F0E4600214B
:103880008DB0044617460D4607AA304601F10108DF
:10389000FFF7AAFDB8B99DB127B13A4608212046E5
:1038A00005F032FCDFF88080DFF880A0DFF880B020
:1038B00000214B1C07AA30460493FFF795FD60B921
:1038C0000DB0BDE8F08F006810B105F08EFF80B23A
:1038D000854238BF05464146D6E70368D0F80490D4
:1038E0001148059305F081FF059B07468BB11A78B7
:1038F0007AB1CDE901380095434652460821204669
:1039000005F002FCB9F1000F05D16069594605F0D8
:1039100068FC0499CDE76A1C02EB470292B2494663
:103920002046FFF72FFFF4E7F9C80000E1C80000C8
:1039300055C20000F7B5064608680D46B8B105F057
:1039400054FF84B20B4F384605F04FFF2B680A4AEC
:10395000009704440821304605F0D6FBA4B26968FC
:103960002246304603B0BDE8F040FFF70BBF0446E7
:10397000E8E700BFF5C80000DCC6000010B5074945
:10398000044605F042FF38B10549204605F03DFFE9
:10399000B0FA80F0400910BD0120FCE7EBC8000040
:1039A000EEC8000010B58368D3F860329B06044669
:1039B00003D50449406905F025FCA368024A9A62D0
:1039C000002010BD72A800001800500008B58369DF
:1039D000034A1B68082105F00EF8002008BD00BF4F
:1039E000FCC800007FB50F4E04460025A268E068C1
:1039F0000DF10E0302F5A172012105F08BFCBDF85B
:103A00000E00A36850B103F5A173009332462B4614
:103A10000821204604F0EFFF0135E7E783F8420173
:103A200004B070BD0CC9000010B58368D3F86032D3
:103A30009A06044603D50749406905F0E3FBA368ED
:103A4000D3F860329B0603D50349606905F0DAFBC1
:103A5000002010BD79A800007EA80000022907B54B
:103A60000DD1536801930E4B009313680D4A012149
:103A700004F0C1FF6FF0150003B05DF804FB83682C
:103A8000094AD3F8603213F0020F4FF00801074BD8
:103A900018BF1346064A04F0AEFF0020ECE700BF53
:103AA00023C900001AC9000068BA000016C9000046
:103AB00038C90000F0B5012985B004460DD053681F
:103AC0000193574B00931368564A012104F093FF6A
:103AD0006FF01505284605B0F0BD8368D3F8603255
:103AE0009A0603D55049406905F08CFB6FF0F90147
:103AF0002046FFF7ABFCFA212046FFF7BDFCA0688B
:103B000000254FF48072294600F5A1708DF80B5006
:103B100005F0C8FE4549606905F074FB606904F072
:103B2000A7FF4FF47A766068036801221F690DF1E0
:103B30000B0103ABB847039B53B9013E4FF47A70B6
:103B4000B6B206F0E4FB002EEDD16FF0850531E052
:103B50009DF80B30A2681B2B57D092F842111B29FD
:103B6000E1D1522B51D11544002385F8423192F80E
:103B700043115B2951D102F5A2701F46022610F8AD
:103B8000011B01363B29B6B22AD1B6F5807FDCD0C5
:103B900006F5A1701044002310F8015B55BBFA2B09
:103BA00028BFFA23FA2F53853B4628BFFA2382F811
:103BB00042511385A368D3F860329B0603D51C4994
:103BC000606905F01FFB002D84D0A368194A9A6232
:103BD0000321194A204604F00EFF6FF0070579E72C
:103BE00007EB870301EB4303303BB6F5807F9FB2C1
:103BF000C5D1AAE703EB8303013605EB4305B6B253
:103C0000303DFF2EABB2C7D99FE751190135ADB298
:103C1000092D81F8423186D9002382F8423194E798
:103C200023C900001AC9000084A8000047CD000085
:103C300088A800001800500049C900002DE9F04F85
:103C4000074689B01546894621B90324204609B0A4
:103C5000BDE8F08F104605F006FC0028F5D04FF0C7
:103C600000084146022424E05C463CE029460AF56F
:103C7000A17005F06FFD064600284ED005F0B5FD99
:103C800082B2601C01323146304405F0E9FD224623
:103C90005946304605F0FBFD4FF020033355BAF886
:103CA000400004440134AAF8404008F1010800240F
:103CB00001994B1C03AA48460193FFF795FB064662
:103CC000F8B131680022284604F0E7FC0028EFD163
:103CD000D6F800B0D7F808A0BBF1000FC4D0584602
:103CE00005F083FD84B2BAF8402001322244B2F5D7
:103CF000807FBBDD0A4A2B460321384605F004FAD3
:103D00000124B8F1000FA1D0B8682A4600F14001A3
:103D100000F5A17004F0D8FF98E70224F1E700BF96
:103D20004CCD00002DE9F84305464FF02003EFF39A
:103D3000118683F31288BFF36F8F104B1C68002C21
:103D400038BF00249CB10E4FDFF838804FF00C09CB
:103D5000D4E90132002D08BF13462BB198F8142086
:103D600009FB02F2B85C98472468002CF0D186F376
:103D70001188BFF36F8FBDE8F88300BF680A002089
:103D8000740A0020F810002000F01F0301229A405E
:103D90000A4BBFF35B8F400903EB800050E8003F04
:103DA00043EA020140E8001CBCF1000FF6D1BFF36A
:103DB0005B8F1A4214BF012000207047800A002048
:103DC00030B51D4B1D7DBFF35B8F05F01F03012236
:103DD0009A401A4B690985B0D04303EB810353E83D
:103DE000001F01EA000443E8004CBCF1000FF6D1CB
:103DF000BFF35B8F114217D0114C0C2202FB05421E
:103E000007CA01AB83E807000E4A7AB193E80700BE
:103E100005F074FD0020FFF785FF0C236B430022A3
:103E2000E118E250C1E9012205B030BD82F31188EA
:103E3000BFF36F8FEEE700BFF8100020700A00207C
:103E4000740A0020FD9800002DE9F041374BDFF89F
:103E5000F4801C7D88B007462046FFF795FF60B9C7
:103E60006E463A462146304605F045FB96E8070087
:103E70000C2505FB048585E807000C23634308EB4C
:103E8000030218F80300650904F01F06C8B37B1C81
:103E90000FD0D2F808E02648264A4FF4004C002103
:103EA0000023ECFB0E01FCF72BF90121381A06F078
:103EB0000EFA02F0C1FF0120FFF734FFBFF35B8F62
:103EC0001D4B0122B24003EB850353E8001F114351
:103ED00043E800100028F8D1BFF35B8F0C2303FBED
:103EE000048494E8070005AB83E80700134A1AB17D
:103EF00093E8070005F0EFFCFFF762FF03F076F9A7
:103F000001200F4ABFF35B8F0123B340DB4302EB79
:103F1000850555E8002F1A4045E800210029F8D111
:103F2000BFF35B8F08B0BDE8F08100BFF810002040
:103F30003F420F0040420F00700A0020D798000057
:103F4000800A0020740A0020014803F045BE00BF2B
:103F500014B0000008B5D0B14368042B11D1002281
:103F60000368BFF35B8F53E8001F012903D143E8C7
:103F700000200028F7D1BFF35B8F074808BF104629
:103F800008BD3BB1006802F065FE0020F8E76FF461
:103F9000E040F5E70148F3E7E98FFFFFEA8FFFFF15
:103FA00010B5044618B90D4B0D485B689847616819
:103FB00008290DD031F004030AD011F0020108D015
:103FC0000848214606F029F8002323600023636097
:103FD00010BD2068142205F065FCF7E79801002069
:103FE0009ECD0000840A002010B5044618B9164B77
:103FF00016485B6898476368042B23D0082B21D0B0
:10400000CBB92368BBB912484FF0FF324FF0FF33F2
:10401000214602F0E3FB08B923681BB90A4B0D489F
:104020005B68984720681422002105F03BFC636818
:1040300043F002036360206806F038F8636843F0D9
:104040000103636010BD00BF980100209ECD0000F9
:10405000840A0020C4CD000008B508B34368042BCF
:1040600010D101220368BFF35B8F53E8001F0029C2
:1040700003D143E800200028F7D1BFF35B8F0BD1B9
:10408000002008BD53B100684FF0FF324FF0FF33FE
:1040900002F062FD0028F3D00348F2E70348F0E79E
:1040A0006FF4E040EDE700BFE98FFFFFEA8FFFFF0D
:1040B00008B5064906484023142205F093FFBDE8E1
:1040C00008400449044803F0E9BD00BFA00A0020ED
:1040D000840A00202CB000001CB00000034B43F801
:1040E000302003EBC0035960704700BFF801002087
:1040F000014910220A60704710ED00E072B640409E
:1041000080F31188BFF36F8FBFF34F8F30BF62B65C
:10411000BFF36F8F704700BF72B6494081F31188BB
:1041200020BF80F3118862B6704700BF43B2002BF6
:1041300008DB012200F01F0002FA00F05B09024ACE
:1041400042F82300704700BF00E100E0054B420940
:1041500000F01F0053F82220012303FA00F0104062
:10416000704700BF00E100E043B2002BA8BF03F19D
:10417000604301F10101B8BF064B4FEA4111ACBFEA
:1041800003F5614300F00F00C9B2B4BF195483F8BE
:104190000013704714ED00E038B505460C46114693
:1041A0001A46FFF79BFF6AB2002A04F10103AEBF73
:1041B00002F16042064A05F00F014FEA4313DBB2F9
:1041C000AABF02F56142535482F80033284638BD35
:1041D00014ED00E030BFFFF7FDBF00BF0B4A08B58C
:1041E0000B4B22F07F029A60BFF34F8FBFF36F8FAC
:1041F000D3F8882022F47002C3F8882002F050FA25
:1042000003F042F900F0D6F902F054FA0000000081
:1042100000ED00E00A4A0B4993680968C3F8B01042
:104220000949C3F8AC004B6843F080534B6000234E
:1042300083F31188BFF36F8F9368D3F8B000704792
:10424000F8100020C8B1000000ED00E013498A68B2
:104250004FF030001044EFF3098C80E8F01F20206D
:1042600080F31288BFF36F8F0D4F4FF00066CA695D
:104270008A603E60D2F8AC000023C2F8AC3080F314
:10428000118804B5104600F033FABDE8044002F18D
:10429000300090E8F01F8CF309887047F810002078
:1042A00004ED00E01EF0040F0CBFEFF30880EFF305
:1042B0000980816911F8021C0229FFD001B505F0BF
:1042C00025F901BD42F8203C009B42F81C3C0A49FC
:1042D000019B42F8183C029B42F8143C21F001017A
:1042E0004FF0807342F8043C42F8081C0023203A47
:1042F0000265C0F8AC307047158100000C4A0346D7
:10430000906898B113F1160FD0F89C0005D0A0F179
:1043100020029A4206D8834204D281422CBF002157
:10432000012100E00021002908BF0020704700BFE4
:10433000F810002008B5094B98600D46144600F0AF
:10434000D7F9204685F30988002163B681F31188E7
:10435000BFF36F8F0022002303F0DCFEF810002073
:1043600001B572B60B4A906900281EBF0021916109
:1043700005F095FE62B6EFF30580A0F110004FEA5C
:10438000C0000549014409C99847BDE801400349F7
:1043900008470000F8100020F8010020A1430000A9
:1043A000044B9968D869884203D003494FF0805282
:1043B0000A607047F810002004ED00E038B5194B92
:1043C00014469A6A9A6A9A6A0546900719D5586BF4
:1043D0009A6A120615D519B19A6A22F080029A6279
:1043E0009A6A9A6A9A6AD1060ED49B6A9A070BD483
:1043F00000200C4A936A43F0FF039362002323706A
:1044000038BD6FF01500EBE7064B5B681B05EFD579
:104410002946FFF773FF0028EAD080F309880220BD
:10442000E7E700BF00ED00E00D4B9A6A9A6A9A6ACE
:10443000920508D59A6B9A6A120404D518B19A6A43
:1044400022F400429A62064B9A6A9A6AD20558BFD1
:104450009A6A9A6A002042F47F429A620870704712
:1044600000ED00E0074B9A6A9A6A9A6A9A6A9A6A19
:104470009A6A9A6A6FEA02426FEA12429A620020CE
:10448000704700BF00ED00E070B53E4B5B688AB03E
:104490000D46C3F30803002686F31188BFF36F8F20
:1044A00002F07F41B1F17F4F11D102F00C010829D8
:1044B0000DD0120701D4054601260022033B8DF8DA
:1044C0000720032B57D8DFE803F0044E524B354644
:1044D000F3E72C4BDC6A14F002044CD1DA6A002AB0
:1044E00018DBDB6A5B0015D5AB6933F8022C4DF69F
:1044F00002739A420DD003F1604303F626631B78E2
:1045000003B30DF1070201212846FFF757FF0446C8
:1045100000E02C689DF8073093B92022294602A8B4
:1045200005F0B5F9099B46B3C3F3080222B96FEA57
:1045300053236FEA4323099302A9204604F0E4FFC2
:104540000AB070BD104B1B782BB10DF10701012093
:10455000FFF76AFFDBE70D4B1B889BB2002BD9D01E
:10456000FFF780FFD3E70DF107020021CCE70DF143
:1045700007010020ECE70024CCE723F4FF7323F0CD
:104580000103D8E700ED00E029ED00E02AED00E0AE
:10459000024A536943F010035361704700ED00E095
:1045A000EFF30880EFF3098101B57246FFF76CFF66
:1045B00001BD00BF044800232021C2180133302B65
:1045C00082F80013F9D1704700E100E0002080F389
:1045D0001488BFF36F8F06F02BF800201149086094
:1045E000BFF34F8F104880F3088800F031F8202087
:1045F00080F311880D484FF0AA014FF4026205F0D4
:1046000051F90A484FF40261401880F30988EFF32A
:1046100014800221084380F31488BFF36F8FFFF7E3
:10462000DDFD000094ED00E0C025002040270020C3
:10463000064A11680023C1F3072118468B4200D1B6
:104640007047936010610133F8E700BF90ED00E020
:1046500008B572B6002383F31388FFF7E9FF144B04
:104660004FF0FF32C3F88020C3F88420C3F88820BD
:10467000C3F88C20C3F89020C3F89420C3F8982086
:10468000C3F89C20C3F88021C3F88421C3F8882193
:10469000C3F88C21C3F89021C3F89421C3F8982162
:1046A000C3F89C2162B6BFF34F8FBFF36F8F08BD75
:1046B00000E100E0064B9B68834207D1EFF30583DE
:1046C00023B1044A536843F08053536002F074BE30
:1046D000F810002000ED00E0024B034A03480121DE
:1046E00000F06AB8000004200000002040B0000084
:1046F000D0F89C20054B203A1A60054A2021C3E9D6
:1047000001121846012100F061B800BFA00F00207F
:1047100000000B15F0B51E4F00268E4201DB10463F
:10472000F0BD446884B353B104F1FF3C14EA0C0FAC
:1047300018D11F2C16D905681CEA050F12D1202CA0
:104740000568D0F808C0D2B20FD9B4F1004F0ED826
:10475000013CB4FA84F4C4F11F046400072A4CEA53
:10476000040406D96FF01502D9E70824F6E73E24C1
:10477000F4E725F01F05154345F0100544F001044A
:10478000BA60FD6001323C6101360C30C5E700BF04
:1047900090ED00E0034B05225A60BFF34F8FBFF34B
:1047A0006F8F704790ED00E0BFF35F8F014B0022E9
:1047B0005A60704790ED00E010B5034C0123227859
:1047C000FFF7A8FF207010BD7913002008B5084A34
:1047D00000231278FFF79EFF10F1160F03D0054B50
:1047E0000022072800DD08BD98601A610130F8E753
:1047F0007913002090ED00E013490868082810B5EF
:104800001ED8FFF7D1FF114C49680022904201F1F8
:104810000C0105D10E4B1870FFF7BCFF002010BD36
:10482000A26051F80C3C23F01F03134343F0100324
:10483000E36051F8043C43F0010323610132E5E7F2
:104840004FF0FF30EBE700BF4CB0000090ED00E010
:1048500079130020014B1860704700BFA8000020AA
:104860000CB41FB509B90DF10300CDE9020107AB86
:10487000069A0648019302A9FCF748FF029B002212
:104880001A7005B05DF804EB02B07047BD980000E7
:104890004FF02003EFF3118183F31288BFF36F8F82
:1048A0000F4A0123C2F840354FF08042C2F87835F4
:1048B0000C4A1268082A08D10B4A1268052A04D843
:1048C0000A48825C0AB10A4A13604FF08043012211
:1048D000C3F8802581F31188BFF36F8F00207047E4
:1048E00000E00140300100103401001000CE000053
:1048F000380600404FF08043C0B2C3F81C05BFF338
:104900004F8F0549054BCA6802F4E0621343CB6040
:10491000BFF34F8F00BFFDE700ED00E00400FA0594
:1049200020B1034B800143F001031847704700BFDB
:1049300090A800000E4A70B5841AA3100D4C5C4379
:104940000546E4B20C2000FB04200E46402108443A
:1049500004F0E8FF011E05DB074B03EBC4046368AA
:104960009847002128463346BDE87040184700BFED
:10497000BC0F0020B76DDBB698B000002DE9F04108
:10498000104E841BA310104C5C43E4B20C2565430D
:10499000804605F140000F463044402104F0DBFF23
:1049A000011E09DB094A7319C3E90E27084B53F8A6
:1049B0003430BDE8F041184740463B46BDE8F04181
:1049C000184700BFBC0F0020B76DDBB6B9990000D7
:1049D00098B00000002270B5012104461046FFF790
:1049E000C3FB0020FFF7A2FB0F4801F0DBF80F4BE1
:1049F000984215D105F022FA26690D49304603F098
:104A00002DFB00280BDB012535642469084904F1DE
:104A10001C0003F023FB002801DBE564002070BDCF
:104A20006FF00400FBE700BF694A00000000AD0B17
:104A3000D8B0000001460C2309484B4370B5C41898
:104A4000D4E90E5600224033A263184404F0A1FFBB
:104A50002DB132462B460348BDE87040184770BD63
:104A6000BC0F0020BCA6000010B1012804D0704784
:104A7000034B1B6C5B0701D1FFF7DCBF704700BF26
:104A8000BC0F002010B505F040FC4FF47A730C46C3
:104A9000A0FB030103FB0411054AC30B43EA414396
:104AA000BDE81040C90B0120C2E9003101F08AB80D
:104AB0009804002008B54FF02003EFF3118183F331
:104AC0001288BFF36F8F114A136843F0020013F08E
:104AD000010310600CD04FF08042D2F80C34D2F8B1
:104AE0000C2413F0010303D0094804F052FF012302
:104AF00081F31188BFF36F8F23B1BDE80840002018
:104B0000FFF798BFBDE80840FFF7BCBF0C100020BE
:104B1000FC0F002010B505F0F8FB4FF47A730C463B
:104B2000A0FB030103FB0411054AC30B43EA414305
:104B3000BDE81040C90B0120C2E9003101F074B892
:104B4000A0040020084BBFF35B8F53E8002F22F036
:104B5000020143E800100028F7D1BFF35B8FD307B1
:104B600001D4FFF7D7BF70470C1000202DE9F74F95
:104B70004FF080470446D7F8186406F480364FF0AB
:104B80002003EFF3118883F31288BFF36F8F05F0D2
:104B9000BCFB4FF47A730A46A0FB030103FB02112E
:104BA000D7F80C94D7F80C34254BD3F800B0254B2C
:104BB000C50BD3F800A045EA414588F31188BFF33F
:104BC0006F8F214ADFF89880204F2046082103F09C
:104BD00012FF19F0010FDFF88C901D4AB9F81A3056
:104BE0000093204614BF43463B46082103F003FFD1
:104BF000A5EB0B03009320465B46164A0821A5EB64
:104C00000A0503F0F8FE53462046134A0095082192
:104C100003F0F1FE2046114A082103F0ECFEB9F83A
:104C20003630009320460A4A002E14BF43463B46C6
:104C3000082103F0E0FE002003B0BDE8F08F00BFC4
:104C400098040020A00400200BCE000006CE000037
:104C500016CE000030CE000052CE000073CE000011
:104C600056C20000BC0F00207FB500220123CDE911
:104C7000022304ABCDE90433094ACDF800D06B46DA
:104C8000CDF804D004F0BEFE002805DB4FF48042CE
:104C90000023684602F04CF807B05DF804FB00BF43
:104CA000D7990000024AC3B21C2003FB00207047C2
:104CB000BC0F00202DE9F8433A49BFF35B8F06464D
:104CC000012251E8003F41E800200028F9D1BFF35C
:104CD0005B8F33B9344935484B60CB608A6003F051
:104CE000D0F9731E012B32D8012E07D14FF080432B
:104CF000D3F81C3403F00303012B28D005F0B7F9D7
:104D0000044618B92A4B1B78002B44D14FF02003DE
:104D1000EFF3118583F31288BFF36F8F0124254FC2
:104D2000DFF89480DFF894904FF08042D2F8183486
:104D3000D2F81824D2030CD503F00303012B01D0C1
:104D4000012E06D10CB385F31188BFF36F8FBDE838
:104D5000F883ACB12846FFF7DFF94FF08042D2F874
:104D60001835002BE0D139680029DDD03B603B6865
:104D70000123C2F81835C8F88031C9F80030D3E7EC
:104D80000021212002F0E8FAE7E74FF080430222F9
:104D9000C3F80423DBE74FF080430222C3F8082363
:104DA0000546BCE710100020AC0F0020D80F0020F3
:104DB000CA1700200401004000E100E008000040A4
:104DC0000A2838B5064D044603D128680D2104F0A1
:104DD00034FE2868E1B204F030FE204638BD00BF42
:104DE0001410002008B5084B0848186005F0BDF8FD
:104DF00038B10748FFF72EFD0548FCF779FB002086
:104E000008BD6FF01200FBE7141000201CA7000083
:104E1000C14D0000420970B5034602D0012A1DD0E1
:104E200070BD0F4E326951680029F9D00C6803F04B
:104E30001F030125002C05FA03F538BF00248A68FA
:104E40002A4002D04B6830469847002CE8D02368AF
:104E5000002B38BF002321461C46F0E7014EE1E756
:104E6000D4A60000ECA6000030B54068047B01F039
:104E70001F05B2F5005F45EA441585B04FF0000408
:104E800004D1284601F070F9002032E0B2F5804FDD
:104E9000CDE902442FD1B3F5003F0CBF0423052315
:104EA0008DF80830836823FA01F1C9072FD4B2F5D1
:104EB000A03F2CD16A09012A05F01F031C4A03F503
:104EC000E07318BF4FF0A04252F82330DB071ED426
:104ED0000DF107042146284601F0B2F8154B98421F
:104EE00014D1204601F0F6F8134B98420ED06FF023
:104EF0000B0005B030BDB3F5C02F05D0B3F5003FB2
:104F00000CBF02230123CBE70323C9E7039400234B
:104F1000194602AA284600F071FF074B984204D1B7
:104F20000121284601F0DCF8AEE76FF00400E0E76D
:104F3000000300500400AD0B0000AD0B10B501F0F4
:104F4000B9F8044668B901F08DF8084B98420AD1C7
:104F50000748214601F06EF8224605210620FFF79A
:104F600003F9002010BD6FF00400FBE70000AD0B5B
:104F7000154E00002DE9F04347683B7B01F01F050B
:104F800085B00E4645EA43151446CAB902A928461B
:104F900001F056F80446284601F008F9484B9842BB
:104FA00004D06FF0040005B0BDE8F083844205D161
:104FB0009DF8080001F088F8A042F2D10020F2E745
:104FC0004FF000090DF103013046CDE9029901F0DF
:104FD00037F84B46804602AA4946284600F00EFFA5
:104FE000374B984202D06FF01500DCE7804503D1C3
:104FF0009DF8030001F068F8A3054ED5314B324A05
:10500000234093423AD00CD8062B14D004D893B145
:10501000022BE8D104230EE0B3F5801FE3D1012376
:1050200009E02A4A93422BD0B3F5A00F2AD0B3F55A
:10503000800FD8D102238DF8043084F48073C3F339
:105040000023E0068DF8053054BFC4F3401303235A
:1050500021058DF8063017D57B68012101FA06F687
:10506000C3F80865002201A9284600F073FF144B1D
:10507000984214BF6FF01500002094E70723DAE789
:105080000523D8E70323D6E7620541BF7B680121EA
:1050900001FA06F6C3F80C65E4E7E3064FF00003F7
:1050A00054BFC4F3401403241A4601A928468DF8BE
:1050B000044000F0A3FE024B98423FF47FAF92E71A
:1050C0000000AD0B0600F0000600100002004000DA
:1050D000F0B54B79012B26D0032B21D110268B79EB
:1050E000032B1DD1CC790CB1012C19D10A7912B145
:1050F000022A15D10E220B684568B3F5164F2D68AC
:1051000065D02DD8B3F5165F64D016D8B3F5966F79
:1051100062D00AD8B3F5967F61D0B3F5167F61D01F
:105120006FF0850052E00026D9E7B3F5166F5CD02A
:10513000B3F5965FF4D1374B3CE0B3F5E14F57D070
:1051400007D8B3F5615F55D0B3F5964FE8D1324B30
:1051500030E047F61227BB42E2D14FF4000329E0CA
:10516000B3F5613F48D013D8B3F5963F47D009D87F
:105170004DF6C027BB4244D0B3F5614FD0D14FF4B8
:105180006B0317E0B3F5E13FCAD14FF0EB7311E0C9
:10519000B3F5612F38D008D8204FBB4237D0B3F5D4
:1051A000E12FBDD14FF0E86304E01D4FBB42B7D102
:1051B0004FF08053C5F82435036903C934432243B3
:1051C0000433C5F86C2583E803000020F0BD4FF4DC
:1051D0001D03EFE7134BEDE74FF49E23EAE74FF48F
:1051E000A033E7E74FF41C33E4E74FF41D23E1E776
:1051F0000D4BDFE70D4BDDE74FF06C73DAE70C4B3F
:10520000D8E74FF46503D5E74FF07063D2E74FF06E
:105210008063CFE700B0130000A04E0090D00300E1
:1052200040420F000050270000C0750000F03A0017
:1052300000903A0100F01F0240090128044B02F5DA
:10524000E07218BF4FF0A043890043F82210704766
:1052500000030050F8B5066905460F4604F007FF45
:1052600010B9204B1B7883B94FF02003EFF3118462
:1052700083F31288BFF36F8F284604F0A0FC28BB8D
:1052800084F31188BFF36F8FEEE76424284604F09F
:1052900096FC70B9012004F0CFFD013CF6D100214D
:1052A000212002F059F8F0E784F31188BFF36F8FE3
:1052B000F5E74FF02003EFF3118483F31288BFF377
:1052C0006F8F284604F07BFC0028EDD03146012288
:1052D00001F8147F284604F005FD84F31188BFF31C
:1052E0006F8FF8BDCA17002000F01F024009012887
:1052F000044B02F5E07218BF4FF0A043032143F8BE
:10530000221070470003005000F01F0140090128DF
:10531000044B4FF0010218BF4FF0A0438A40C3F87E
:1053200008257047000300502DE9F041D0F80480B3
:105330000769D8F800400023C4F800353860456894
:105340000646E868421C04D0FFF7DEFFE868FFF776
:10535000CBFF2869431C06D02B7F002B14BF0321F1
:105360000021FFF767FF6869421C04D0FFF7CCFFFC
:105370006869FFF7B9FFA869431C06D06B7F002B53
:1053800014BF03210021FFF755FFD5E903122B6855
:10539000C3F80C15C3F81425D5E90512C3F8081590
:1053A0003169C3F8102504313046FFF791FE0546F8
:1053B000002846D1D8F80430990719D507F116000E
:1053C00000F0F0FF224B98423ED1B87DC30003F1BC
:1053D000804303F5F83304F10C0204F59071C3F82F
:1053E0001015C3F814251B4A01238340C2F8043565
:1053F0000823C4F8003598F808305BB9C4F81031B8
:10540000D4F8103107F11503C4F834350123C4F87A
:1054100038352360D8F804309A075CBF4FF48072A7
:10542000C4F80423DB0644BF4FF48003C4F80433FC
:1054300014370023C4F84475C4F848350123A36029
:10544000E3602846BDE8F0816FF00405F9E700BF8E
:105450000000AD0B00F00140194970B5044622F080
:105460007F460868C1E90023A6F50013101AB3F5BA
:10547000400F4FF000050AD2124B19680A060B0ABA
:105480009219114943F10003C1E90023012502F0FB
:10549000EDF8A30003F1804303F58833D3F84025EA
:1054A000B2420BD11DB94FF40002C3F84025074B9F
:1054B0004FF4803000FA04F4C3F8444370BD00BFD9
:1054C000C004002038100020A80400200010014073
:1054D00010B501238340114ABFF35B8FDC4352E8D0
:1054E000001F01EA040C42E800CEBEF1000FF6D125
:1054F000BFF35B8F4FF4803202FA00F002F180427A
:1055000002F58052C2F80803BFF35F8FBFF36F8FBD
:105510000B4214BF0120002010BD00BF341000203A
:105520000123124ABFF35B8F834052E8001F1943E7
:1055300042E8001CBCF1000FF7D1BFF35B8F0C4AAF
:105540004FF480338340C2F804330A4BBFF35B8FC0
:105550001B68BFF35B8F23FA00F0C30742BF064B03
:105560004FF40032C3F80021704700BF3410002010
:10557000001001403010002000E100E00D4B1B68DE
:10558000190A1806BFF35F8F0B4BD3F80435C01808
:1055900041F10001B3F5801F0AD2084BD3E9002383
:1055A000994208BF904203D210F1807041F100018E
:1055B000704700BF3810002000100140A8040020F0
:1055C0002DE9F04F85B016461F460546FFF780FFD0
:1055D0000190FFF7D3FFB94208BFB0427FD2B6EBCC
:1055E000000867EB010900234FF080724B4508BFAC
:1055F0004245C0F08580444B03EB0513D3E90223F9
:105600009F4208BF964254D04FEA85094FF4803B31
:1056100009F1804905F150080BFA05F209F58839BE
:105620004FEA88081FFA88F80292384AD9F84005EC
:1056300026F07F4308F1804808F588381C469346D9
:10564000D2F804A5A0EB0A0020F07F402AF07F41A9
:105650000128C9F8401505D10393132004F057FE23
:105660002A4A039B02990AF1020CA4EB0C0020F0D9
:105670007F40B0F5000F88BF64460020C8F80000E6
:10568000D8F80000CBF8441324F07F40C9F8400557
:10569000DBF80405824506D0201A023820F07F404E
:1056A000B0F5000F19D8E41A24F07F44321947F1FD
:1056B0000003154C290104EB0510C0E902230E9AE2
:1056C0000F9B625043600024019B13B12846FFF7F3
:1056D00027FF204605B0BDE8F08F2046B0E7012344
:1056E0000B4ABFF35B8FAB4052E8001F194342E8FF
:1056F00000100028F8D1BFF35B8F32463B46D8E755
:105700006FF01504E0E700BFB00400200010014076
:105710003010002073B5194B194D00244FF0FF30A5
:105720004FF0FF31C5F80845C3E902014FF480335B
:10573000C5F80433134B02264FF400320121C5F89B
:1057400004631120C3F880212246FEF70DFD1120CD
:10575000FEF7ECFC0C4A012313600C4A2B6013602B
:105760000B4B0C4A0093019400232046FFF728FFBF
:105770003046FFF79FFA204602B070BDB00400200B
:105780000010014000E100E008100140341000204A
:1057900059540000FFFF7F002DE9F743344CD4F843
:1057A00004339A0709D5334B1A6832B100221A60C4
:1057B000314A1B681368013313604FF02003EFF385
:1057C000118283F31288BFF36F8FD4F80433DB03A5
:1057D00012D5BFF35B8F294B53E8001F21F0010066
:1057E00043E80006002EF7D1BFF35B8F244B00295E
:1057F00036D11968002933D1002382F31188BFF311
:105800006F8F53B3FFF7BAFE06464FF02003EFF356
:10581000118083F31288BFF36F8F1A4BD3E902898B
:10582000494508BF46454FF000021ED34FF0FF36F2
:105830004FF0FF37D3E90015C3E902671A604FF450
:105840008033C4F8483380F31188BFF36F8F21B1E0
:10585000009542464B460020884703B0BDE8F083E0
:10586000002119601B680123C7E71146EBE700BF61
:1058700000100140041101403810002030100020B9
:1058800040110140B0040020144B13B5B0F1FF3FAC
:1058900008BF1846441E002C1EDD9C42A8BF1C46B3
:1058A000FFF76CFE0E4B0F49D3E90023801AB0F5C9
:1058B000000F28BF002401300444084800918442AE
:1058C00028BF044612194FF00000019043F1000375
:1058D000FFF776FE02B010BD0024E1E7FFFF7F0076
:1058E000C00400205954000008B5FFF747FE024BE2
:1058F0001B68C01A08BD00BFC0040020034B186815
:10590000A0F1080358425841704700BF3001001011
:10591000064B1B68082B06D1054B1B68052B02D8CC
:10592000044AD05C70470020704700BF300100106F
:1059300034010010DECE0000024AD2F80034002B01
:10594000FBD0704700E0014010B5FFF7D7FF40B132
:105950004FF080430022C3F80C21C3F81021C3F894
:105960003825FFF7CBFF002846D04FF080525B4B25
:10597000D2F80414C3F82015D2F80814C3F824157B
:10598000D2F80C14C3F82815D2F81014C3F82C154B
:10599000D2F81414C3F83015D2F81814C3F834151B
:1059A000D2F81C14C3F84015D2F82014C3F84415DB
:1059B000D2F82414C3F84815D2F82814C3F84C15AB
:1059C000D2F82C14C3F85015D2F83014C3F854157B
:1059D000D2F83414C3F86015D2F83814C3F864153B
:1059E000D2F83C14C3F86815D2F84014C3F86C150B
:1059F000D2F84424C3F87025FFF78AFF10B1384B62
:105A0000384A1A60FFF784FF18B1374BFB22C3F8FE
:105A10001825FFF77DFF48B13449354B0A681B68EC
:105A200022F00F0203F00F0313430B60FFF770FF28
:105A300018B1304B4FF400721A60FFF75FFF48B1A6
:105A40004FF08043D3F80024D20744BF6FF0010227
:105A5000C3F80024284B1B68082B0ED1274B1B686A
:105A6000052B02D8264AD35C3BB14FF01023D3F864
:105A700008224FF08043C3F858254FF01023D3F885
:105A80000022002A03DBD3F80432002B22DA1D495E
:105A90000123C1F80435FFF74FFF4FF01020122407
:105AA000C0F80042FFF748FFC0F80442FFF744FF88
:105AB0000023C1F80435FFF73FFFBFF34F8F1249B2
:105AC000124BCA6802F4E0621343CB60BFF34F8FFE
:105AD00000BFFDE70E4B0F4A1A6010BD00C000402A
:105AE0008C5600404881030000F00040E40E004066
:105AF000580200104096024030010010340100109E
:105B0000D8CE000000E0014000ED00E00400FA05FE
:105B1000040100200090D00370B501250368B3FA9A
:105B200083F2202AC2F11F0414D0BFF35B8F05FA61
:105B300004F223EA020250E8006F9E4204D140E8DA
:105B4000002CBCF1000FF6D1BFF35B8FE6D1024809
:105B50000C7070BD0148FCE70000AD0B0200AD0BFE
:105B60000368CB40DB0710B515D4012303FA01F11C
:105B70000368BFF35B8F41EA030250E8004F9C4289
:105B800004D140E8002CBCF1000FF6D1BFF35B8FCD
:105B9000EED1024810BD0248FCE700BF0000AD0B8B
:105BA0000400AD0B044B1A7922B9012218609A80C7
:105BB00002487047024870473C1000200000AD0BBF
:105BC0000C00AD0B10B1012820D070474FF080437E
:105BD000D3F81824D3F8181411F4803F194611D0C3
:105BE00002F00302012A0DD1C3F818250C4B002244
:105BF0001A601B684FF080430222C3F8042301227D
:105C00009A6070470023C1F81835EFE7054B002272
:105C10001A601B684FF08043C3F804031860704794
:105C2000040100400001004038B510B1012818D02F
:105C300038BD4FF080430222C3F80823184A106091
:105C40001268184A0121116042F210751C46D4F8FE
:105C50001834DB03ECD5012004F0EEF8013DF6D159
:105C6000E6E7114B4FF080440022C4F808031A60A5
:105C70001B680E4B42F210751860D4F80C34D4F83F
:105C80000C24D20303F0010305D523B1012004F055
:105C9000D3F8013DF1D1064B00225A71C8E700BF8D
:105CA000040100400C0000400001004004000040DE
:105CB0003C100020164B1A6810B56AB100221A6019
:105CC0001B684FF080430122C3F80823114B587919
:105CD00010B95A711B6898470F4B1A6872B10022AD
:105CE0001A601B684FF08043D3F81824D3F81814B7
:105CF000920704D10122C3F818259A6010BD022230
:105D0000C3F80823034BBDE810401B680120184767
:105D1000000100403C10002004010040036803F033
:105D20001F025B09012B0260024818BF4FF0A04020
:105D3000704700BF0003005070B500F108030C4C21
:105D400034F81330DA0505460E4607D5C3F343236E
:105D500004EBC30254F8333052689847A3682BB160
:105D6000E26831462846BDE87040184770BD00BF64
:105D700008010020124B083010B433F81020D10570
:105D80001BD5C2F3432122F4F85223F8102003F16B
:105D90001004002034F8022B12F4807F03D0C2F3E9
:105DA0004322914209D001303028F3D1002243F838
:105DB0003120044810BCFFF7D3BE10BC704700BFB1
:105DC000080100207C01002038B50A4C00F10805CC
:105DD00034F815309A0606D55B0B074A03F5A27313
:105DE000002142F82310FFF7C5FF002324F81530E7
:105DF00038BD00BF08010020006000402DE9FF41D0
:105E00001D46044617460B4609B34D4E00F10808DF
:105E100036F8182002F02202222A03D1494804B0A1
:105E2000BDE8F0810022CDE900228DF80E208DF82A
:105E30000F200DF10E010DF10F0204F009F836F8F4
:105E4000183023F0020343F0010326F8183097B10D
:105E50003B483E787A6804F1080330F813108F0746
:105E60000CD5002ADAD130F8132022F01C0242EAC5
:105E7000860220F81320CDBB3348D0E721F0200163
:105E8000C904C90C20F81310002AECD0032EC5D881
:105E900017782EB92D4A07F5A27142F82160E2E782
:105EA000BA0002F1804202F5C0424FEA042ED2F855
:105EB00010C52CF0030CC2F810C5D2F810C52CF494
:105EC0004F3C2CF4407CC2F810C5D2F810C50EF43B
:105ED0007C5E4CEA064C41EA47314CEA0E0C41F03C
:105EE000200120F81310C2F810C5BCE7D5E90067FF
:105EF0002046FFF73FFF002EBED0114D2B689E427B
:105F000004D16B689F4201D1002209E010480DF1D5
:105F10000F01FFF701FE0C4B984280D19DF80F2036
:105F200045F8326005EBC20308345F6035F8143081
:105F300043EA422343F4807325F814309CE700BF02
:105F4000080100200400AD0B0000AD0B0060004014
:105F50007C010020F0B5044685B0154609B300F178
:105F60000807314E36F81730980701D49A0658D4EE
:105F700013F01C0F02D04B78012B52D001238DF867
:105F80000F300023CDE900134A1C8B1C20460DF175
:105F90000F0103F05DFF36F8173043F0030326F8D6
:105FA000173015B9214805B0F0BD1F4E04F10807A0
:105FB00036F81700830734D595F800C0614689008C
:105FC00020F0200001F18041C00401F5C041C00C67
:105FD00026F817000023C1F810356A78002AE1D0AE
:105FE000D1F81035AD7823F4991323F4F853C1F8A0
:105FF0001035D1F810E5230203F47C53120443EA70
:106000000E0302F440322D05134305F4801540EAD7
:106010004C302B4340F0200026F81700C1F8103513
:10602000C0E70348BFE700BF080100200000AD0B38
:106030000400AD0B014BC3E90201704708010020C9
:106040000830054B33F810309A0643BF5B0B03480A
:106050000B700348704700BF080100200000AD0B23
:106060000400AD0B38B50E4C94F87850B5B96022E9
:10607000294604F1100003F015FC0620FEF756F83F
:10608000084B09481D601B68084B4FF00042C3F8DD
:106090000423012384F87830636738BD0448FCE7A3
:1060A000080100207C6100400000AD0B0060004052
:1060B0000500AD0B034B93F87800003818BF0120A2
:1060C000704700BF0801002001460148FFF748BDA6
:1060D0007801002001460148FFF71EBD780100202D
:1060E00037B51F4B00F10802044633F812309A0608
:1060F0001DD513F002051AD15B0B9A0002F1804006
:1061000000F5C24002F1804202F5C042056000681D
:10611000D2F8100540F00100C2F8100529B10122A3
:1061200002FA03F30F4AC2F8043303B030BDC3F3DD
:106130008203042B10D0052B10D001A80194FFF787
:10614000EDFD019BD0F81015D94001F0010102319D
:10615000204603F0C4FEE8E70321F9E70221F7E750
:1061600008010020006000400E4B00F1080233F8E7
:106170001230990613D59A0711D45B0B01229A406D
:106180009B00094903F1804303F5C043C1F808238C
:10619000D3F8102522F00302C3F810257047002120
:1061A00003F09DBE08010020006000400E4B00F18E
:1061B000080213B513F81230DB07044611D5FFF7B8
:1061C000D3FF2046FFF700FE01A80194FFF7A6FDCC
:1061D000019B03F5E073022240F82320034802B03C
:1061E00010BD0348FBE700BF080100200000AD0B15
:1061F0000400AD0B2DE9F04F644B6548654900255F
:1062000087B001222C461E6836B1D0F804631642CE
:106210001EBF1C601E68154304338B424FEA4202C6
:10622000F1D15D4F3B687BB34FF0A0435B4ED3F899
:1062300020250492C3F82025D6F820350593C6F80A
:10624000203500960DF110094FF000084FF0010BBA
:10625000D9F80030F3B908F12008B8F1400F09F17E
:106260000409F5D13B603B6800994FF0A043D3F897
:1062700020250492C3F82025009BD3F820350593F0
:10628000C1F820351343DDD10124002D66D107B0BC
:10629000BDE8F08F93FAA3F3B3FA83F308EB030698
:1062A00006F108023E4B039633F81220C2F3820334
:1062B000F40801939A4604AB06F007000BFA00FCC1
:1062C000185D20EA0C00185503A89108FFF726FD79
:1062D000039C04F5E0744B0750F82440C4F30144D8
:1062E00023D551463046FFF727FD03A80396FFF755
:1062F00015FD039A02F5E072E4B250F82220C2F3D1
:106300000142944207D10021304603F0E8FD2146C6
:10631000304603F0E4FD03A80396FFF7FFFC039B60
:106320000BFA03F3C0F8203592E7022C0CBF0321CF
:106330000221304603F0D3FD019B032B04D0022C35
:1063400007D1BAF1010FE6D151463046FFF7F4FC10
:10635000E1E7032CDFD1BAF1020FF4E795FAA5F3D8
:10636000B3FA83F304FA03F29B0003F1804303F5CD
:10637000C04325EA0205D3F81005D3F81015C0F381
:106380000520C1F30141FFF7D7FC7EE70061004023
:1063900000600040206100407C610040000300502C
:1063A0000801002001460148FFF7B6BB8401002028
:1063B000F8B50779224E0C460C2179430546701832
:1063C000037A002B3AD1725062684260697928687A
:1063D0009C46DAB2914229D840F30730FDF7A6FE79
:1063E0002B686278D3F80415164821F0030102F0F7
:1063F00003020A43C3F80425D3F80815A27821F054
:10640000030102F003020A43C3F80825D3F810156C
:10641000227821F00F0102F00F020A43C3F8102581
:106420000C2303FB076601233372F8BD9A0002F5C3
:10643000A072013340F802C08258CAE70248F4E76C
:10644000441000200000AD0B0500AD0B03680122D5
:106450001A600379034A0C2101FB032302221A72FA
:10646000704700BF441000200368044901221A61EC
:1064700003790C2000FB03131A72704744100020AC
:106480002DE9F0410E4C0F4F0F4E00254FF4803890
:10649000236873B1D7F8043308FA05F21A4208D01A
:1064A00000232360A4F50040236880B2D6E90031C0
:1064B00098470135042D04F10404E9D1BDE8F081C9
:1064C00040810040008000404410002010B5144C72
:1064D000144A1549032323616361144BA261E361EC
:1064E0004FF4806323620023A3626362E362226647
:1064F0000F4A6266E01D1022A2662367E3666367A7
:1065000003F048F9BFF35F8F0A49204603F042F9D0
:10651000BFF35F8F2023A371BFF35F8F10BD00BF58
:1065200050100020E4CE0000EDCE0000CA13002081
:10653000BA130020F1CE00002DE9F74F134E0F469D
:106540001946134B9246A3EB0608124A4FEAE8039A
:10655000814602FB03F800254FF0180BBD4203D122
:10656000284603B0BDE8F08F39F91540002C0BDD4B
:10657000A04509D3013C0BFB04600191D0470028E2
:10658000EFDB01990135E9E70020F6E7BCA6000042
:1065900034A70000ABAAAAAA0E4B70B553F820404E
:1065A000013053F82060A64200D870BDD4E9003510
:1065B0002846984765B1EB6830B10028B8BF404223
:1065C000FF28A8BFFF2018705A7842F001025A70C5
:1065D0000834E8E7B4B10000034A044B02609B1A98
:1065E0000348DB1058437047BCA6000034A70000E6
:1065F000ABAAAAAA014B986898307047F8100020FF
:1066000070B5154B154A88B006AEB82505FB0035A8
:10661000044603460821304601F0C4FC0F23012242
:10662000CDE903320E4A0F4905960023CDE9013327
:10663000182303FB04234FF4B070009300FB0411F4
:10664000094B4FF4A072284600F07AF96B7B23F0D7
:1066500004036B7308B070BDC8040020F8CE0000BE
:10666000F8100020E02500202D6B000008B50A4B33
:10667000012202201A70FFF78FFF01F001F90320B9
:10668000FFF78AFF00F0F0F9F9F7B4FE034A137B35
:1066900023F00103137308BDCA17002080050020F2
:1066A0000248034A0021121A03F0FCB8E00300205C
:1066B0008819002080B5DFF8D880B4B088F3088846
:1066C0002D4D2E4E6B69DFF8CC9043F400730024FF
:1066D0006B61E02385F82230EC772C766C76AC7613
:1066E00085F820406B6A43F4E0236B6285F8234011
:1066F000FDF74EFFFDF7FCFC4FF0FF33AB62EB62A2
:10670000FEF77AF8FDF7E8FF40F20113ADF8243008
:1067100006ABB360CDE92D4403F026FC2046FFF71D
:106720003BFF0120164DFFF737FF00F07BFD154BB7
:106730000593012314490094CDE903434FF480628B
:106740004B46CDE901442846F56100F0F9F86A7B33
:1067500022F004026A730746284603F0FDFC204637
:10676000FFF74EFF094BF3604A4639462846347519
:10677000C6F80480FDF7DEFD00ED00E0F810002013
:106780008005002002CF0000C0210020C8040020A6
:10679000602F00206D66000070B50E4B0E4CA342BA
:1067A00001D3002070BDD3E9030141EA000212F0D9
:1067B00003020BD19D685A61AA4201D11C33EEE756
:1067C0005E690E60013259610144F5E76FF0150012
:1067D000E8E700BF8C0300208C030020D3B50C46F3
:1067E00016461F464FF02003EFF3118183F3128802
:1067F000BFF36F8F43695BB123601B68436183699B
:1068000001338361002081F31188BFF36F8F11E0A2
:1068100056EA070203D123606FF00B00F3E702464C
:10682000CDE90067083000F04FFC18B9024B9B68B7
:106830005B69236002B0D0BDF8100020F8B50546B2
:106840000E464FF02003EFF3118783F31288BFF356
:106850006F8F064B9C6A24B987F31188BFF36F8F43
:10686000F8BD20463146A847646FF4E7F8100020D1
:106870004FF02003EFF3118183F31288BFF36F8F82
:10688000094A936A834207D15B6F936281F311884F
:10689000BFF36F8F70471346002BF7D05A6F8242B9
:1068A000F9D1426F5A67F1E7F810002010B504469D
:1068B00008B9054B9C68202204F1780002F074FFAF
:1068C000002084F8970010BDF8100020437B102BA7
:1068D0000ED8102B1CD8DFE803F01D09131B151B65
:1068E0001B1B171B1B1B1B1B1B1B19000B4870477B
:1068F000202B11D00A4A0B48802B08BF1046704746
:106900000948704709487047094870470948704767
:106910000448704708487047084870472FCF000068
:106920003ECF000007CF00000FCF000017CF0000C0
:1069300020CF000025CF000056C2000035CF000058
:106940002DE9F04F85B0984600F15803C0E91633A1
:106950000732129B037322F0070A0423002501F17A
:10696000200B43730AF12007119B85600446C0E9A0
:1069700006550E468373C5730F445246AA215846E6
:10698000DDF84C9002F08EFF109B02930F9B019359
:106990000E9B0093C4E927BA4346C4F8A4503A4674
:1069A00031462046FDF78EFC0E9BA3660F9BE366E7
:1069B000109B6565C4F8648023674FF02003EFF3F4
:1069C000118283F31288BFF36F8F104EB16A616733
:1069D000B46282F31188BFF36F8FB9F1000F11D049
:1069E0001F22494604F1780002F0DEFE84F8975039
:1069F000B3680BB1D3F8A830C4F8A830384605B056
:106A0000BDE8F08F84F87890F2E700BFF81000201E
:106A1000F0B587B000250595109D04950F9D039551
:106A20000E9D0295DDE912670D9D01950C9D009567
:106A30000446FFF785FF7B1C08BFB6F1FF3F05D07A
:106A400056EA070305D1204600F0E2FA204607B0D7
:106A5000F0BD044932463B4604F1180000F07EFDCB
:106A6000F4E700BF79A100002DE9F0472A4E2B4D35
:106A700086B0B046B54205F1300410D300F0DCF921
:106A8000264CDFF89CA04FF4004940F2E73600277F
:106A9000444521D306B0BDE8F04700F0A7BB54F849
:106AA000043C059354F8103C049354F8143C0393AD
:106AB00054F8183C029354F81C3C019354F8203CC1
:106AC000009354E90A2354E90C01FFF739FF54F805
:106AD000303C5D652546CDE7636A5A1C0DD023EA3C
:106AE000E37330463946C9FB0301B94208BFB042DF
:106AF000256804D1284600F08BFA3034C8E74FF4FB
:106B00007A720023F9F7FCFA02460B4605F11800E9
:106B1000514600F023FDF0E78C0300208C03002099
:106B200079A10000004870470063070208B5094CCE
:106B30004FF02002EFF3118382F31288BFF36F8FBF
:106B400003F0B5FBA061FDF77FF90028F0D1FDF758
:106B5000D5FAEDE7F81000202DE9F341044616467A
:106B60001F464FF02003EFF3118883F31288BFF321
:106B70006F8FC368354A6BB180689168884219D0BD
:106B800056EA070318D188F31188BFF36F8F6FF0AF
:106B90000F000CE0916891F90E1021610133E36060
:106BA0009368A36088F31188BFF36F8F002002B051
:106BB000BDE8F0812169F0E791F90E1090F90E30EF
:106BC0009942A8BF19466FF07E029142B8BF1146A4
:106BD0008B422FDD00F08CFA0546CDE900671C489A
:106BE0002246414600F070FA0028E0D04FF0200322
:106BF000EFF3118683F31288BFF36F8F2368216947
:106C00009C420AD04BB193F90E309942A8BF194665
:106C10006FF07E039942B8BF1946A06890F90E3014
:106C2000994209D16DB10A48314600F0F3F86FF08E
:106C30000A00BCE70025D0E700F05AFA0028F2D19C
:106C4000F0E786F31188BFF36F8FF0E7F8100020AC
:106C5000CB17002038B583680446002B37D01F4A75
:106C60009268934236D1DA7B013ADA73C368012B1A
:106C700005D9013BC36000F0B9FA002038BD4FF0E0
:106C80002003EFF3118583F31288BFF36F8F01693F
:106C9000806890F90E30994201D000F029FA204620
:106CA00003F0B9FAA06060B190F90E2022610022D1
:106CB000C0F8B02003F050FA0948294600F0AAF8BD
:106CC000D9E7E06085F31188BFF36F8FD3E76FF0EA
:106CD0001500D3E74FF0FF30D0E700BFF8100020D9
:106CE000CB17002038B504464FF02003EFF3118591
:106CF00083F31288BFF36F8F03F08DFA50B1002237
:106D0000C0F8B02003F028FA29460848BDE838400A
:106D100000F080B8D4E902329A4218BF0133A36070
:106D2000022104F1100003F03AFCEDE7CB1700203C
:106D300037B514461D464FF02003EFF3118183F35E
:106D40001288BFF36F8F836843B1013B836081F387
:106D50001188BFF36F8F002003B030BD54EA0503E4
:106D600006D181F31188BFF36F8F6FF00F00F3E747
:106D70000246CDE90045024800F0A6F9ECE700BF65
:106D8000CB17002010B5084C23685BB1FEF7ACFDB3
:106D900003462068054A0344BDE810401361002102
:106DA00003F095BA10BD00BF2C110020F810002090
:106DB000F8B504460D464FF02003EFF3118683F338
:106DC0001288BFF36F8F104B00224FF4004740F240
:106DD000E73000211A61E7FB040100234FF47A72C7
:106DE000F9F78EF9002C094B09DC1860084B1D607F
:106DF000FFF7C8FF86F31188BFF36F8FF8BD022835
:106E0000B8BF0220F1E700BFF81000202C110020CD
:106E10002811002049B9EFF3058030B9054BDA6934
:106E20009B689A4201D0FDF7F5B981F31188BFF351
:106E30006F8F7047F81000204FF02003EFF311819F
:106E400083F31288BFF36F8F044B9A68D37B013BA7
:106E5000D37381F31188BFF36F8F7047F810002050
:106E600038B502460C480D4D03F06CF9044600B9E4
:106E7000EC68AB684AB95A7BD20606D1A26922B93E
:106E8000DA897F2A01D9EB6138BD9C4201D0FFF736
:106E900079FFEC61F8E700BF18110020F81000201E
:106EA00070B590F90D20437B002A014604DA03F007
:106EB0007F03437303F001F94B7B174A63F07F03B1
:106EC00010464B7350F8203F556A834208BF002399
:106ED000002B38BF0023CBB191F90E6093F90E401F
:106EE000A6420FD0A41B002C0CDD5868C1E900306D
:106EF000016059609068431A5842BDE8704058419B
:106F0000FFF7AEBFAB4201D01B68E4E7C1E9000563
:106F100029605162EEE700BFF810002070B501460D
:106F20004FF02003EFF3118483F31288BFF36F8FC8
:106F3000164B174A98681568A8421D4606D1FFF7F8
:106F400021FF84F31188BFF36F8F70BD0026166098
:106F5000104A1268BAB1C2897F2A14D8427BD2067D
:106F600011D10D4A90F90E60126896420BDB0B4A64
:106F7000904208D01A698A4202DCFFF791FFDEE7EF
:106F8000521A1A61DDE700232B61DAE7F8100020BE
:106F9000241100202C11002028110020C8040020FA
:106FA00070B490F90D30427B002B2DDBD3062BD132
:106FB00083694BBB154962F07F0242730A464D6AF2
:106FC00052F8204F944218BF2346002B38BF0023AD
:106FD000ABB190F90E6093F90E40A6420BD0A41B02
:106FE000002C08DD5A68C0E900321060586070BC9F
:106FF0000020FFF735BFAB4201D01B68E8E7C0E9CE
:10700000002528604862F2E770BC7047F810002045
:1070100010B54FF02002EFF3118482F31288BFF312
:107020006F8F427B510704D484F31188BFF36F8FB5
:1070300010BD22F004024273FFF7B2FF214602485E
:10704000BDE81040FFF7E6BECB17002008B590F969
:107050000D20437B002A014604DA03F07F034373CB
:1070600003F02BF8044B9868431A58425841BDE886
:107070000840FFF7F5BE00BFF81000202DE9F041F1
:10708000064614461D464FF02003EFF3118783F3A5
:107090001288BFF36F8F03F091F887F31188BFF365
:1070A0006F8F6B1C08BFB4F1FF3F08D022462B4600
:1070B00006F118000349BDE8F04100F04FBABDE801
:1070C000F08100BF79A1000010B5074B9868074B0D
:1070D0000C4618601146DDE90223FFF7CFFF20467A
:1070E000BDE81040FDF796B8F810002024110020EC
:1070F000F8B504464FF02003EFF3118683F31288AE
:10710000BFF36F8F437BDA0649B238D18569002D12
:1071100035D103F07F03437302F0CFFF437B8173CC
:1071200063F07F0343731748034653F8207F9F4261
:1071300018BF3D46002D476A1A462B4638BF00232C
:10714000C3B193F90E50A94210D06D1A002D0DDD78
:107150005A68C4E9003214605C600120FFF780FEC9
:10716000012086F31188BFF36F8FF8BDBB4201D0B9
:107170001B68E5E7C4E900273C604462EDE7A173C2
:107180000020EEE7F810002070B50446183003F038
:1071900078F84FF02003EFF3118683F31288BFF3E2
:1071A0006F8F94F90D20637B002A05DA03F07F03CB
:1071B0006373204602F081FF0B4D637BA86843F0A8
:1071C00010036373031B58425841FFF749FE86F3CF
:1071D0001188BFF36F8FAB68A34203D1BDE8704045
:1071E00002F0A6BF70BD00BFF810002010B54FF030
:1071F0002003EFF3118483F31288BFF36F8F084BE2
:107200009A68D37B0133D3730020FFF729FE84F300
:107210001188BFF36F8FBDE8104002F089BF00BF37
:10722000F8100020044B002103F12002C3E90822DA
:107230000846FFF7BDBD00BFF8100020F8B54FF0BD
:107240002003EFF3118483F31288BFF36F8F1B4980
:107250008868437B03F07F03437302F02EFF8A6844
:10726000537B084663F07F03537350F8203F4E6A08
:10727000834208BF0023002B38BF0023CBB192F913
:107280000E7093F90E50AF420FD0ED1B002D0CDDA8
:107290005968C2E900310A605A600120FFF7E0FD39
:1072A0002046BDE8F840FCF7B5BFB34201D01B68EB
:1072B000E4E7C2E9000632604A62EEE7F810002017
:1072C0002DE9F04104460D4654EA050104D1FFF7CB
:1072D000B5FF0020BDE8F0816FF001010A1A4FF000
:1072E000FF3161EB0503012A73F100032ADA03F091
:1072F00008F806194FF02003EFF3118883F3128882
:10730000BFF36F8F114F124BB8681860FFF79EFEE6
:10731000B868104922462B46183000F01FF9BA68A9
:10732000537B43F0100353734046FCF773FF02F0A6
:10733000E8FF301A66EB0601012871F10003B8BFBF
:107340000020C7E76FF00106361AD3E7F8100020D7
:107350002411002079A1000008B50B46013308BFB5
:10736000B0F1FF3F06D1084B9868FFF70DFF4FF0D3
:10737000FF3008BDFFF7A4FF4FF47A7380FB0323AF
:10738000D00B40EA4340F4E7F8100020014B986826
:10739000704700BFF8100020EFF305833BB9054BA1
:1073A0009B68D8897F288CBF00200120704700206F
:1073B000704700BFF81000202DE9F04104464FF05F
:1073C0002003EFF3118683F31288BFF36F8F437BA3
:1073D0001A0705D586F31188BFF36F8FBDE8F081DA
:1073E00023F0200242F00801D20923D14173A3689F
:1073F00013B1204602F069FE04F1180002F041FFCB
:1074000004F158074FF00008A56DBD4200D0CDB97A
:107410000120FFF725FD2046FFF72AFA104B9B6855
:10742000A342D7D1EFF30583002BD3D13046FCF72D
:10743000F1FECFE703F05F0343F00803437302F06C
:107440003CFED4E7284602F040FE05F1180002F0A9
:1074500018FFC5F8B0802846FFF7A2FDD4E700BFAB
:10746000F8100020D3B5DDE90667089CCDE9006778
:10747000FFF72AFE1CB1034B9B685B69236002B0D7
:10748000D0BD00BFF810002008B50648064A0749DD
:10749000121A02F0FCF9BDE80840054A0549064801
:1074A00002F0F5B900000020DC03002084CF0000CA
:1074B0000000000084CF000000000020034B1B6888
:1074C0000BB9FEF711BA0020704700BF3011002041
:1074D00030B5036868B10A4A5268904209D043B196
:1074E000D3E90421D0E90445121945EB0101C3E9B0
:1074F0000421426813605A600023C0E9003330BDA4
:107500008801002038B5134B1C689C4208BF00243A
:10751000FFF7D4FF0546BCB1D4E90401401B61EB81
:10752000E571012871F1000311DB6FF000420023C7
:10753000824273EB010400DA1046074B1B6913B15A
:107540009842A8BF184638BD6FF00040F5E700200C
:10755000F3E700BF88010020F8100020B3F1FF3FDF
:1075600008BFB2F1FF3F2DE9F74F044692469B4614
:1075700073D081604FF02003EFF3118583F31288FD
:10758000BFF36F8F6FF00103B3EB0A084FF0FF32C8
:1075900062EB0B09B8F1000F79F100011CDB3048F8
:1075A000D0E900105B1A62EB0002B3EB0A0662EB53
:1075B0000B07012E77F10003BCBF01260027C4E9A9
:1075C0000467284AD2E9003C93421ED1C4E9002C4A
:1075D000CCF8004054602DE0FFF770FF1AF1010372
:1075E00000934BF100030193DDE90023121843EBF4
:1075F000E073C4E90423E4E7B6EB080067EB090194
:107600006345C4E90401E1D01B68002BDED0D3E957
:107610000489D4E90467464577EB0901ECDAB8EB55
:10762000060069EB0701C3E904015968C4E90031A8
:107630000C605C60136893420BD09C4209D1FFF749
:1076400061FF18B1084B1B69834202D00021FEF78D
:107650001BF985F31188BFF36F8F03B0BDE8F08F7E
:107660003806002088010020F81000202DE9F74F8F
:107670000646FFF753FC4FF02003EFF3118483F32A
:107680001288BFF36F8F2C4DDFF8B0A0DFF8B0B0D9
:107690002E605146D5F800C0DBF800006246D317D3
:1076A0005845DAE90089CDE900230DD060B1D0E971
:1076B0000467B445BB411EDA009BB6EB030C019B8B
:1076C00067EB0306C0E904C6009B13EB0802019BAD
:1076D0004FF0000643EB0903C1E900232E60FFF7DA
:1076E00011FF3146FEF7D0F884F31188BFF36F8F96
:1076F00003B0BDE8F08F18EB06084FF000024FF022
:10770000000349EBE679C0E90423ACEB0606CAE9BD
:1077100000892E60FFF7DCFE84F31188BFF36F8FC2
:10772000836898474FF02003EFF3118483F31288A6
:10773000BFF36F8F0149ADE73011002038060020FC
:107740008801002010B54FF02003EFF3118483F37C
:107750001288BFF36F8FFEF7C7F8064BD3E90023FB
:10776000121843F1000384F31188BFF36F8F1046A2
:10777000194610BD380600202DE9F3471F46294B56
:107780009D68012385F8603085F8613052EA07036F
:1077900016460CBF0123002305F16002804602F06B
:1077A0001CFE81464FF02003EFF3118A83F3128809
:1077B000BFF36F8F95F8604064B90146524640466A
:1077C00002F0A9FD8AF31188BFF36F8F204602B043
:1077D000BDE8F087002385F8603056EA070306D13C
:1077E0008AF31188BFF36F8F6FF00A04EEE7CDE9DB
:1077F00000670D4A0D485146FFF766FC04464FF0FE
:107800002003EFF3118583F31288BFF36F8F2A46AD
:107810004946404602F07FFD85F31188BFF36F8F24
:10782000D4E700BFF810002090010020CB17002003
:1078300038B503464FF02002EFF3118582F312882A
:10784000BFF36F8FC160012181600068834206D160
:1078500085F31188BFF36F8F0024204638BDD0E92F
:10786000003213605A600023C0E9003302F02CFE9E
:10787000294604460148FFF7CDFAEEE7CB17002072
:10788000024A0349034800F080BB00BF56C2000013
:1078900045CF000054CF000038B5064C064DAC4231
:1078A00001D3002038BDD4E90112204602F092FE37
:1078B0001434F4E78C0300208C0300201FB5094B1F
:1078C000029302AB00240093074908488DF80C404E
:1078D0004FF0FF334FF4806200F0F8F8204604B018
:1078E00010BD00BF7BCF0000602F002040060020AD
:1078F0002DE9F04F4B4E85B004464FF0FF384FF066
:10790000FF394FF02003EFF3118783F31288BFF3A1
:107910006F8FD4F8B850D4F8D03085B923F0040272
:107920005D07C4F8D02033D40023CDE90089029349
:1079300004F1C00239463C48FFF794FDE1E7D4F872
:10794000BC202968C4F8B810954201D1C4F8BC1015
:1079500043F00203C4F8D030EB6823F0040343F093
:107960000103EB606B6887F31188BFF36F8F2846C4
:1079700098474FF02003EFF3118B83F31288BFF386
:107980006F8FEB68990723F001020BD4EA600EE0D9
:1079900004F1C80500220121284602F054FC002809
:1079A000F8D1C1E7306823F00303EB6070B9D4F875
:1079B000D03023F00203C4F8D0308BF31188BFF32A
:1079C0006F8FD8059DD4FFF739FC9AE707684FF011
:1079D000000A002F38BF00275346426895420146EF
:1079E0000ED10168BAF1000F14D172683160904273
:1079F00000D1716040F8083BFFF774F9514600234D
:107A0000002FD4D03A68002A38BF002238468A4670
:107A10001746E2E7CAF800107268904208BFC6F83D
:107A200004A0E7E734110020CB170020F8B5C368A5
:107A30009A0704460E46C3F340051FD45F071FD4C0
:107A40000A680AB982680A60D80744BFA36833602D
:107A500037684CBF022501257FB31B4B9B68BB4297
:107A600011D102F004FB80F00100C0B2D7F8D03091
:107A7000D907C3F3800223D53AB140B96FF00F059F
:107A80000023336013E00020F0E71B07F6D4002347
:107A90002360D7F8BC3063B9C7E92E44384602F0FA
:107AA000A1FDE36843F00403E3603368A360284664
:107AB000F8BD1C60C7F8BC40F0E76FF01505DFE7C4
:107AC0006FF01205DCE700BFF8100020F0B589B0B8
:107AD00004460020C4E92E000E9D04F1C000C4E954
:107AE000300004F1C800C4E932001DB32879002831
:107AF00040F2011008BF0120C4F8D00000204FF070
:107B0000FF364FF0FF37CDE90330CDE90100CDE975
:107B10000667094B00942046FEF77AFF25B12968D5
:107B200011B12046FEF7C2FE204609B0BDE8F04084
:107B300002F0A5BA0120DFE7F178000010B50A4C89
:107B400023681BB101232360002010BD00F0D6F88C
:107B50000028F7D00138062803D8044B53F820003A
:107B600010BD034810BD00BF3C110020CCB1000087
:107B7000FE8FFFFFBFF34F8F0549064BCA6802F423
:107B8000E0621343CB60BFF34F8F00BFFDE700BF40
:107B900000ED00E00400FA05F0B4094F094E0A4C6C
:107BA0000A4A0B4D0B494FF0FE333B60526833607D
:107BB000236000242B60C1F80045F0BC104700BFD3
:107BC00000B4025004B4025008B4025098010020DE
:107BD0000CB4025000A00250D0E90012014BC3E9DE
:107BE000001270479801002010B5044630B1636858
:107BF000DB0602D500232360636010BD024B0348FF
:107C00005B689847F3E700BF98010020E8B10000E7
:107C100068B143683BB1DB0607D5BFF35F8F002334
:107C200003601846704703487047034870476FF475
:107C3000E0407047EA8FFFFFE98FFFFF10B5044671
:107C400020B1002211232260636010BD0148FFF7BC
:107C5000A3FFF6E710B20000C0B14368A3B1DB0692
:107C600010D50122BFF35B8F50E8003F40E80021B0
:107C70000029F9D1BFF35B8F012BF3D0BFF35F8FE6
:107C80000020704703487047034870476FF4E04096
:107C9000704700BFE98FFFFFEA8FFFFF70B5D0E9A3
:107CA0000023134C134DC4E90023D0E90263C4E957
:107CB0000263114B086818604868586088689860CB
:107CC000D1E90360D5F81411DE601861CB060DD53B
:107CD0000023C5E94433C5E96D3305F58870904745
:107CE000236805F5DA70BDE87040184770BD00BF25
:107CF000A8010020CC170020B801002010B500F02A
:107D000033F820B1032400F067F8204610BD00F0DE
:107D100035F890B900F0B0F890B90F4B1B681B0E06
:107D2000F02B08D10D4A0E4B12689A420AD0072454
:107D300000F01CF8E7E70624FAE70424204610BD0B
:107D40000024F5E7012000F097F804460028F7D159
:107D5000044B1860D9E700BF28B9025024BA02507A
:107D60000000E0200CBA025000207047002070474D
:107D7000014B1860704700BF04BA025010B511489B
:107D800000F048F800B110BD0F4800F043F800289B
:107D9000F9D10E4C204600F03DF80028F3D10C4BF1
:107DA0000C481C6000F036F801460028EBD100F0CA
:107DB0002DF8044608B1204610BD00F03FF82046DB
:107DC000FAE700BFF0010020E4010020EC010020F0
:107DD000F4010020E801002008B5084800F024F86C
:107DE000074800F021F8074800F01EF8064800F0A8
:107DF0001BF8BDE8084000F00BB800BFF001002000
:107E0000E4010020EC010020E80100200020704780
:107E1000704700BF08B5034B02681B68106898479D
:107E2000002008BDA801002008B5034B02685B686C
:107E300010689847002008BDA801002070B5094CC3
:107E4000094D2069AB68984718B1084B08485B6832
:107E50009847084AEB68206900211160BDE870402E
:107E6000184700BFB8010020A80100209801002099
:107E700034B200005011002070B51A4D1A4E04465D
:107E8000B26828699047F0B95CB1184C2368ABB16F
:107E9000012B1AD0013B23602869F3689847002022
:107EA00070BD124C216839B9114B124A0120C3F838
:107EB00000051368002BFCD101312160F3682869AB
:107EC0009847002070BD0C4870BD0A4A1368002B0B
:107ED000FCD1074A6FF07E40C2F80035FFF748FF3B
:107EE0002368D7E7B8010020A80100205011002026
:107EF00000A0025010B90250E98FFFFF08B5F9F752
:107F00005DFA002008BD034640B1426802F003025A
:107F1000022A06D0032A04D0012A05D06FF01500EA
:107F200070471A68002AF9D00020986070474268AC
:107F300002F00302022A10B5034681600AD0032A28
:107F40000BD10468002000225A6008B1FFF770FCD2
:107F5000204610BD00680024F5E700242046F2E723
:107F60000020704730B58A680C68551C14B14B6806
:107F7000934201DC8D6030BD013B934208BF00227B
:107F80008D600CBFE254A054F5E70FB407B504A907
:107F900051F8040B0191F9F7B1FA03B05DF804EB65
:107FA00004B070470CB407B504AB53F8042B01932D
:107FB000F9F7B2FA03B05DF804EB02B07047038B37
:107FC00013F0070305D10368002B0CBF002003202A
:107FD0007047022B05D1438B002B14BF00200420D7
:107FE0007047012B05D10368002B0CBF0020052032
:107FF0007047002070472DE9F0410D4607461946AD
:10800000281D90461E46FFF792FF044638B13346BE
:10801000424629463846A446BDE8F0416047BDE8DF
:10802000F08110B44FF02004EFF3118284F3128832
:10803000BFF36F8F416110BC0121F9F781BA10B510
:108040000C4640B139B1081DFFF75DFF28B9A368A0
:1080500033F0030301D06FF0150010BD38B50C46A6
:10806000054658B151B10B6843B14B6833B11C227E
:10807000002101F017FC2C61002038BD6FF01500C5
:10808000FBE770B504460E46FFF7D9FF051E31DB4E
:108090004FF02003EFF3118183F31288BFF36F8F4A
:1080A000638B208B4FF6FF75AB4200F007022ED09A
:1080B000022A0ED1013363831546012381F311880F
:1080C000BFF36F8FB3B1002331462046FFF793FF14
:1080D00010E0830701D0062A0ED1002333606368C5
:1080E00093B9C4E90066154662B90A4620460221E2
:1080F000F9F726FA284670BD052A0CBF6FF08505F2
:108100006FF004050023D9E71E606660EBE76FF0AF
:108110000A05F7E7044608B5084611461A46A0477F
:10812000FFF734F9FCF7C6FA00EBC10040884008BD
:108130007047F8B503460C46FFF7F6FFB0FA80F03B
:10814000C0F11F0003EB800CCA00DCF81060171DA3
:108150008DB2063256B9012101FA00F0D968014307
:10816000D960CCF81040DD539D52F8BDF1000431C8
:10817000585AD85303EBC0009E52C5805D52F4E7B5
:10818000043ACB1D0A4423F0070322F00702D21A57
:10819000F0B4D4080360B4FA84F0C0F12400800085
:1081A000C11D00259C60DD60C90803F1100618445C
:1081B000864218D1480040F00100588003EBC10608
:1081C000601A47001D8077809E1823F8311003EB5A
:1081D000C40475809852628842F001026280184699
:1081E000F0BCFFF7A6BF46F8045BE1E72DE9F74FC7
:1081F0009946D37814466F2BA3F1410206460F46E9
:1082000001922DD028D8582B14BF0A251025DDF84F
:108210003080AA464FF0000B52465B463046394646
:10822000F7F76EFF092AD3B21FD830335F45DBB2B0
:1082300008BF564508F8013D01D3C84512D8237838
:108240009B0605D5082D16D1A37843F00803A3702B
:10825000404603B0BDE8F08F03F0F703702BD3E77F
:108260000825D4E706460F46D6E7019A192A94BF97
:1082700037335733DAE7102DEAD1A37843F01003F0
:10828000E5E72DE9F0410746884615461E461446A7
:10829000B442A4EB050002D33EB923782BB114F805
:1082A000010B4146B8470028F2DABDE8F0814FF0F3
:1082B00000407047F0B5856986680769044685B156
:1082C000354023683B44981B904228BF10467F1BD3
:1082D0006369B84228BF38461D4406440D60A66055
:1082E000F0BDB6FBF7F507FB1565EAE770B5054687
:1082F0000C46FFF7DCFF6E682B692A6831191A44B7
:1083000091420AD8864292BF0023B0FBF3F0434368
:10831000C91AC5E90111002070BD6FF01500FBE717
:108320002DE9F34180460E46154600272A4601A94D
:108330004046FFF7BFFF314604460246019801F070
:10834000A6FA2D1B2744264401D0002CEED1394635
:108350004046FFF7CBFF384602B0BDE8F0812DE97B
:10836000F041C3684668B34204460F46904606D9BA
:108370000569FFF79CFFB0FBF5F005FB0066A569FA
:10838000E168236985B10D40701A404528BF404619
:108390000646581BB042636928BF30461D4401445D
:1083A0003D60E160BDE8F081B1FBF3F503FB15151D
:1083B000EAE7F8B54768C368BB4205460C4612D9E0
:1083C0000669FFF774FFB0FBF6F0704307442968B5
:1083D0002144B9429FBF091A2960E960002088BF83
:1083E0006FF01500F8BD0020F1E72DE9F34180465C
:1083F0000D4616460027324601A94046FFF7AFFF5B
:1084000004462DB102460199284601F040FA254460
:10841000361B274401D0002CEDD139464046FFF7EA
:10842000C8FF384602B0BDE8F0810B0704D5A0F1C3
:108430004103192B98BF203070472DE9F04F87B0CA
:108440008A4614460293054618B9012007B0BDE8D4
:10845000F08F0029F9D0029B002B00F01A8104F064
:1084600004030A460493A846214618F8010BFFF7B7
:10847000DCFF0346C0B23F281778064624D013F02D
:10848000C00F0AD1C0B12A2835D021463846013262
:10849000FFF7CBFF86421ED0D7E75B287BD05C2856
:1084A000F3D1E307F1D46878FFF7BFFF10F0FF06C0
:1084B00018BF05F10208E8E7E40601D52F2FC5D063
:1084C000381E18BF0120C1E7002FBED02F2F04D1C6
:1084D000A107BAD401324546C5E72E2FFAD1049B35
:1084E000002BF7D05245B0D0A307F3D512F8013CCA
:1084F0002F2BEFD1A9E76878FFF797FFC1B22A29A0
:1085000018D02E2F09D1049B3BB152459DD0A7070F
:1085100003D512F8013C2F2B97D079B914F0020043
:1085200094D0E60600F1B7802F21104601F04FF9F4
:108530000038C6E718F8010F2146DDE72F2921D0C2
:10854000029B16465F1E24F0040904F0020AB3469B
:1085500021469BF80000FFF768FF10F0FF0506F1C9
:1085600001063FF472AF3B464A4659464046FFF784
:1085700064FF01287FF46AAF2F2DE8D1BAF1000F14
:10858000E5D062E7A507DBD5104601F020F90246E9
:108590000028A0D159E7002F3FF457AF2F2F02D169
:1085A000A0073FF552AF21463846FFF73EFF009047
:1085B000B8F1000F3FF449AF6B78212B01D05E2B4F
:1085C00026D1023501230193012304EA03014FF070
:1085D000000B03912E46214616F8010B0593FFF779
:1085E00024FF5FFA80F9B9F15D0F059B13D12BBB16
:1085F000019B5B453FF429AF002E3FF426AF711C71
:1086000003D15B2F7FF421AF46460132B04662E7CB
:1086100045460023D7E7B9F12F0FF2D0B9F15C0F2F
:1086200008D1039B53B968782146FFF7FEFEAE1CC4
:108630005FFA80F9B9F1000F3FF407AF33782D2BC3
:1086400020D170782146FFF7F0FE10F0FF0019D01E
:108650005D2817D05C2806F102050AD1039B43B9B7
:10866000B078FFF7E2FE10F0FF0006F103053FF4DB
:10867000ECAE009B4B4503DB8342D8BF4FF0010BB0
:108680000023A7E7009B35464B4508BF4FF0010B81
:10869000F6E70320DAE60846D8E64023FFF7CDBE2A
:1086A000704708B50020F9F7F1FB08B50120F9F78C
:1086B000EDFB83681B6A03B11847704710B51C4671
:1086C0004368D868FFF791FE2060002010BD2DE9B7
:1086D000F04145681E462B681B7C0C46174653B17B
:1086E00001EB020844452B6820D1D3E90121376012
:1086F0000120904717E0A868FFF712FE2B68306052
:108700000C330121BFF35B8F53E8002F43E80010C7
:108710000028F9D1BFF35B8F2AB92B6818688368EA
:10872000DB6903B198470020BDE8F081186814F8B0
:10873000011B83685B689847D4E743681B6810B5E2
:108740001C682046FFF7B5FFA368DB6A0BB1204623
:108750009847002010BD08B543681B68197411B113
:108760001868FFF7A6FF002008BD2DE9F3418046F9
:108770000D4683685B6C03B19847D8F808305B6B93
:1087800013BB0027E86801A90269FFF793FDD8F839
:108790000830064600282FD09B6901994BB302464A
:1087A000404698470446002CE868214618BF012738
:1087B000FFF79CFD0CB1A642E4D04FB12B6800201E
:1087C000D3E90121904703E0404698470028D8D1DB
:1087D000D8F808305B6ADBB9A86801A90269FFF71D
:1087E000BEFD0446D8B94046FFF763FF2B68DC6046
:1087F00021E06FF05704D6E79B6933B101220DF1F8
:108800000301404698470446D4E76FF05704D1E788
:10881000404698470028DFD102B0BDE8F081D8F883
:10882000083001995B6963B10246404698470146AA
:10883000A868FFF7BEFD2B680120D3E9012190470E
:10884000EAE76FF05701F3E70346BFF35B8F53E8A6
:10885000000F40EA010243E8002CBCF1000FF6D102
:10886000BFF35B8F70470346BFF35B8F53E8000F86
:1088700000EA010243E8002CBCF1000FF6D1BFF37F
:108880005B8F704738B58368D3F86432DB070446E2
:108890001AD4406803685B689847054620B9E068C9
:1088A00000F063FDA3681D71A3685B6B13B12946DB
:1088B00020469847A3680022C3F80C23FEF766FD04
:1088C000BDE83840FBF7F6BE6FF00F05ECE773B577
:1088D0008568090101F51A71044616460D4401AA7E
:1088E0006946284601F071FE009B23B1284601F03D
:1088F00069FE2046B04702B070BDFEF7ABB908B5BF
:1089000010B100F072FF80B208BD0EB403B503AA27
:1089100052F8041B0192FAF753FD02B05DF804EB24
:1089200003B0704708B50B4600F51970042123B158
:10893000FFF78AFFC0F3800008BD6FF00401FFF766
:1089400092FFF7E708B50B4600F51870012123B137
:10895000FFF77AFF00F0010008BD6FF00101FFF79B
:1089600082FFF7E78B6820B903F51A700021FEF744
:108970005FBF03F52670F9E7FEF7EEB8F8B50446D9
:1089800080681F460379022B0D46164607D0BDE8C6
:10899000F8404FF4805100F51970FFF755BF4FF0C4
:1089A000FF324FF0FF3300F53E70FFF7E5FFA3689D
:1089B000D3F86422110504D49B6B13B9204600F050
:1089C0001AFB3B4632462946204600F075FBA36859
:1089D000D3F86422120504D49B6B13B92046FAF72E
:1089E000B9FE606900F044F8A068BDE8F84000F501
:1089F0003E70FFF782BF0CB407B504AB53F8042BED
:108A00000193FFF7BBFF03B05DF804EB02B07047C2
:108A10002DE9F04107460E4614460D460CB9BDE857
:108A2000F081102CA04628BF4FF010082A46A91B41
:108A300043463846FAF75CFCA4EB08044544EDE7EE
:108A400010B5044680684FF0FF324FF0FF3300F559
:108A50003E70FFF791FF2046F9F7F8FDA068BDE8EA
:108A6000104000F53E70FFF748BF83689963704778
:108A7000026983681268016810B50446C0689847A7
:108A8000236900221A6010BD38B5CB681B7C022B0D
:108A900005460C4604D10A2802D10D20FFF7F4FF49
:108AA000236922681B68D554226913680133136057
:108AB0006268934202D12046FFF7DAFF002038BDFA
:108AC000202805D0093804288CBF002001207047D9
:108AD0000120704708B510B100F087FE80B208BDD4
:108AE00010B5047B438922442144B2FBF3F0B1FB6F
:108AF000F3F403FB102003FB1411401A10BD10B552
:108B0000047B438921441019B1FBF3F1B0FBF3F06E
:108B1000401A10BD037B30B544891944B1FBF4F50C
:108B200004FB151101311A440180B2FBF4F3591C06
:108B300004FB1323013501338580C180438030BDA0
:108B40002DE9F84F002506460F4614469846056065
:108B50002078002800F0B580FFF7B2FF18B100239D
:108B600004F8013BF4E73268531C4345336047F88F
:108B7000224000F0A680054694F80090B9F1000F5D
:108B8000E6D0002D40F08980B9F1270F06D0B9F169
:108B90005C0F00F08A80B9F1220F76D12046FFF7F2
:108BA00099FF611C0246204600F05AFE4D46E3E75D
:108BB0002046FFF78FFF611C0246204600F050FE62
:108BC0000025D9E7302925D102234FF0000AE15CC6
:108BD000A1F13002D0B207285FFA83F917D8013328
:108BE00042EACA0A052B5FFA8AFAF0D19946204672
:108BF000FFF770FF09F1FF3BA344821CA2EB0902BF
:108C00002046594600F02CFE04F801ABB4E7B9F158
:108C1000020FECD178293ED102234FF00009E25C2B
:108C2000A2F130015FFA81FCBCF1090FD8B219D86A
:108C300041EA0912032B5FFA82F911D14FF0040BBC
:108C40002046FFF747FF0BF1FF3AA244821CA2EB3C
:108C50000B022046514600F003FE04F8019B8BE70F
:108C60000323DCE7A2F16101052903D8573A42EA60
:108C70000912DFE7A2F14101052901D8373AF6E7E9
:108C8000022808D04FF0030BDAE74846FFF718FF39
:108C900000287FF45DAF01346EE7A94588D0B9F1B3
:108CA0005C0FF8D161788D428CD12046FFF712FF1E
:108CB00004F1010902464946204600F0D1FD4C4628
:108CC0005AE72846BDE8F88FF8B50E461146154616
:108CD000074600F03FFD04462846FFF7FBFE054629
:108CE000C4B1A74207D214F8013C202B02BF0135C2
:108CF000ADB204F1FF342046FFF7ECFE3388421B8F
:108D00005B1B013233806119204692B2BDE8F84006
:108D100000F0A6BDF8BD2DE9F041884686B01746A3
:108D2000044628B10146142201A800F0B0FD01ACB0
:108D3000002631463A462046FAF756FB01360546EC
:108D400028B12968404600F060FD0028F1D128468E
:108D500006B0BDE8F0812DE9F0471C46DDF8208023
:108D60009DF8249000230F46164623602368BB42DB
:108D700005461BD256F8230000F075FB2368824697
:108D800018B1013323602846F0E756F82310424615
:108D90002846FFF7C0FF48B123685A1C2260B9F18A
:108DA000000FE3D08045E1D1236055462846BDE859
:108DB000F0872DE9F8430646FFF78CFE054656BBC3
:108DC000BDE8F8834CB16A1C9BB20137D21AF01986
:108DD00000F046FD2D1BADB24C4608F101081FFA0C
:108DE00088F36A1E93421F46EADAF05DFFF768FED9
:108DF0000028F2D001339BB29AB29542EDD9F05CD3
:108E0000F118FFF75DFE5A1C81460028DAD00134C4
:108E1000A4B21346F0E74FF000084446DFE7F8B588
:108E2000846894F84230054653B9AB689A8FDA8764
:108E3000F8BD013A92B2A28722B984F84220F4E741
:108E400004F14206A28FB31813F8010CFFF738FEA5
:108E500003460028EDD1B0549FB216FA83F1F05DBD
:108E6000FFF72EFE01330028F6D1002FDDD0A38FAF
:108E70000133DA1B304600F0F3FCA38FDB1BA38722
:108E8000D3E70EB403B503AA52F8041B0192FAF714
:108E900097FA02B05DF804EB03B07047026838B58A
:108EA00004461068958F10B100F09FFC80B22268D4
:108EB000528D4319B3FBF2F002FB1030B0FA80F090
:108EC000400938BD826838B504461068D58F10B1A6
:108ED00000F08BFC80B2A268528D4319B3FBF2F014
:108EE00002FB1030B0FA80F0400938BDF8B50446F6
:108EF00080680D46C18F828F20300D44FFF70AFE37
:108F0000A068ADB2C18F2A462030FFF7F8FD0746B2
:108F1000A0682A46C18F2030FFF7E2FD794206465D
:108F20002046FAF793FA31462046FAF7A5FAA368E5
:108F3000DD87F8BD2DE9F8430C1E064632DA64429F
:108F400024B24FF0FF35AFB222E0B368B3F83EE091
:108F5000B3F83C9003F1420800207346A3EB0E01E6
:108F600009B20BB96A1C10D0994501D1012D0CD062
:108F700018F8032042F0200CACF1610CBCF1190F81
:108F80000CD9303A092A09D948B13046FFF7AEFF6B
:108F9000013C24B2631CD8D1BDE8F88301203B44D6
:108FA0009BB2DBE70125CEE78368D98F494209B23E
:108FB000FFF79CBF8368998FDB8FC91A09B2FFF74F
:108FC00095BF8368DB8F1BB14FF0FF31FFF78EBF7A
:108FD00070478368DA8F9B8F9A4202D20121FFF794
:108FE00085BF70478368DA8F9A871344002283F81D
:108FF0004220FAF71FBA10B504468068828FC18FED
:109000002030FFF787FDA368198C2046C1F10101CC
:10901000FAF732FAA368998C20460139FAF716FA62
:109020002046BDE81040FAF705BA2DE9F0410546A3
:1090300086B00F461446002614B906B0BDE8F0818C
:10904000686803682246D3F80C80B9196B46C0479C
:10905000009A1644A41A002AEED1AB6819790329A4
:10906000EAD0022913D803F52673012101A801F0E3
:1090700087FA4FF0FF324FF0FF33012101A8FEF7CE
:109080007BFBA86800F5267001F09CFAD4E7D3F8C2
:1090900064229207FBD5BFF35B8F03F5197353E886
:1090A000002F22F0020243E800210029F7D1BFF38C
:1090B0005B8FC1E7FFF7B9BFF7B50F4681681E4662
:1090C000D1F86032DB060446154617D591F82E30EC
:1090D000BB4213D002222E3101A800F0D8FB394642
:1090E0002046FAF725FA606929463246FAF768F908
:1090F00001A92046FAF73CFA03B0F0BD6069324698
:109100002946FAF75DF9F7E70CB407B504AB53F855
:10911000042B0193FFF7D0FF03B05DF804EB02B01E
:1091200070472DE9F0418668B58FAB18FF2B0746D5
:10913000884614461FDCF38FED1A42331E44ADB24D
:109140002A463146301900F08BFB22464146304614
:1091500000F09DFBBA68938F23449BB2938713441E
:10916000002283F84220BB68D3F86012890704D438
:10917000DA8F1444DC87BDE8F08129463846BDE823
:10918000F041FAF76FBAFFF7CCBF38B583680546F0
:109190009C8FD88F241AA4B28CB142301844224636
:1091A000411C00F05DFBAA68938F611E013B938711
:1091B00028460122BDE8384089B2FAF753BA38BDD3
:1091C00083689A8F10B5044652B1DB8F43B14FF0DC
:1091D000FF31FFF78BFE2046BDE81040FFF7D5BFFB
:1091E00010BD0EB403B503AA52F8041B0192FAF79E
:1091F000E7F802B05DF804EB03B070478369002024
:10920000186070470EB403B503AA52F8041B01920C
:10921000FAF7D6F802B05DF804EB03B07047836844
:10922000BFF35B8F03F5187353E8002F42F002027F
:1092300043E800210029F7D1BFF35B8F002070477E
:109240008368BFF35B8F03F5187353E8002F22F098
:10925000080243E800210029F7D1BFF35B8F00200B
:1092600070478368BFF35B8F03F5187353E8002FD3
:1092700022F0020243E800210029F7D1BFF35B8FFF
:10928000002070478368BFF35B8F03F5187353E8C2
:10929000002F22F0100243E800210029F7D1BFF38C
:1092A0005B8F002070478368BFF35B8F03F51873F3
:1092B00053E8002F42F0080243E800210029F7D1CB
:1092C000BFF35B8F002070478368BFF35B8F03F5AC
:1092D000187353E8002F42F0100243E800210029E0
:1092E000F7D1BFF35B8F0020704708B58368006833
:1092F000D3E900210A6051600022C3E900221989E4
:109300005B8919440C31FFF754F8012008BD002394
:10931000C3607047F8B51F460346164653F8044F1E
:109320009C4202D100203880F8BDC568B1B9002D3B
:10933000F8D0AC4202D10023C360F3E76C68C4608C
:10934000002CEFD0228904F10C01304600F09FFA86
:1093500023893B800022F2540120E5E7002DEED066
:109360008368AB42E7D02C68E9E738B50446051DB1
:109370006368AB4204D02046FFF7B7FF0028F7D15F
:1093800038BD2DE9F74F036802F10C05C5F100085F
:109390001B6908F0030845449D4204468A46174667
:1093A00041D80023C360002A3DD000F10409406881
:1093B00081452DD101934FF0000B20682A4601A969
:1093C000FEF778FF8542064630D920682A4601A973
:1093D000FEF770FF85422AD131462068FEF786FFEE
:1093E000B0441FFA88F82E46019D51462F81A5F8FA
:1093F0000A803A4605F10C0000F049FA63682068DB
:10940000C5E9003931465D606560FEF76FFF0AE02F
:1094100001900028CFD003899342CCD10C3000F0CA
:109420000FFA0028C7D103B0BDE8F08FDCD0206868
:109430000021FEF75BFF6368994508D12068082288
:10944000C0E900BB0021104400F02CFAB5E720462B
:10945000FFF74BFF0028B0D1F0E7031DC0E901334F
:109460000023C360704710B5044608B9002010BD42
:1094700000F0BBF9002380B28342F7D2E25C3F2ABE
:1094800003D02A2A01D00133F6E70120EFE710B517
:10949000044680684FF48072002100F5A17000F04E
:1094A00001FAA068828F00F1420100F5A17000F07E
:1094B000EEF9A06800F5A170FFF77BFCA36813F537
:1094C000A17007D000F091F983B2A2680133A2F82D
:1094D000403010BD0346F8E710B504468068B0F888
:1094E000402000F5A171423000F0D1F9A368B3F833
:1094F00040209A8710BD0022C0E900228260704798
:1095000008B50020F8F7C2FC00F051BD0146006824
:1095100000F04DBD00210120FFF7F6BF08B5FAF7B6
:1095200059FEBDE80840FAF73BBF30B50278202A63
:10953000034600F10100F9D0A2F109010429F5D98F
:109540002B2A08D02D2A0ABF034600210121013B06
:1095500000200A2506E003460021F8E7C2F13002A8
:1095600005FB002013F8012FA2F13004092CF5D9D6
:1095700001B9404230BD2DE9F84384468846014692
:109580000C4614F8013B202B33D0A3F1090004282A
:109590002FD92D2B2FD14B788C1C0121002A5CD088
:1095A000102A09D1302B07D1237803F0DF03582B81
:1095B0004ED163781022023401F10047013F0026AA
:1095C000B7FBF2FE304602FB1E79A3F13005092DF0
:1095D00017D82B469A4224DD751C07D070451DD83C
:1095E00001D14B451ADC00FB0230012614F8013B87
:1095F000EBE72146C4E72B2B04BF4B788C1C0021E2
:10960000CCE743F02005613D192D0AD8A3F14105AF
:109610001A2D34BF372557255B1BDBE74FF0FF368C
:10962000E4E7731C09D1FCF7E5FF22230360384609
:10963000B8F1000F07D1BDE8F88301B14042B8F19D
:10964000000FF8D00EB104F1FF3CC8F800C0F2E7FB
:109650003023002AB0D10822AEE7302BA4D00A2252
:10966000AAE72DE9F04184460F4605462C4614F83A
:10967000013B202B35D0A3F10901042931D92D2B31
:1096800031D16B78AC1C4FF0010E002A5ED0102A4D
:1096900009D1302B07D1237803F0DF03582B50D1A9
:1096A0006378102202344FF0FF310026B1FBF2F153
:1096B00002FB01F86FEA08083046A3F13005092DD6
:1096C00018D82B469A4225DD002E20DB88421ED872
:1096D00001D143451BDC00FB0230012614F8013B9D
:1096E000EBE72546C2E72B2B04BF6B78AC1C4FF091
:1096F000000ECAE743F02005613D192D0AD8A3F1F9
:1097000041051A2D34BF372557255B1BDAE74FF08B
:10971000FF36E3E7002E08DAFCF76CFF2223036034
:109720004FF0FF3047B9BDE8F081BEF1000F00D027
:109730004042002FF7D00EB104F1FF3CC7F800C043
:10974000F1E73023002AAED10822ACE7302BA2D0BB
:109750000A22A8E72DE9F04191F800800546B8F10A
:10976000000F10D04C1C204600F03FF807462E4654
:1097700016F8013B63B1984508D13A462146304678
:1097800000F04FF810B92846BDE8F0813546EEE705
:109790001D46F8E70139034611F8012F0AB91A707E
:1097A000704703F8012BF7E770B5013905462C46E1
:1097B00042B111F8013F561E2BB92A4404F8013B6F
:1097C000A242FBD170BD05F8013B3246EFE7C9B2BA
:1097D00003461A788A42184603F1010304D0002A8E
:1097E000F7D1002918BF00207047034600201A5CFB
:1097F00002B970470130FAE7034600201A5C0AB14B
:10980000884200D170470130F8E7431E013913F850
:10981000012F11F8010F824201D1002AF7D1101A4D
:10982000704730B50024A24208D0035D0D5DAB4205
:1098300002D10134002BF6D1581B00E0002030BDCE
:1098400010B55AB10139841810F8012B11F8013FF5
:10985000A04201D09A42F7D0D01A10BD1046FCE7C2
:10986000431A934210B500EB020308D301390246B4
:109870009A420BD011F8014F02F8014BF8E70A4465
:1098800012F8014D03F8014D8A42F9D110BD10B50F
:10989000431E0A44914200D110BD11F8014B03F858
:1098A000014FF7E7C9B202440346934200D1704723
:1098B00003F8011BF9E74FF0FF3070474B68012BAD
:1098C00007DD0B6818700B6801330B604B68013BB8
:1098D0004B600020704784B004AB03E907009DF89B
:1098E0000430062B08D14FF080430122C3F8002535
:1098F000BFF34F8F20BFFDE704B0704784B004ABC7
:1099000003E90700002383F31188BFF36F8F04B0CE
:1099100070470269CBB20C2103FB0121086C00F0F7
:10992000070070474FF02003EFF3118283F3128892
:10993000BFF36F8F036813F0C00301D08B4207D1D0
:1099400001230360002082F31188BFF36F8F7047FB
:109950004FF0FF30F7E710B54FF02003EFF311821F
:1099600083F31288BFF36F8F036803F00704012CA1
:1099700006D10160002082F31188BFF36F8F10BD04
:1099800003F0C0038B4214BF4FF0FF306FF077003D
:10999000F1E74FF02003EFF3118283F31288BFF356
:1099A0006F8F036803F0C00343F00203036082F388
:1099B0001188BFF36F8F7047006910B4CBB21C24BD
:1099C00003FB0400002110BC10470020FCF7FAB88C
:1099D0000020FCF729B91046FDF784B938B5CCB2A0
:1099E0000C23054663430069403380211844FFF788
:1099F00099FF002805DB696801EBC4046368984798
:109A0000002038BD2DE9F843CDB20C2704696F431F
:109A1000064607F140008021204490469946FFF712
:109A20009AFF002807DB3C44C4E90E89736853F8A9
:109A3000353098470020BDE8F88383685B68184795
:109A400043685B68D3F810350B60002070474368AB
:109A50005B68D3F8040542400A404240C3F804253D
:109A60000020704743685B680020C3F80815704702
:109A700043685B680020C3F80C15704743685A6858
:109A8000D2F804354B40C2F8043500207047036912
:109A9000586830B558B10024814213D108685CB9C8
:109AA0009C685860A14200D198600020086072B99B
:109AB000002030BD2846EFE720609868814208BF4B
:109AC0009C60F2E705680446002DF3D13AB15A686C
:109AD0000A60986859600028EAD19960E9E76FF058
:109AE0001500E6E743681B68D3F80423D10510B4DA
:109AF00018D5D3F82021AAB14FF02001EFF311823D
:109B000081F31288BFF36F8FD3F8201131B1002198
:109B1000C3F82011D3F820110121D96082F31188F4
:109B2000BFF36F8F42685268D2061AD54FF02002F9
:109B3000EFF3118182F31288BFF36F8FD3F85821AE
:109B400012B10022C3F800250269D2680AB1126975
:109B50001AB94FF48002C3F8082381F31188BFF3C8
:109B60006F8F0269D2685AB1D3F8581151B1947B02
:109B70000021116134B14FF48000C3F808039173E0
:109B800010BC7047D3F8241121B10021C3F824116F
:109B9000D3F824311368002BF2D0516810BC184759
:109BA00002690B46D2E9010183E8030000207047F7
:109BB00043681B68D3F88004C3F880047047426888
:109BC0001368D3F8580140B95268920706D4D3F805
:109BD0002001003818BF01207047012070474368FA
:109BE00002691B68D3F8100148B1527D0A70002049
:109BF000C3F81001D3F8102101221A6070474FF00A
:109C0000FF307047002A10B504460FDD43681B681B
:109C1000D3F8100148B122690020C3F81001D3F82D
:109C20001001527D0A700120186010BD0020FCE771
:109C3000436801691A684FF02000EFF3118380F345
:109C40001288BFF36F8FC968002088734FF48001BA
:109C5000C2F8041383F31188BFF36F8F7047036951
:109C6000DB6801229A7370470369DB689A7B02F014
:109C7000FF0162B942681268D2F8580140B1D2F8C7
:109C8000040310F4800003D0196101207047002004
:109C9000704743681B68D3F81001003818BF0120D3
:109CA000704743681B681022C3F804237047436859
:109CB0001B681022C3F80823704743681B684FF4E1
:109CC0000072C3F80423704743681B684FF40072A6
:109CD000C3F808237047012070470369DB68C3E9B4
:109CE0000012704740680368C3F84415C3F848255C
:109CF0000022C3F82021D3F82011C3F85821D3F84B
:109D000058214268D20641BF0822C3F800254FF40B
:109D10008002C3F8042301229A607047F8B50669EF
:109D2000F3689C89BFF35B8F9442A8BF1446054635
:109D30001033012253E8000F002803D143E8002725
:109D4000002FF7D1BFF35B8F0CBF134600231DD04C
:109D50001C462046F8BDF268C85C9268D0540133B6
:109D6000A342F8DB4FF02003EFF3118783F312884F
:109D7000BFF36F8F2846FFF722FFF36840B91861E1
:109D8000044687F31188BFF36F8FE2E70023E7E70C
:109D9000996822462846FFF7A5FFF2E738B54368E1
:109DA0001D68D5F804335B02044605D4D5F80403D6
:109DB00010F0100006D138BDFFF756FF0028F5D08F
:109DC0000120F8E72046FFF764FF003818BF0120A4
:109DD000F1E710B50022044601210220FAF7C4F988
:109DE0000220FAF7A3F92046BDE81040FBF79CBA21
:109DF00010B50022044601212820FAF7B5F92820E1
:109E0000FAF794F92046BDE81040FBF78DBA704789
:109E100008B5FBF7B3FB08BD08B50020FAF76AFDEB
:109E2000FDF78CBE08B5FAF78FF8FAF741F9BDE8EF
:109E30000840FDF783BE004700F069BA08B500206E
:109E4000FAF784F918B9BDE80840FAF76FB908BD08
:109E5000F7B5019001A8DDE9084617461D46FBF756
:109E60005DFF019B002F00EB830014BF0223002342
:109E7000002918BF43F00103002D14BF4FF00C0C54
:109E80004FF0000C002C43EA0C0314BF4FF4E06CBD
:109E90004FF0000C002E43EA0C03D0F8002714BF4B
:109EA0004FF4403C4FF0000C43EA0C0322EA03035A
:109EB00001B109780FB13F787F0019430DB12D78BA
:109EC000AD0039430CB1227814020D430EB136783F
:109ED00036042C433443C0F8004703B0F0BD1FB52F
:109EE0000DF10F03019300238DF80F1000931A4614
:109EF0001946FFF7ADFF05B05DF804FB03680122CA
:109F0000DA60704730B54FF4803400688C4063B13C
:109F10008B0003F5A0730025C550C358C0F8044357
:109F200001F5A87140F8212030BDC0F80843F7E7DB
:109F300070B4046840F20116D4F800528E4025EA4D
:109F40000605C4F80052D4F800522B43C4F800327E
:109F50009DF80C3070BCFFF7D5BFFCF7B7BA08B559
:109F6000FFF7FBFF002008BD704738B1C3681888B1
:109F7000C0F30800A0F5807358425841704740690B
:109F800070B413460D4660B901462A4670BCFCF712
:109F9000D3BA013130F811403444A4B29442F8D914
:109FA000F3E7002147F6FF764FF6FD72F2E7F8B5CA
:109FB00005460E464FF02003EFF3118783F3128816
:109FC000BFF36F8FFDF7E2F9314604462846FFF7ED
:109FD00023FF87F31188BFF36F8F2046BDE8F84059
:109FE000FAF768BB30B50024846141EA020414F03A
:109FF0000304C0E9023201610CD14461A34203D1E0
:10A00000C0E90000002030BD45690D6001344161A8
:10A010001144F3E76FF01500F5E7F8B504460D4677
:10A020004FF02003EFF3118683F31288BFF36F8F95
:10A0300047697FB900F0EFF860B12A684261C0F863
:10A04000B07000F089F8314604F10800BDE8F8402E
:10A05000FCF7E0BE2B6862691A602B686361A36934
:10A06000013BA36186F31188BFF36F8FF8BDEFF357
:10A070000580003818BF0120704778307047FCF722
:10A08000C7BF10B5D0E927420023934202D10B602D
:10A09000002010BDE05CAA28F9D10133F5E708B52E
:10A0A000F9F78EFEBDE80840FFF7B1BE0346002079
:10A0B000C3E90200C3E900337047D0E900321360FE
:10A0C0005A600023C0E90033704708B5FFF7F5FF79
:10A0D000437B23F0020343730023836008BD90F9A0
:10A0E0000E3091F90E00834214BFC01A0020704751
:10A0F00010B54FF02003EFF3118483F31288BFF300
:10A100006F8FFFF7E2FF84F31188BFF36F8FBDE815
:10A110001040183000F0B5B8034620B9EFF30582BF
:10A120000AB9FAF777B883F31188BFF36F8F7047D6
:10A130004FF02003EFF3118083F31288BFF36F8F8A
:10A14000FFF7EABF03460068834203D0002838BF08
:10A15000002070470020704710B54FF02003EFF348
:10A16000118483F31288BFF36F8FFCF719FF84F318
:10A170001188BFF36F8F10BD10B501464FF020035B
:10A18000EFF3118483F31288BFF36F8F10F80B3C49
:10A1900013F0280F0DD151F8103C18380BB1FFF710
:10A1A00094FF11F80B3C23F0140301F80B3CFCF76F
:10A1B000F7FE84F31188BFF36F8F10BD38B50446E6
:10A1C0000D46FCF743FF637B43F002036373B5B1B5
:10A1D0002B68A5609D4208BF0023002B38BF0023D9
:10A1E0009BB194F90E1093F90E20914208D0521AA7
:10A1F000002A05DD5A68C4E9003214605C6038BD8D
:10A200006A68934201D01B68EAE76B68C4E90053AF
:10A210001C606C60F3E738B54FF02003EFF3118555
:10A2200083F31288BFF36F8FFFF78CFF044620B1D2
:10A23000FFF74BFF183000F024F885F31188BFF3C7
:10A240006F8F204638BD38B54FF02003EFF31185EE
:10A2500083F31288BFF36F8FFFF774FF044658B182
:10A26000C0F8B0104261FFF730FF183000F009F875
:10A270002046FCF795FE012085F31188BFF36F8F10
:10A2800038BD10B54FF02002EFF3118482F312882D
:10A29000BFF36F8F03683BB1FDF71AF9002084F319
:10A2A0001188BFF36F8F10BD6FF01500F7E710B581
:10A2B0004FF02003EFF3118483F31288BFF36F8F05
:10A2C000FDF720F984F31188BFF36F8F10BD70B5CF
:10A2D00004460D464FF02003EFF3118683F31288F6
:10A2E000BFF36F8FFDF70EF9012805DDA04203DBF8
:10A2F00029462046FBF7C8FA86F31188BFF36F8F13
:10A3000070BD08B5FDF71EFA08BDFDF71BBA08B110
:10A31000FAF706BB7047142370B503FB0101002454
:10A320000126814200D170BD11F8073C41F80C4C68
:10A3300003F01F03082B0DD806FA03F313F48B7FE9
:10A3400008D051F8143C2BB151F8105C2B605D60C3
:10A3500041E9054482F31188BFF36F8F4FF020036A
:10A36000EFF3118283F31288BFF36F8F1439D8E7AC
:10A37000F8B51746D0E90023904204460D4605D1B2
:10A380006368C5E900431D606560F8BD002BF7D028
:10A39000986800B1603807B1603F3946FFF79FFE0B
:10A3A0000028EDDC2668B442EAD0002E38BF002633
:10A3B000002EE5D0B16801B160393846FFF78FFE55
:10A3C000002805DD7368C5E900631D607560DCE782
:10A3D0006368B342D4D03668EAE72DE9F84F002528
:10A3E0008B4614461F4682462E46A8465D4502DB34
:10A3F0003046BDE8F88F4FF02003EFF3118983F367
:10A400001288BFF36F8F9AF80D3003F01F03013BE2
:10A41000072B0FD8DFE803F01E040E0A0E0E0E25E0
:10A42000DAF810309B682BB1022320E0DAF8103004
:10A430001B688BBB47BB237833B39AF80D3003F00E
:10A440001F03013B072B30D8DFE803F033282F2808
:10A450002F2F2F38DAF810309B68002BEAD0012319
:10A4600005E0DAF810301B6A002BE3D01023DAF88D
:10A470000C20CAF80880C2F345310B4363F3523213
:10A48000CAF80C2084F8008089F31188BFF36F8F1D
:10A4900001350AF1140AA9E70423E8E7DAF8100005
:10A4A000224651461030FFF763FFCAF808400136D4
:10A4B000EAE7DAF8100022465146F4E7DAF810002D
:10A4C000224651462430EEE72DE9F84384680546DC
:10A4D0000E4644B16378012B38D114F8533C13F085
:10A4E00002030AD12370EB68C3F345310E43002009
:10A4F00066F35233A860EB600DE054E90E234FF091
:10A50000FF316FF001008B4208BF824205D100236A
:10A5100023706FF00A00BDE8F883A4F1600840469C
:10A52000FFF7E6FD082E0CBF6FF003030023236541
:10A5300014F8533CDB0602D154F8487C0FB10023D9
:10A54000D0E74046FFF708FE2770CCE7022BF6D194
:10A550002378002BC7D054F8047C002FF4D04FF0A0
:10A560000008A4F1140904F11400FFF78AFEC4F8EE
:10A570002C804946384600F03CF884F80080B2E769
:10A5800010B5D204090201F4F85102F400220A4382
:10A59000017B00240A43C0E90323846010BD034605
:10A5A0000068834208D0D0E9003213605A6000236B
:10A5B000C0E90033FFF788BF70470023C0E90000FF
:10A5C0008360704700238360704783680B60C368B3
:10A5D0001360704710B400F10C04C0E9034410BCD0
:10A5E000FDF7CEBD20B100221146C030FFF72BBED3
:10A5F000704737B5019008464FF02003EFF31185FF
:10A6000083F31288BFF36F8F01A9FDF70FFA044699
:10A6100085F31188BFF36F8F002804DDFCF7BCFEC3
:10A6200008B1FCF70BFE204603B030BD70470000B8
:04A63000FBF78AB9F1
:08A63400FC5AFF7F0100000049
:10A63C009148000000000000D5490000BCA60000B5
:10A64C005F9F000000000000996700000000000000
:10A65C0099780000000000003D4F0000ECA60000BF
:10A66C003D4F0000D4A60000219E00000000000019
:10A67C00F19D000004A70000D39D00001CA7000062
:10A68C00E54D000000000000155700000000000020
:10A69C00C125000000000000259E00000000000005
:10A6AC00BD78000000000000E1090000000000007F
:10A6BC00B6CE000098B0000080B0000078030020F7
:10A6CC00BC0F002040A80000C3CE000008B1000061
:10A6DC00E4B0000080030020181000203AA800000D
:10A6EC00BCCE000018B10000E4B000007C030020D8
:10A6FC002410002034A80000CACE000094B1000041
:10A70C0028B1000084030020EC0000202EA80000DB
:10A71C00D1CE000074B1000028B1000088030020E5
:08A72C00D400002028A8000061
:10A73400C1C5000014000020540700205C00002064
:10A7440002000000D8AD0000640A002000000000F0
:0CA75400CAC50000E0030020A01900208E
:10A760000000000098A800000000000018AE0000E3
:10A7700000000000ACA800000000000014AD0000C4
:10A780000000000080AD000000000000C0A8000034
:10A790000000000004AE0000000000002CAE00002D
:10A7A0000000000028AC0000000000006CB00000B9
:10A7B00000000000D4A8000000000000E8A800008D
:10A7C00000000000FCA800000000000040AE0000F7
:10A7D0000000000054AE00000000000010A90000BE
:10A7E0000000000024A900000000000038A90000BB
:10A7F000000000004CA900000000000060A900005B
:10A800000000000074A900000000000088A90000FA
:10A81000000000009CA9000000000000B0A900009A
:08A8200000000000C4A90000C3
:10A8280000800080FF7F00800080FF7F0080008024
:0EA83800FF7F00800080FF7F00800080FF7F98
:0AA84600FFFFFFFFFFFFFFFFFFFF12
:10A850001B5B4A00001B5B4800001B5B324A000088
:10A860001B5B4A00001B5B6D00001B3700001B38A0
:10A8700000001B5B3F336C00001B5B4800001B5B50
:10A88000324A00001B3700001B38000000000000A7
:10A890000338FDD870470000ACBB0000B3BB00001C
:10A8A00000000000FD7E0000000000008ABB0000E8
:10A8B00094BB000008AC00001D0E0000000000006A
:10A8C00018BC000024BC0000000000007D0C00004B
:10A8D0000000000002BB00000FBB000010AC000035
:10A8E000ED0900000000000033BA000044BA000087
:10A8F000000000006107000000000000CBB900006C
:10A90000D4B90000000000009D0900000000000014
:10A910006DBC00007BBC000000000000BD0D00000D
:10A92000000000006BBA000089BA000000000000BF
:10A93000650B000000000000E5B90000EEB9000062
:10A9400000000000F50B00000000000015BA000038
:10A9500024BA000000000000F10800000000000020
:10A9600064BB000075BB000000000000710A00001D
:10A97000000000002ABB000045BB000000000000F2
:10A98000C90A000000000000F7B9000006BA000084
:10A99000000000004109000000000000D3BB0000DF
:10A9A000E3BB000000000000DD0C00000000000020
:10A9B0004BB900005DB90000000000003D0D000033
:10A9C00000000000D4BA0000E5BA000018AC000096
:10A9D000450C0000000000001BBF000025BF000068
:10A9E000000000002D050000000000004CBF00002A
:10A9F00056BF000000000000090500000000000034
:10AA00007DBF000087BF000000000000E5040000DB
:10AA100000000000A5BF0000AFBF00000000000064
:10AA2000C104000000000000CDBF0000DBBF00003B
:10AA3000000000009D0400000000000012C00000A3
:10AA400020C00000000000007904000000000000A9
:10AA500057C000006AC0000000000000550400005C
:10AA600000000000000000000000000000000000E6
:10AA700000000000000000009BBD0000A3BD00001E
:10AA800000000000D906000000000000B4BD000076
:10AA9000BCBD000000000000BD060000000000007A
:10AAA000CDBD0000D5BD000000000000A1060000E3
:10AAB00000000000E6BD0000EEBD00000000000048
:10AAC0008506000000000000FFBD000007BE00007A
:10AAD00000000000690600000000000018BE000031
:10AAE00020BE0000000000004D0600000000000035
:10AAF00031BE000039BE0000000000003106000039
:10AB0000000000004ABE000052BE0000000000002D
:10AB1000150600000000000062BE00006ABE0000D2
:10AB200000000000F9050000000000007BBE0000EE
:10AB300083BE000000000000DD05000000000000F2
:10AB400094BE00009DBE000000000000C105000092
:10AB500000000000AFBE0000B8BE00000000000012
:10AB6000A505000000000000CABE0000D3BE000022
:10AB7000000000008905000000000000E5BE0000A4
:10AB8000EEBE0000000000006D05000000000000A7
:10AB900000BF000009BF00000000000051050000D8
:10ABA00000000000000000000000000000000000A5
:10ABB0000000000000000000EEBC0000FDBC000032
:10ABC000000000003D0700000000000025BD00005F
:10ABD00036BD000000000000190700000000000062
:10ABE00060BD000071BD000000000000F50600001F
:10ABF0000000000000000000000000000000000055
:10AC0000000000000000000000000000D8A90000C3
:10AC10000000000078AA000000000000B8AB0000AF
:10AC20000080004000040000ABC20000B2C200007F
:10AC300004AD00000000000000000000C2C20000DF
:10AC4000C9C20000000000007120000000000000E8
:10AC5000D8C20000DFC200000CAD00000000000000
:10AC600000000000E7C20000EEC20000000000008B
:10AC70004D1F00000000000008C3000010C30000CA
:10AC800000000000151F00000000000025C30000A8
:10AC90002CC3000000000000E11E000000000000C6
:10ACA0003BC3000043C3000000000000B51E0000CD
:10ACB0000000000000000000000000000000000094
:10ACC000000000000000000053C3000058C3000053
:10ACD00000000000AB8600000000000065C300001B
:10ACE0006AC3000000000000A3860000000000000E
:10ACF0000000000000000000000000000000000054
:10AD000000000000000000003CAC0000000000005B
:10AD1000C8AC0000F9C3000000C4000078AD00001A
:10AD20000000000000000000BCA6000034A70000E6
:10AD300034A7000034A7000034A700002BC4000093
:10AD400010C40000000000001D22000000000000F0
:10AD500032C4000037C400000000000031210000B0
:10AD600000000000000000000000000000000000E3
:10AD70000000000000000000000000003CAD0000EA
:10AD800039C5000040C50000BCAD0000B122000084
:10AD900000000000E0B900007AC5000000000000DB
:10ADA000C1230000020100000000000000000000BC
:10ADB0000000000000000000000000000000000093
:10ADC00094AD00003A0000004007002000000000A1
:10ADD000380000201C0000205B1300201E00000033
:10ADE000B590000034A7000054000020F5250000B5
:10ADF0003B87000057870000CF860000BD8600001B
:10AE000000000000F0C80000AFC800000000000013
:10AE1000A53200000100000074CA00007ACA0000D8
:10AE200000000000293A0000010000002FCA0000C5
:10AE300037CA000000000000E539000001000000F2
:10AE400083C900008AC9000080AE0000B53A000046
:10AE50000101000048CA00004ECA000088AE000090
:10AE600000000000000000000000000098AE00009C
:10AE700000000000D4AE00000000000010AF000091
:10AE8000000000004CAF00000000000074AF0000A4
:10AE900000000000D8AF0000E1CB0000EBCB0000C9
:10AEA00000000000419200000100000023CC0000DF
:10AEB0002ACC000000000000A79200000100000062
:10AEC0000000000000000000000000000000000082
:10AED0000000000016C9000018CD000000000000AE
:10AEE000859200000100000068BA000030CD00002B
:10AEF00000000000C99200000100000000000000F6
:10AF00000000000000000000000000000000000041
:10AF100016C90000C6CC00000000000063920000CB
:10AF20000100000068BA000005CD0000000000002C
:10AF30001F9200000100000000000000000000005F
:10AF400000000000000000000000000088CA0000AF
:10AF500090CA000000000000A539000001000000B8
:10AF600000000000000000000000000000000000E1
:10AF700000000000D4CA0000E3CA000068AE000070
:10AF8000000000000000000093CB00009ACB0000FE
:10AF900070AE00000000000000000000B1CB000017
:10AFA000B6CB000078AE00005D3A00000101000061
:10AFB000C9CB0000CFCB000090AE00000000000025
:10AFC0000000000000000000000000000000000081
:10AFD000000000000000000061CC000067CC000011
:10AFE00000000000FD9100000100000095CC000071
:10AFF0009ACC000000000000CD39000001000000E4
:10B000000000000000000000000000000000000040
:10B01000000000000000000001950000E93F000072
:10B02000A13F000059400000553F0000A000002053
:10B030008800002098000020000000009000002000
:10B04000000000200000000000000B0602000000CD
:10B0500054B0000000000000F1CD000026000207FF
:10B0600000000020F9CD000022000B117ECE000070
:10B0700090CE0000D0B000006D4B0000000000003A
:10B08000694C0000DD990000059A000000000000F6
:10B090001399000000000000B54A0000454B000075
:10B0A000CB990000D1990000A8CE0000AFCE0000DF
:10B0B000000000006D4B00000100000000000000D7
:10B0C0000000000000000000000000000000000080
:10B0D00000000000A8B000007D49000035490000D4
:10B0E00000000000754F0000419A00004F9A0000D8
:10B0F000659A0000719A00007D9A0000694E000078
:10B100008F9A000000000000FFFFFFFF00000050CA
:10B110000000000000000000FFFF000000030050DE
:10B120000000000001000000DF9B000055520000FD
:10B13000B19B0000D1500000A19B00001D9D0000AC
:10B14000059C0000319C00005F9C0000699C000091
:10B15000A39C0000AF9C0000699C0000939C000031
:10B16000BB9C0000C99C00009D9D0000D79C000076
:10B17000DB9C0000002000400200000000000000F6
:10B180000D0000000E000000050000000700000098
:10B1900001010000008002400200000000000000E9
:10B1A0002200000021000000FFFFFFFFFFFFFFFF64
:10B1B000010000003CA6000094A600009CA6000030
:10B1C000B4A60000BCA60000F5FFFFFFFF8FFFFF45
:10B1D000FF8FFFFFFE8FFFFFFE8FFFFFFD8FFFFF43
:10B1E000FC8FFFFFFC8FFFFF6D757465785F6672E3
:10B1F00065652063616C6C65642077697468204EB6
:10B20000554C4C20706172616D6574657200000070
:10B2100043616E277420696E697469616C697A652F
:10B22000206D757465782C20776173204E554C4CD9
:10B230000D0A0000436F756C64206E6F74206C6F94
:10B24000636B20706F7765722073617665206D7512
:10B25000746578005374617274696E67205261641A
:10B26000696F2054657374206578616D706C650A30
:10B2700000556E61626C6520746F20676574207480
:10B28000686520436C6F636B206D616E61676572EA
:10B290000A00436C6F636B2072657175657374206F
:10B2A0006661696C65643A2025640A00436C6F63CB
:10B2B0006B20636F756C64206E6F74206265207301
:10B2C0007461727465643A2025640A00436C6F638C
:10B2D0006B2068617320737461727465640A004E38
:10B2E00052465F524144494F5F4D4F44455F494587
:10B2F00045453830323135345F3235304B42495470
:10B30000004461746120726174653A2025730A00FB
:10B310004E52465F524144494F5F4D4F44455F4254
:10B320004C455F4C523530304B424954004E5246EA
:10B330005F524144494F5F4D4F44455F424C455F2A
:10B340004C523132354B424954004E52465F5241C5
:10B3500044494F5F4D4F44455F424C455F324D423B
:10B360004954004E52465F524144494F5F4D4F444D
:10B37000455F424C455F314D424954004E52465F55
:10B38000524144494F5F4D4F44455F4E52465F32F4
:10B390004D424954004E52465F524144494F5F4D21
:10B3A0004F44455F4E52465F314D42495400524131
:10B3B00044494F5F5458504F5745525F5458504F6F
:10B3C0005745525F4E6567343064426D00545820D3
:10B3D000706F7765723A2025730A00524144494FD5
:10B3E0005F5458504F5745525F5458504F5745522D
:10B3F0005F4E6567333064426D00524144494F5F90
:10B400005458504F5745525F5458504F5745525F0C
:10B410004E6567323064426D00524144494F5F547B
:10B4200058504F5745525F5458504F5745525F4EF2
:10B430006567313664426D00524144494F5F54584C
:10B44000504F5745525F5458504F5745525F4E65C5
:10B4500067313264426D00524144494F5F54585045
:10B460004F5745525F5458504F5745525F4E65678E
:10B470003864426D00524144494F5F5458504F5711
:10B4800045525F5458504F5745525F4E656734647C
:10B49000426D00524144494F5F5458504F574552F6
:10B4A0005F5458504F5745525F3064426D005241CF
:10B4B00044494F5F5458504F5745525F5458504F6E
:10B4C0005745525F506F733264426D005241444998
:10B4D0004F5F5458504F5745525F5458504F57453F
:10B4E000525F506F733364426D00524144494F5F65
:10B4F0005458504F5745525F5458504F5745525F1C
:10B50000506F733464426D00524144494F5F545848
:10B51000504F5745525F5458504F5745525F506FE8
:10B52000733564426D00524144494F5F5458504F47
:10B530005745525F5458504F5745525F506F7336BE
:10B5400064426D00524144494F5F5458504F574533
:10B55000525F5458504F5745525F506F7337644293
:10B560006D00524144494F5F5458504F5745525F08
:10B570005458504F5745525F506F733864426D00B6
:10B580005452414E534D49545F5041545445524ECC
:10B590005F3131303031313030005472616E736D53
:10B5A000697373696F6E207061747465726E3A208E
:10B5B00025730A005452414E534D49545F50415433
:10B5C0005445524E5F3131313130303030005452B9
:10B5D000414E534D49545F5041545445524E5F5271
:10B5E000414E444F4D00506172616D6574657273D8
:10B5F0003A0A0044617461207261746520756E6B53
:10B600006E6F776E206F722064657072656361740F
:10B6100065643A2025640A0D0A00545820706F773B
:10B62000657220756E6B6E6F776E3A2025640A0026
:10B630005472616E736D697373696F6E207061749B
:10B640007465726E20756E6B6E6F776E3A2025642E
:10B650000A005374617274204368616E6E656C3ABF
:10B6600020256868750A456E64204368616E6E65C2
:10B670006C3A20256868750A54696D65206F6E20E4
:10B6800065616368206368616E6E656C3A2025753C
:10B69000206D730A44757479206379636C653A2070
:10B6A00025752070657263656E740A0A0052582011
:10B6B00073776565700A0054582073776565700A62
:10B6C00000546865206D6F64756C61746564205406
:10B6D00058206861732066696E69736865640A0042
:10B6E0005265636569766564207061796C6F616429
:10B6F0003A0A004E756D626572206F662070616354
:10B700006B6574733A2025640A0025733A206261E0
:10B710006420706172616D657465727320636F750A
:10B720006E742E0A00556B6E6F776E2061726775AE
:10B730006D656E743A2025730A00466F722025737A
:10B7400020636F6E6669672E6D6F64652063686144
:10B750006E6E656C206D7573742062652062657411
:10B760007765656E20256420616E642025640A007B
:10B770004368616E6E656C2073657420746F20255C
:10B78000640A0053746172742074686520545820F0
:10B79000636172726965720A005374617274207415
:10B7A0006865206D6F64756C617465642054582001
:10B7B000636172726965720A0044757479206379F5
:10B7C000636C65206D7573742062652062657477A3
:10B7D00065656E203120616E642039392E0A00556E
:10B7E0006B6E6F776E20617267756D656E743A204F
:10B7F00025732E0A0025733A2062616420706172FD
:10B80000616D657465727320636F756E740A0043B1
:10B8100068616E6E656C206D757374206265206260
:10B8200065747765656E203020616E642038300A5B
:10B8300000456E64206368616E6E656C207365748C
:10B8400020746F3A2025640A0044656C6179207485
:10B85000696D65206D75737420626520626574770B
:10B8600065656E203020616E64203939206D730A61
:10B870000044656C61792074696D6520736574207E
:10B88000746F3A2025640A00496E76616C69642001
:10B89000444344432076616C75652070726F76690D
:10B8A0006465640A0044434443205644444820737A
:10B8B000746174652025640A5772697465202730A5
:10B8C0002720746F20746F67676C652073746174D0
:10B8D00065206F66204443444320524547300A5751
:10B8E000726974652027312720746F20746F676731
:10B8F0006C65207374617465206F66204443444313
:10B9000020524547310A0044434443207374617414
:10B91000652025640A577269746520273127206FD6
:10B92000722027302720746F20746F67676C650A58
:10B93000005374617274206368616E6E656C20736D
:10B94000657420746F3A2025640A00746F67676C11
:10B95000655F646364635F737461746500546F67EB
:10B96000676C652044434443207374617465203CD4
:10B9700073746174653E2C2069662073746174650C
:10B98000203D2031207468656E20746F67676C6598
:10B990002044432F44432073746174652C206F72DC
:10B9A000206966207374617465203D2030207468BE
:10B9B000656E20746F67676C652044432F44432095
:10B9C00056444448207374617465007072696E74E3
:10B9D0005F7278005072696E7420525820706179DD
:10B9E0006C6F61640073746172745F727800537479
:10B9F0006172742052580073746172745F74785F5E
:10BA000073776565700053746172742054582073A5
:10BA1000776565700073746172745F72785F7377B5
:10BA20006565700053746172742052582073776595
:10BA3000657000706172616D65746572735F7072BC
:10BA4000696E74005072696E742063757272656EEF
:10BA5000742064656C61792C206368616E6E656C1E
:10BA600020616E6420736F206F6E00737461727456
:10BA70005F647574795F6379636C655F6D6F64751E
:10BA80006C617465645F74780044757479206379BF
:10BA9000636C6520696E2070657263656E74202822
:10BAA00074776F20646563696D616C206469676990
:10BAB00074732C206265747765656E203031206167
:10BAC0006E6420393929203C647574795F63796329
:10BAD0006C653E007472616E736D69745F70617441
:10BAE0007465726E005365742074686520747261A9
:10BAF0006E736D697373696F6E20706174746572B3
:10BB00006E006F75747075745F706F776572004F3B
:10BB1000757470757420706F77657220736574200A
:10BB20003C7375625F636D643E0073746172745F31
:10BB300074785F6D6F64756C617465645F63617266
:10BB40007269657200537461727420746865206D47
:10BB50006F64756C617465642054582063617272FF
:10BB60006965720073746172745F74785F63617287
:10BB70007269657200537461727420746865205430
:10BB800058206361727269657200646174615F72EA
:10BB9000617465005365742064617461207261741E
:10BBA00065203C7375625F636D643E0063616E6324
:10BBB000656C0043616E63656C2074686520737703
:10BBC000656570206F7220746865206361727269A8
:10BBD00065720074696D655F6F6E5F6368616E6E3C
:10BBE000656C0054696D65206F6E20656163682027
:10BBF0006368616E6E656C20696E206D73202862CB
:10BC000065747765656E203120616E64203939294D
:10BC1000203C74696D653E00656E645F6368616EAB
:10BC20006E656C00456E64206368616E6E656C20A5
:10BC3000666F722074686520737765657020286967
:10BC40006E204D487A20617320646966666572656E
:10BC50006E63652066726F6D2032343030204D483F
:10BC60007A29203C6368616E6E656C3E0073746176
:10BC700072745F6368616E6E656C00537461727498
:10BC8000206368616E6E656C20666F7220746865F3
:10BC9000207377656570206F722074686520636813
:10BCA000616E6E656C20666F722074686520636FCC
:10BCB0006E7374616E74206361727269657220289C
:10BCC000696E204D487A20617320646966666572EA
:10BCD000656E63652066726F6D2032343030204DA2
:10BCE000487A29203C6368616E6E656C3E00706125
:10BCF000747465726E5F72616E646F6D005365740B
:10BD000020746865207472616E736D697373696FF6
:10BD10006E207061747465726E20746F2072616E33
:10BD2000646F6D2E007061747465726E5F313131B5
:10BD3000313030303000536574207468652074727F
:10BD4000616E736D697373696F6E20706174746571
:10BD5000726E20746F2031313131303030302E002E
:10BD60007061747465726E5F3131303031313030F2
:10BD70000053657420746865207472616E736D6918
:10BD80007373696F6E207061747465726E20746F66
:10BD90002031303130313031302E00706F733864E3
:10BDA000426D00545820706F7765723A202B38200E
:10BDB00064426D00706F733764426D005458207098
:10BDC0006F7765723A202B372064426D00706F7375
:10BDD0003664426D00545820706F7765723A202B9C
:10BDE000362064426D00706F733564426D005458A4
:10BDF00020706F7765723A202B352064426D007099
:10BE00006F733464426D00545820706F7765723AD6
:10BE1000202B342064426D00706F733364426D00D8
:10BE2000545820706F7765723A202B332064426D2E
:10BE300000706F733264426D00545820706F7765E4
:10BE4000723A202B322064426D00706F733064426E
:10BE50006D00545820706F7765723A20302064422C
:10BE60006D006E65673464426D00545820706F77C2
:10BE700065723A202D342064426D006E6567386427
:10BE8000426D00545820706F7765723A202D38202B
:10BE900064426D006E6567313264426D0054582013
:10BEA000706F7765723A202D31322064426D006EDA
:10BEB0006567313664426D00545820706F77657243
:10BEC0003A202D31362064426D006E656732306451
:10BED000426D00545820706F7765723A202D3230D1
:10BEE0002064426D006E6567333064426D005458C3
:10BEF00020706F7765723A202D33302064426D00D8
:10BF00006E6567343064426D00545820706F7765F9
:10BF1000723A202D34302064426D006E72665F31BB
:10BF20004D6269740031204D6269742F73204E6F29
:10BF3000726469632070726F70726965746172797E
:10BF400020726164696F206D6F6465006E72665F58
:10BF5000324D6269740032204D6269742F73204E35
:10BF60006F726469632070726F7072696574617258
:10BF70007920726164696F206D6F646500626C6521
:10BF80005F314D6269740031204D6269742F7320F6
:10BF9000426C7565746F6F7468204C6F7720456EC6
:10BFA0006572677900626C655F324D626974003258
:10BFB000204D6269742F7320426C7565746F6F74C5
:10BFC00068204C6F7720456E6572677900626C65FA
:10BFD0005F6C723132354B626974004C6F6E672052
:10BFE00072616E676520313235206B6269742F7320
:10BFF0002054582C20313235206B6269742F732005
:10C00000616E6420353030206B6269742F7320526A
:10C010005800626C655F6C723530304B6269740039
:10C020004C6F6E672072616E676520353030206B13
:10C030006269742F732054582C20313235206B6282
:10C0400069742F7320616E6420353030206B626913
:10C05000742F732052580069656565383032313568
:10C06000345F3235304B62697400494545452038AC
:10C0700030322E31352E342D3230303620323530BC
:10C08000206B6269742F7300556E657870656374F8
:10C090006564207465737420747970653A20256432
:10C0A0000A006E7266785F74696D65725F696E69A9
:10C0B00074206661696C656420776974683A20252C
:10C0C000640A000000010000000804200804401079
:10C0D000000000000000000020286E696C29004666
:10C0E00061696C656420746F207265626F6F743A69
:10C0F000207370696E6E696E6720656E646C65731F
:10C10000736C792E2E2E0A005A657068797220762B
:10C11000657273696F6E2025642E25642E25640A6E
:10C1200000557074696D653A202575206D730A009D
:10C130005363686564756C65723A20257520736970
:10C140006E6365206C6173742063616C6C0A0054CB
:10C150006872656164733A0A002570204952512063
:10C16000253032642020202020287265616C2073E5
:10C17000697A6520257A75293A09756E7573656443
:10C1800020257A7509757361676520257A75202FDA
:10C1900020257A752028257A75202525290A002A48
:10C1A000004E41002573257020252D3130730A0083
:10C1B000096F7074696F6E733A20307825782C207F
:10C1C0007072696F726974793A2025642074696DA0
:10C1D000656F75743A20256C6C640A00097374618C
:10C1E00074653A2025732C20656E7472793A202587
:10C1F000700A00556E61626C6520746F206465740E
:10C2000065726D696E6520756E75736564207374F3
:10C2100061636B2073697A6520282564290A0A0006
:10C2200009737461636B2073697A6520257A752CB4
:10C2300020756E7573656420257A752C2075736181
:10C24000676520257A75202F20257A752028257589
:10C25000202525290A0A006379636C65733A202535
:10C2600075206877206379636C65730A00257020F8
:10C27000252D31307320287265616C2073697A65D1
:10C2800020257A75293A09756E7573656420257ABB
:10C290007509757361676520257A75202F20257AC9
:10C2A0007520282575202525290A006B65726E6585
:10C2B0006C004B65726E656C20636F6D6D616E64B2
:10C2C00073006379636C6573004B65726E656C20F7
:10C2D0006379636C65732E007265626F6F740052D0
:10C2E00065626F6F742E00737461636B73004C69C9
:10C2F0007374207468726561647320737461636B16
:10C300002075736167652E007468726561647300DF
:10C310004C697374206B65726E656C20746872650D
:10C320006164732E00757074696D65004B65726E83
:10C33000656C20757074696D652E00766572736921
:10C340006F6E004B65726E656C2076657273696FF7
:10C350006E2E00636F6C6400436F6C6420726562C4
:10C360006F6F742E007761726D005761726D20726D
:10C3700065626F6F742E005B25705D002020726512
:10C380007175697265733A2025730A0052454144FC
:10C39000590044495341424C454400646576696301
:10C3A00065733A0A002D2025730020282573290A79
:10C3B000002D2025730A00505245204B45524E4512
:10C3C0004C20313A0A002D204E6F6E650A00505203
:10C3D00045204B45524E454C20323A0A00504F53AF
:10C3E000545F4B45524E454C3A0A004150504C491F
:10C3F000434154494F4E3A0A0064657669636500CB
:10C4000044657669636520636F6D6D616E6473006A
:10C410004C69737420636F6E66696775726564201A
:10C4200064657669636573206279206C6576656CF6
:10C4300073006C697374004C69737420636F6E666B
:10C440006967757265642064657669636573005514
:10C4500073696E6720646174612077696474682011
:10C4600025640A00496E636F7272656374206461AB
:10C4700074612077696474680A005265616420768B
:10C48000616C756520307825780A00577269746987
:10C490006E672076616C756520307825780A0064B7
:10C4A00065766D656D206C6F616420737570706F5B
:10C4B0007274732073657474696E67206279706139
:10C4C0007373206F6E20612073696E676C652069DD
:10C4D0006E7374616E63652E0A004C6F6164696EE1
:10C4E000672E2E2E0A7072657373206374726C2D22
:10C4F00078206374726C2D7120746F206573636192
:10C5000070650A002D2D002D6500556E6B6E6F77DE
:10C510006E206F7074696F6E20222573220A004EA0
:10C52000756D626572206F66206279746573207222
:10C530006561643A2025640A006465766D656D0066
:10C54000526561642F7772697465207068797369C8
:10C5500063616C206D656D6F7279226465766D65BF
:10C560006D2061646472657373205B7769647468BD
:10C57000205B76616C75655D5D0055736167653A3A
:10C580000A6465766D656D206C6F6164205B6F7009
:10C5900074696F6E735D205B616464726573735D53
:10C5A0000A4F7074696F6E733A0A2D65096C69746D
:10C5B000746C652D656E6469616E2070617273655F
:10C5C00000756172743A7E2420007368656C6C5F3C
:10C5D0007561727400537562636F6D6D616E647323
:10C5E0003A0A005741524E494E473A204120707254
:10C5F000696E74207265717565737420776173203C
:10C600006465746563746564206F6E206E6F74205A
:10C61000616374697665207368656C6C2062616320
:10C620006B656E642E0A006E6F74207465726D699E
:10C630006E617465643A2025630A00506C6561730D
:10C640006520737065636966792061207375626324
:10C650006F6D6D616E642E0A004572726F723A20C2
:10C66000726571756573746564206D756C7469703D
:10C670006C652066756E6374696F6E20657865639E
:10C680007574696F6E730A003A20636F6D6D616E29
:10C6900064206E6F7420666F756E6400546F6F2037
:10C6A0006D616E7920617267756D656E7473206956
:10C6B0006E2074686520636F6D6D616E642E0A0074
:10C6C00025733A2077726F6E6720706172616D65B5
:10C6D00074657220636F756E740A000A2573257382
:10C6E000005368656C6C20746872656164206572C3
:10C6F000726F723A20256400506C6561736520701A
:10C700007265737320746865203C5461623E2062D8
:10C710007574746F6E20746F2073656520616C6C26
:10C7200020617661696C61626C6520636F6D6D611B
:10C730006E64732E0A00596F752063616E20616C00
:10C74000736F2075736520746865203C5461623E88
:10C7500020627574746F6E20746F2070726F6D70CC
:10C7600074206F72206175746F2D636F6D706C65CE
:10C77000746520616C6C20636F6D6D616E647320F5
:10C780006F722069747320737562636F6D6D616E73
:10C7900064732E0A00596F752063616E207472797C
:10C7A00020746F2063616C6C20636F6D6D616E64CB
:10C7B000732077697468203C2D683E206F72203C9E
:10C7C0002D2D68656C703E20706172616D657465B9
:10C7D0007220666F72206D6F726520696E666F726F
:10C7E0006D6174696F6E2E0A000A5368656C6C2067
:10C7F000737570706F72747320666F6C6C6F77698D
:10C800006E67206D6574612D6B6579733A0A20201F
:10C810004374726C202B202861206B65792066722E
:10C820006F6D3A206162636465666B6C6E707577DC
:10C83000290A2020416C7420202B202861206B6560
:10C84000792066726F6D3A206266290A506C6561C4
:10C85000736520726566657220746F207368656CFD
:10C860006C20646F63756D656E746174696F6E20A2
:10C87000666F72206D6F72652064657461696C7398
:10C880002E0A000A417661696C61626C6520636FF3
:10C890006D6D616E64733A0A00253038583A200095
:10C8A000253032782000202020007C007C0A0050B7
:10C8B00072696E7473207468652068656C70206D91
:10C8C0006573736167652E001B5B25642563001B20
:10C8D0005B313B3325646D001B5B34303325646D65
:10C8E000002573252D2A7325733A002D68002D2D00
:10C8F00068656C7000202D20002020004C6F737440
:10C90000206C6F67733A20256C750A005B253364D1
:10C910005D2025730A006F66660025733A2573252E
:10C92000730A0020756E6B6E6F776E207061726196
:10C930006D657465723A20004563686F2073746199
:10C940007475733A2025730A004E6F2072657370F8
:10C950006F6E73652066726F6D20746865207465F4
:10C96000726D696E616C2C20617373756D656420E6
:10C9700038307832342073637265656E2073697A5B
:10C98000650A00726573697A6500436F6E736F6C38
:10C99000652067657473207465726D696E616C20C3
:10C9A00073637265656E2073697A65206F722061AA
:10C9B0007373756D65732064656661756C74206949
:10C9C0006E20636173652074686520726561646FB1
:10C9D0007574206661696C732E204974206D7573BF
:10C9E000742062652065786563757465642061668E
:10C9F0007465722065616368207465726D696E612B
:10CA00006C207769647468206368616E6765207460
:10CA10006F20656E7375726520636F7272656374E3
:10CA2000207465787420646973706C61792E006875
:10CA30006973746F727900436F6D6D616E64206805
:10CA40006973746F72792E007368656C6C0055732E
:10CA50006566756C2C206E6F7420556E69782D6C30
:10CA6000696B65207368656C6C20636F6D6D616EBA
:10CA700064732E00636C65617200436C65617220A3
:10CA800073637265656E2E0064656661756C740013
:10CA9000417373756D65203830206368617273204F
:10CAA00073637265656E20776964746820616E6473
:10CAB0002073656E6420746869732073657474698B
:10CAC0006E6720746F20746865207465726D696E7E
:10CAD000616C2E006261636B73706163655F6D6F83
:10CAE000646500546F67676C65206261636B737087
:10CAF000616365206B6579206D6F64652E0A536FE5
:10CB00006D65207465726D696E616C73206172650C
:10CB1000206E6F742073656E64696E672073657034
:10CB200061726174652065736361706520636F6411
:10CB30006520666F72206261636B7370616365204C
:10CB4000616E642064656C65746520627574746FD1
:10CB50006E2E205468697320636F6D6D616E642062
:10CB6000666F72636573207368656C6C20746F20E8
:10CB7000696E746572707265742064656C65746545
:10CB8000206B6579206173206261636B73706163F0
:10CB9000652E00636F6C6F727300546F67676C650E
:10CBA00020636F6C6F7265642073796E7461782E88
:10CBB000006563686F00546F67676C652073686514
:10CBC0006C6C206563686F2E00737461747300531E
:10CBD00068656C6C20737461746973746963732E17
:10CBE000006261636B7370616365005365742064F8
:10CBF0006966666572656E74206573636170652031
:10CC0000636F646520666F72206261636B7370612D
:10CC1000636520616E642064656C657465206B6576
:10CC2000792E0064656C65746500536574207468C2
:10CC3000652073616D652065736361706520636F46
:10CC4000646520666F72206261636B7370616365F7
:10CC500020616E642064656C657465206B65792E57
:10CC6000007265736574005265736574207368653E
:10CC70006C6C207374617469737469637320666F7C
:10CC80007220746865204C6F67676572206D6F64F1
:10CC9000756C652E0073686F770047657420736844
:10CCA000656C6C2073746174697374696373206656
:10CCB0006F7220746865204C6F67676572206D6FB6
:10CCC00064756C652E0044697361626C65207368DD
:10CCD000656C6C206563686F2E2045646974696EAD
:10CCE00067206B65797320616E64206D6574612DBA
:10CCF0006B65797320617265206E6F742068616E58
:10CD0000646C656400456E61626C65207368656C77
:10CD10006C206563686F2E0044697361626C6520E6
:10CD2000636F6C6F7265642073796E7461782E0026
:10CD3000456E61626C6520636F6C6F726564207311
:10CD4000796E7461782E001B5B366E00436F6D6DDB
:10CD5000616E642062756666657220697320746F07
:10CD60006F2073686F727420746F20657870616EC5
:10CD70006420616C6C20636F6D6D616E6473206DF7
:10CD800061746368696E672077696C64636172645B
:10CD9000207061747465726E3A2025730A006D7597
:10CDA0007465785F696E69742063616C6C6564207A
:10CDB00077697468204E554C4C20706172616D65C6
:10CDC00074657200436F756C64206E6F7420616CC3
:10CDD0006C6F63617465206D75746578206265663B
:10CDE0006F726520696E697469616C697A696E67D2
:10CDF00000464C4153485F30005352414D5F300074
:10CE00000000010000006E6F742000484620636C33
:10CE10006F636B3A0A00092D20257372756E6E6977
:10CE20006E67202875736572733A202575290A008C
:10CE3000092D206C6173742073746172743A20251B
:10CE400075206D7320282575206D732061676F290B
:10CE50000A00092D206C6173742073746F703A207E
:10CE60002575206D7320282575206D732061676FEF
:10CE7000290A004C4620636C6F636B3A0A006E729D
:10CE8000665F636C6F636B5F636F6E74726F6C0071
:10CE9000436C6F636B20636F6E74726F6C20636F93
:10CEA0006D6D6D616E64730073746174757300539E
:10CEB000746174757300434C4F434B004750494FA6
:10CEC0005F31004750494F5F3000554152545F3148
:10CED00000554152545F3000000000000001010085
:10CEE000000000005465726D696E616C005254540C
:10CEF000005345474745520069646C652025303230
:10CF000064006D61696E00756E6B6E6F776E007098
:10CF1000656E64696E670070726573746172740027
:10CF2000646561640073757370656E646564006444
:10CF3000756D6D790061626F7274696E67007175ED
:10CF4000657565640076322E372E39392D6E637320
:10CF5000312D31002A2A2A20426F6F74696E6720B2
:10CF60005A6570687972204F53206275696C64202D
:10CF70002573202573202A2A2A0A00737973776F74
:04CF8000726B71005F
:10CF840000030000500000000A000000320000000E
:10CF9400617F0000ECAD0000C8AD0000000000009F
:10CFA400000000000000000000000000400000003D
:10CFB4008835002000000000000000000000000090
:10CFC4000000000000000000080000008035002080
:10CFD4000000000000000000010000006C000020C0
:10CFE400000000000000000000000000000000003D
:10CFF400000000000000000000000000000200002B
:10D0040080330020000000008C0300200100000099
:10D01400A003002001000000B40300200100000070
:10D02400C803002001000000B798000000000000C1
:10D03400000000007A13002020000000000000001F
:10D0440000000000000000009A13002020000000EF
:10D05400000000000000000000C201000001030005
:10D06400AC000020000000000000000000000000F0
:10D0740000C2010000010300C00000200000000005
:10D08400000000000090D003000000000000000039
:10D09400000000000000000000000000000000008C
:10D0A400000000000000000000000000000000007C
:10D0B400000000000000000000000000000000006C
:10D0C400000000000000000000000000000000005C
:10D0D400000000000000000000000000000000004C
:10D0E400000000000000000000000000000000003C
:10D0F4000000000000000000FF000000000000002D
:10D1040000000000FFFF0F008801002088010020BC
:10D11400900100209001002000000000757B0000B9
:10D1240040110020110000003D7C0000E97B00005C
:10D13400597C0000117C0000DC010020A0010020CB
:10D14400D401002000000000CC0100204411002084
:10D154001100000048110020110000004C110020B3
:10D1640011000000BC010020C8010020C001002003
:08D17400B8010020EC010020CD
:10D17C00B55C0000379E0000000000001595000013
:10D18C001CA70000E59A00000000000015950000A7
:10D19C00000000001595000000000000159500002F
:10D1AC00F5610000379E000000000000159500009E
:10D1BC0000000000816400000000000015950000D4
:10D1CC0000000000159500000000000015950000FF
:10D1DC0000000000159500000000000015950000EF
:10D1EC0000000000159500000000000015950000DF
:10D1FC000000000015950000000000009957000089
:10D20C0000000000159500000000000015950000BE
:10D21C0000000000159500000000000015950000AE
:10D22C00000000001595000000000000159500009E
:10D23C00000000001595000000000000159500008E
:10D24C00000000001595000000000000159500007E
:10D25C00000000001595000000000000159500006E
:10D26C00000000001595000000000000159500005E
:10D27C00000000001595000000000000159500004E
:10D28C00000000001595000000000000159500003E
:10D29C00000000001595000000000000159500002E
:10D2AC00000000001595000000000000159500001E
:10D2BC0004A70000E59A000000000000159500008E
:10D2CC0000000000159500000000000015950000FE
:10D2DC0000000000159500000000000015950000EE
:10D2EC0000000000159500000000000015950000DE
:10D2FC000000000000000000000000000000000022
:04D30C00000000001D
:10D310008C0300208C0300200000000000000000AF
:10D320000E000000A0030020A00300200000000069
:10D33000000000000E000000B4030020B403002031
:10D3400000000000000000000E000000C8030020E4
:10D35000C803002000000000000000000E000000D4
:04000003000045CDE7
:00000001FF
